:020000040800F2
:10000000F0FF0010A18805088515050869D80108CA
:10001000418905084189050841890508000000005B
:100020000000000000000000000000008915050825
:100030008D150508000000009115050829A7010885
:100040004189050841890508418905084189050854
:10005000418905084189050821AF000829AF00083A
:1000600031AF000839AF000841AF00085DAC0008AF
:1000700071AC000885AC000899AC0008ADAC000874
:10008000C1AC0008D5AC00084189050841890508C4
:1000900041890508418905084189050849AF0008DB
:1000A00045C50008A5C4000855C5000895C400084A
:1000B000CDC40008DDC40008EDC400087DA300081D
:1000C000E5B9000885A30008E9B9000841890508D9
:1000D000418905085DA0010861A1010865A2010828
:1000E00051AF000841890508DD57050865C50008BE
:1000F0001DC5000875C500080DC50008E9AC00085D
:100100004189050841890508FDC4000841890508A1
:1001100069A301086DA401086DDA0008A5DA0008DA
:10012000FDAC000811AD000825AD000839AD000890
:100130004DAD000841890508418905084189050838
:100140004189050841890508418905089515050873
:1001500061AD000875AD000889AD000871A5010802
:100160008DA30008EDB900084189050841890508FB
:100170004189050841890508418905084189050823
:080180004189050841890508C9
:10800000074BD0F8E4105B68D0F8F0205B1A9A4276
:10801000B8BFC0F8F030012380F81C310020704751
:10802000001000E0B74B00EB800270B503EBC20418
:1080300053F832205268B2F814C01CF0010F4FEA16
:1080400080016AD15FFA8CFE1EF0020F3DD0BFF3B3
:108050005F8F257F012D5FFA85FC00F0CC80148BAB
:10806000BFF35F8F0C1803EBC404257F022D00F0D3
:10807000E3800C1803EBC404257F032D06D1A47FF5
:1080800024B193F87940002C40F0E5809488A4B2A4
:1080900044F48064948093F978C001EB000E03EB04
:1080A000CE0E9EF81CE00EF1010EE6450CD1002428
:1080B00083F8794093F87A40002C40F0B680084469
:1080C00003EBC00300225A7670BD1EF0040F5BD193
:1080D0001EF0400E00F0C880158A93F978C0666AD9
:1080E000EDB206F80C505FFA8CFE267F0EF101040B
:1080F00064B2E51CAE4283F87840A44600F02A81C1
:108100000D1803EBC5052D7FAC42C6D10EF1020C54
:108110004FFA8CFC83F878C0BFE7B2F800C02CF4AB
:10812000006C4FEA0C4C4FEA1C4CA2F800C0B2F8AD
:1081300000C01FFA8CFC4CF4806CA2F800C0A57F34
:108140004FF0000C83F878C0002D46D093F879509A
:10815000002D3FD0012483F879400C1803EBC404B0
:10816000247F022C04D11488A4B244F40064148047
:108170000C1803EBC404A47E44F0010414820844E8
:1081800003EBC0031B7F70BDA57F4FF0010C83F88C
:108190007AC0002D6FD093F87950002D70D10C1853
:1081A00003EBC404647F002C00F0AE80148893F8C5
:1081B00078C0A4B244F400740CF1010C14804FFA9E
:1081C0008CF483F87840B2F800C01CF4807FFAD1B8
:1081D000A44662E7E47EFF2CBCD00C1803EBC40479
:1081E000A57E05F0FE051582E27EFF2AC7D0FF229C
:1081F00083F87820C3E7A47F002C3FF430AF93F8D6
:108200007940002C3FF42BAF148824F480642404BC
:10821000240C1480BFF35F8F148B148883F87AC00A
:10822000A4B244F40074148030E7948824F44074B9
:108230002404240C948042E7A47F002C3FF419AF5F
:1082400093F87940002C3FF414AF148824F4806430
:108250002404240C1480948824F480642404240CC2
:10826000948093F978C018E71FFA8CF52D0631D465
:1082700093F978C011E793F87940002C8FD095E7F7
:10828000257F022D15884AD925F480652D042D0CF3
:108290001580158A666A93F978C0EDB206F80C501D
:1082A000666A1488A4B244F4007414805FFA8CFCEB
:1082B000158A0CF1010464B2EDB2355595880CF1C4
:1082C000020CADB24FFA8CF445F4806583F8784027
:1082D000958078E793F978506E1C42D0266A765DD7
:1082E0001682247F05F1010C4FFA8CFC644583F85B
:1082F00078C07FF4D2AE948824F480642404240CE3
:108300009480CAE6281900201488A4B244F480742A
:108310001480012483F8794093F9784053E7ADB293
:1083200045F400751580158A666A93F978C0EDB238
:1083300006F80C505FFA8CFC666A158A0CF1010491
:1083400064B2EDB20CF1030C35554FFA8CF483F89E
:10835000784038E7958825F480652D042D0C9580AC
:10836000CEE6E57E1582A57F83F878E01DB9247FEF
:10837000002C7FF404AF948824F480642404240C3B
:108380009480FCE61B4B01681B4A03F5727C03E0FA
:1083900063452CD053F82C2F9142F9D170B593F846
:1083A00004E0427996450AD0634505D053F82C2F56
:1083B0009142F4D06345F9D14FF0FF3070BD9E4635
:1083C0008468DEF80C50A5424FF0000208D001325C
:1083D000032A0EF10C0EE7D0DEF80C50A542F6D1C0
:1083E000DEF81050C668B542F1D150B270BD4FF002
:1083F000FF3070474CA105080000014030B5EAB1DC
:108400008E464FEA014C034600F1C005002419686E
:108410009A6841EA0C0142EA0E029A60C3E900142C
:108420000C33AB42F3D1D0F8C030C0F8C44043EABB
:108430000E03C0F8C030C0F8C84030BD4FEA014E4E
:108440008C46E0E783691969B3F80CC00A6830B458
:108450009C6822F0010224680A60A28992B222EA92
:108460000C02A281027D04681F2A06D96568203AA1
:1084700008209040284245D0FEE72568082090401B
:108480002842F9D1202000FA02F2A260264A12788E
:10849000002A35D01A7E012A39D0D3F8F4200132CF
:1084A000C3F8F420EFF31181502282F31288586848
:1084B0005C6C026822EA04029C6C2243C9B202602E
:1084C00081F31188D3E90C401A6999681D6C096819
:1084D00014605061D3E90E40546090600024B3F8FA
:1084E000A800D5604C62C862106801242043106067
:1084F0001C7683F8F1408A899B8913439BB28B8158
:1085000030BC7047202000FA02F2E260BEE7002291
:1085100083F8F120D3F8F8000A68013022F0010254
:10852000C3F8F8000A60EBE70400001010B40C4C2C
:108530006368002B11DD002004F1080C0146DCF813
:10854000A03003F1C00259600C339342FBD1636841
:10855000013083420CF5807CF1DC5DF8044B704700
:1085600004000010F0B5494C04EB401C9CF8242496
:1085700002B9F0BD464B4FF08C0E0EFB003E93F857
:10858000DC6493F8DD249EF87E708CF80A749642C1
:108590004FF0000C4FEA40158EF87EC00ED002EB73
:1085A000420C03EBCC0C57009CF8E0C40CF1FF3EEE
:1085B000BEF1010F5CD9BCF1030F53D06019A0F8D4
:1085C0000814EFF31182902383F3128890F80A3491
:1085D000B0F8081443EA41030021D2B29BB280F8FC
:1085E0000A1482F311881A09217882EA13225A4068
:1085F000D9B1D0F82044D0F80C14D4F8A040D2431C
:108600001B019BB202F00F0201208840134304F1CA
:10861000C0015A0013F4004F93B202D162680243C2
:1086200062600C348C42F4D1F0BDD0F82014D0F844
:108630000C04D1F8A0401B0100F110019BB202F024
:108640000F0201208840134304F1C0015A0013F4C3
:10865000004F93B202D16268024362600C34A142BF
:10866000F4D1F0BD02F1010C0CF0030CB445A5D01F
:108670003A4403EBC202131893F8ED1400299DD07D
:108680006319012283F80A2498E700BF0400001050
:1086900028190020704700BF024B03EB401090F8F0
:1086A00025047047040000104368B0F8502010B44F
:1086B0001A83EFF31182502383F312884168446CCC
:1086C0000B6823EA0403C46C2343D2B20B6082F329
:1086D0001188D0E907418268036912681C605961FA
:1086E000D0E909415C60C46A9960B0F86010DC6050
:1086F0000023D1625DF8044B0376704710B4037D0C
:1087000001681F2B09D94C68203B202202FA03F391
:108710001C4215D15DF8044B70470C68202202FA08
:1087200003F31C42F6D00D4A4068002482F840450D
:1087300002685DF8044B22F0010202608B60704712
:10874000064A4068002482F8404502685DF8044B00
:1087500022F001020260CB60704700BF28190020A0
:10876000704700BF0B4890F83C1589B101EB4101FF
:10877000002310B4490000F244501C4650F8232056
:10878000063302B114608B42F8D15DF8044B704798
:10879000704700BF040000100B4890F83C1589B1E9
:1087A00001EB4101002310B4490000F244501C4683
:1087B00050F82320063302B114609942F8D15DF8D5
:1087C000044B7047704700BF040000100120704741
:1087D000034B00EB400003EBC00090F855057047D9
:1087E000040000101F4890F83C35002B39D00022BF
:1087F0002DE9F04300F244531B4E1C4D4FF0500E38
:108800004FF02C0C144607E053F8181B0C6090F83E
:108810003C150132914222DD197C0029F4D05F68B9
:10882000B90AA1F5801105EB010952294FF0FE08A4
:1088300098BF99F8F483EFF311898EF31288796A5F
:108840000CFB08680131C8F86C15B98A89B241F08F
:1088500001015FFA89F8B98288F31188D4E7BDE88D
:10886000F083704704000010281900204CA105086F
:1088700007EE900AB8EE670A704700BFBCEEC00A68
:1088800010EE103A98B2704708B51D2010F006FAA5
:1088900008B183794BB11E2010F000FA08B183793A
:1088A00003B108BD5523C38008BD5523C380F2E73B
:1088B0000D4B0E49DB68DB43C3F30223C3F1040312
:1088C0000122DBB202FA03F301EB000C1B0103F0FF
:1088D000F0038CF80033430900F01F0002FA00F0A7
:1088E00041F82300704700BF00ED00E000E100E028
:1088F000122301480B80704788010020042301489F
:108900000B8070479C0100202048D0F8E837D0F851
:10891000EC2730B59B184FF01A040C8001D11C488D
:1089200030BD1B4AD0F8EA174FF0000E10467546CE
:10893000B3F1204F4FEA137C0CF130040EF1020E1C
:108940002ABF0CF1370C847080F802C0BEF1100F02
:10895000C5704FEA031300F10200E9D1002004467C
:10896000B1F1204F4FEA117303F1300C00F1020016
:108970002ABF373382F812C093740828D4744FEAA0
:10898000011102F10202EBD1014830BD00F0FF1FDE
:10899000A0010020B42282804F224FF4A57C4FF426
:1089A000EB7102814FF487720023A0F802C0C180EE
:1089B0004FF4E17C9621828144220370A0F80AC022
:1089C000C18102824382704782B01F4B0022019214
:1089D0000193019B1D4A04330193019B196893681D
:1089E00003F00C03042B07D0082B0AD0184B194AAC
:1089F000C3F8AC2702B07047154BC3F8AC1702B0F0
:108A000070475368506813F4800F00F03F005368BC
:108A100013D1C3F388130F49B1FBF0F101FB03F34A
:108A20000A4A0B495268C2F3014201325200B3FBB9
:108A3000F2F3C1F8AC3702B07047C3F38813B1FB4F
:108A4000F0F101FB03F3EBE750280040003802404F
:108A5000281900200024F4000123437700207047E8
:108A6000D0E90B2108B583690B4483610AB108463C
:108A70009047002008BD00BF436A1B681B6A5B6803
:108A80005B78024613F0010008BF5077704700BFC3
:108A900070B5224A224C234B94B00546CDE90042E2
:108AA000214A0992A4F108020A922A7F0493201D08
:108AB0000023CDE905039A42CDE90E330B931093C1
:108AC000139314BF0520042011936B6A0C900220AD
:108AD0000122029018688DF80C200E4607928DF83E
:108AE00020208DF834208DF848204EF0F7FD2B7FA4
:108AF00093B1330E04F8073C063C320C330A227063
:108B00006370A670686A69460FF0F0FC6B6A1868BB
:108B10004EF0E4FD14B070BD073CEEE7D820002015
:108B2000C4010020798A0008598A000810B504465B
:108B300094B050220649684651F040FA606A69468E
:108B40000FF0D4FC636A18684EF0C8FD14B010BD75
:108B500094A50508C2628161704700BF2DE9F0410C
:108B60000446406A00681E460F4690464EF0B6FD29
:108B7000237F002B3FD02A4DA0690523EB67030E0E
:108B800085F8453005F146039870020C000A5870CC
:108B90001A703B68C5F888300020D8F80030C5F856
:108BA0009030012E2363C5F8A0002BD0022E20D1D7
:108BB000D8F80420C5F89800796885F89400C5F8BD
:108BC0009C1013441749C5F8A4200120236385F89D
:108BD000A800C5F8AC10144B617F606A03F1140261
:108BE000002914BF194611460FF080FCE36A8BB1CF
:108BF000206BBDE8F0810A4DA0690423EB6705F105
:108C00004503C1E7074B85F89460C5E92630C5F8F0
:108C1000A400E0E7636A18684EF060FDE8E700BF73
:108C200088010020618A0008D4010020704700BF3D
:108C300000B583B081610192049A0093C26201235E
:108C40006A4601A9FFF78AFF03B05DF804FB00BF85
:108C5000043070470D4B93F8B827D3F8B41702448B
:108C6000D2B283F8B82793F8B82708441206C3F89D
:108C7000B40705D593F8B82782F0800283F8B827A7
:108C8000034B012283F8C420704700BF281900203D
:108C9000880100202DE9F047144FD7F8BC57ED0AA2
:108CA0001ED00026B04607F2F479D7F8C037104836
:108CB000D3F828A0C7F8EC87AC19641010234A46F3
:108CC000E102D0470F280BDD0A4B03F1100C53F8DB
:108CD000041B013107D16345F9D12546B542E4DCD7
:108CE000E802BDE8F087661CF8E700BF28190020FD
:108CF000E82000201C2100201C4BD3F80418D3F8D6
:108D000008288A1A322A16D8D3F81C288A4200D397
:108D10007047D3F8102822B31068928810B44469C1
:108D20003231224218BF42835DF8044B08BF0283F0
:108D3000C3F81C18704793F80C28D3F8101802F0E9
:108D4000010219B132B90A68898811830022C3F877
:108D50001C2870470A68898851830022C3F81C28A0
:108D600070473231C3F81C18704700BF2819002023
:108D7000094A92F80C38D2F8102803F001031AB10E
:108D800023B9136892881A83002070471368928869
:108D90005A830020704700BF281900204FF400704C
:108DA000034B1060D3F828380B600020704700BFD9
:108DB00028190020002070470120704701207047CB
:108DC00000207047012143F20102002343F2012CED
:108DD000017202804FF60171FF22A0F804C04381A6
:108DE0008381C38101828274704700BF154BFF22CB
:108DF0004FF0FF3CF0B5C2700271027242724273D2
:108E0000827303F10C076646172516244FF0150EE2
:108E1000002202EB820281189F4200F802E04C70AF
:108E20008D70CE7081F804C00BD093F9062093F8B2
:108E300007E01C7A5D7A93F90A6093F90BC0063358
:108E4000E7E7F0BDE4A505084FF0000C0121022280
:108E5000032380F805C08171C2710372704700BF9F
:108E600000230222037043708370C3700271704745
:108E70002C22022302704370704700BF4FF0010C98
:108E800045210322002380F800C041708270C37026
:108E9000704700BF4FF4F07140F22E4C01804FF448
:108EA0007A71A0F81EC041844FF4FA6C4FF4F5615A
:108EB000A0F820C0818440F2262C41F21231002318
:108EC000A0F81CC0418141F2110C0E210722A0F82C
:108ED00008C080F8261040F2012C4371837143745E
:108EE000438240F2034140F205638270A0F814C04F
:108EF000C182038382767047114A002330B5036034
:108F0000838002F10C054FF448744FF0290E4FF0A6
:108F1000280C03EB430300EB430100F813C081F876
:108F200001E0D3788B70AA428C8008D092F9063089
:108F300092F807C092F808E054890632E9E730BD9C
:108F4000F8A5050884B04FF4E163ADF80430019949
:108F5000ADF80C10BDF80C1081814FF4007C41F28B
:108F600001420023A0F800C0428040F2593C012297
:108F70000093A0F806C08360C28104B0704700BFB0
:108F80002DE9F0430446406A344D006895B00E4622
:108F9000914698464EF0A2FB314B0193314B04931E
:108FA00005F1D0030093217F0223029305F1C8024B
:108FB000012300278DF80C3005920697002936D042
:108FC0008DF834308DF84830CDE90977330ECDE98E
:108FD0000E77CDE9107785F8C9300523CDF82C90B0
:108FE0008DF82070CDF830801397CA350793330C75
:108FF0001D4F2B70330A6B70AE70D7F85C08656A32
:109000000FF096FB637FA88033BB05A928460FF0BD
:109010006DFA636A18684EF061FBD7F860080FF0CC
:1090200087FB636A9880404615B0BDE8F0838DF8F1
:1090300034308DF848300423CDE90911CDE90E1103
:10904000CDE91011CDF82C908DF82010CDF830809E
:109050001391C9350793CAE76946D7E7880100200D
:1090600080210020798A000828190020094910B5BC
:109070004B6C094C43F480434B644022002104F6BE
:10908000640050F0FEFF4FF0FF33C4F8A438C4F87A
:10909000A73810BD003802402819002070B5224BB7
:1090A00093F8DC2493F8DD349A4237D11F4D95F8BC
:1090B0000436E3B195F808461D4B002040F20D3C04
:1090C000B4B19A68998951601668196846F001062A
:1090D0001660A1F848C08A8992B242F480728A81EF
:1090E00095F804260130824203F11803E8DC70BDD4
:1090F0001A68118821F080010904090C11809988EF
:10910000D162118889B241F0800111805462998A3C
:109110009689314389B291819C82E1E74CF0FEFD52
:109120000028C3D170BD00BF281900200400001022
:10913000D42100202DE9F0411E4B93F8DC2493F854
:10914000DD349A422FD11C4F7D68002D12DD384648
:10915000002410F8086BA046013416B1037E012BE1
:109160001CD002691368AC4243F0010300F5807023
:109170001360F1D111F024FBD7F80C46002C0BDD65
:109180000E4A02EBC40411689388888908320343AD
:109190009BB294428B81F6D1BDE8F08180F8F080DB
:1091A000FFF782FADDE74CF0B9FD0028CBD1BDE82E
:1091B000F08100BF281900200400001014060010E0
:1091C0002DE9F04F037D02681F2B83B0044609D9B7
:1091D0005068A3F120052021A940014207D103B026
:1091E000BDE8F08F1068202199400142F7D0514925
:1091F000514D4968C5F8301695F80816A7694F4EC5
:1092000019BB8C2101FB0761D1F88400D1F8FCE087
:10921000D0F800C0DEF80000B1F8888020F001002E
:10922000CEF80000BCF80C1089B221EA0801ACF8B5
:109230000C10297801BB1F2B6FD9A3F1200120232B
:109240008B40D36003B0BDE8F08F8C2101FB076138
:10925000D1F88410D1F810C00868DCF8001021F0B3
:109260000101CCF80010818921F480710904090CF6
:10927000818129780029DED04FF08C0808FB07F89F
:1092800006EB08032E49D3F8FCA0D3F88420019301
:10929000504608F11809D2F800B0894447F058FE4A
:1092A000019BD5F838262649012083F8D000002AF2
:1092B0003AD0BBF800309BB243F08003ABF80030EB
:1092C00008F174084FF0FF334144CBF82C30584676
:1092D00047F0C4FF8C2303FB076600234946C6F80A
:1092E000A030504647F0CAFED6F8FC3016225A602D
:1092F0001A6842F001021A60D6F88420B6F8883065
:10930000126891890B439BB293810A49237D496876
:109310002268C5F834161F2B8FD8202101FA03F3D9
:10932000936003B0BDE8F08F11F04AFA0449C5F824
:109330003806BEE7001000E00400001028190020E5
:10934000A4190020F8B5164D1648174F00214FF408
:109350001A7250F096FE05F688064FF0804105F629
:109360006C043A46002301E054F8332091420BD0BC
:1093700001330E2BF8D100201C354CF0E7FAB54232
:109380000CD055F81C1CECE7084A02EBC3031C3553
:1093900093F84C0D4CF0DAFAB542F2D1F8BD00BFAB
:1093A00028A605086C1E0020000001404CA10508FD
:1093B0002DE9F04111F004FA1F4F204E05464FF001
:1093C00000087C68002C2ADD00231A4607EB0321E5
:1093D000013391F8F9109C4242EA0102F6D142EAC7
:1093E0000804E4B290467368C3F30803A3B9EFF32B
:1093F00011838BB913F0C0FA431BB3F5FA6F02DC8B
:10940000B8F1000FDDD124B10D4B93F86C29542A2B
:1094100009D02046BDE8F08111F0A4F9ECE74446FC
:109420004FF00008DFE7B3F874290132A3F874297C
:109430002046BDE8F08100BF0400001000ED00E010
:1094400028190020BC4B1B780BB9012070472DE96F
:10945000F04FBA4DBA49D5F80428BA4BA1FB021215
:109460005209A3FB023A4FEADA0A0AEB8A0AA2EB94
:109470004A0A85B0B04A5FFA8AF3039302F61C13D6
:1094800002F23C670193002307EB8A0A02F5816927
:109490009846A94BD3F8243A434540F31781D9F8AD
:1094A0001830D9F80460D3E93A34029311F088F9FE
:1094B000029B95F86CC902904FEA860E95F88009D8
:1094C0000EF1085E04F180610EEB431E3939BCF1E8
:1094D000540F0EEB81110EEB801301D1A5F8760924
:1094E000994240F26A811A68002A00F05E811A6C83
:1094F000002A00F07081D3F88020002A00F06D81EE
:10950000D3F8C02003F58073002AE9D1A3EB0E0E37
:1095100099424FEAAE1E40F25081A4EB0E0145295C
:109520004FF0000428BF452103EB81119B462046E4
:1095300026460DE01A6C002A40F0D080D3F8802037
:10954000002A40F0F680D3F8C02003F580732AB9D2
:10955000994206D91A68002AECD04033994200F2A9
:10956000C180112E344640F22C81D6F1150200F153
:1095700028817549029ED1F8D4309E45D5F88439AA
:1095800038BFC1F8D4E0F11A002919DB03F5F42340
:1095900003F590739E4288BF029B6B4988BF0533D9
:1095A000C5F88439684BD3F8D430052B86BF053B0A
:1095B000DBB2002385F880394FF0FF33C1F8D43097
:1095C00042B100FA02F2C4F11404012000FA04F4DA
:1095D00044EA02005D4BC0F3C43203EB8202D2F8CE
:1095E000B81D00F01F0203EB8202D2F8B82D42EA48
:1095F0000131C0F3441203EB8202C0F3842003EB79
:109600008000D2F8B83D41EA0311D0F8B83D41EAF4
:10961000032181EA112383EA131303F00F030F2BB5
:1096200040F0B180B1F5803F80F0AD80BCF1540FC7
:109630004FEA111104D1B5F870390133A5F870392A
:109640003D4AD2F82439B1F5606F03F10103C2F845
:10965000243900F0D480019B998197F85830039801
:10966000834210D0DAF808203B689B1A3B60DAF896
:1096700030207B689B1A7B600023CAF80830CAF848
:10968000303087F858003B6801333B60DAF8083027
:109690000133CAF808304FF6FF73994207D17B684F
:1096A00001337B60DAF830300133CAF83030019B87
:1096B00008F101081433B8F1080F07F15C070AF14B
:1096C0005C0A019309F120097FF4E3AE1A4A0123F1
:1096D000012082F8203A05B0BDE8F08F803399422E
:1096E0007FF63FAF5A469A1A9211541C184A82FBD1
:1096F00004B2A2EBE472012AB8BF01229040012417
:109700001644013A04FA02F210431C4622680AB3D6
:10971000226C002A63D0D4F88020002A61D0D4F8CB
:10972000C02004F58074B2B1A142EFD89B46234615
:109730000EE7C03312E700BF040000102819002014
:109740001F85EB51CDCCCCCC880100204CA1050865
:10975000565555554034A142E8D9E31A9B115A1C7D
:109760002F4B83FB02B3A3EBE273012BB8BF0123A2
:1097700098401E440122013B02FA03F3184323469A
:109780009B462346E4E6BCF1540F2CD0254AD2F880
:1097900024390133C2F82439224AD2F8203901335E
:1097A000C2F820394FF6FF7157E74033A3EB0E0E96
:1097B00099424FEAAE1E3FF6B0AE10B1013885F8BF
:1097C0008009BCF1540F7FF472AFB5F872390133E0
:1097D000A5F872396BE7803398E6C03396E680349B
:1097E000B9E7C034B7E7B5F870390E4A0133A5F8C8
:1097F0007039D2F824390133C2F82439CCE795F80E
:10980000DD3403EB430305EBC303434493F8ED342A
:109810000D2B7FF420AF019A802393771DE700BFC3
:10982000565555550400001010B504464FF04EFE35
:1098300081B22046BDE81040FEF794BE38B50B4D0E
:1098400000EB400005F2445303EBC00393ED027AB2
:10985000D3ED037AE7EE007AC4002C44B0EE670A39
:109860004FF034FED4F84435186038BD04000010C1
:109870000C4AF8B5136855692B4003EA0005556199
:109880007DB1094F0126B5FA85F4C4F11F0407EB39
:10989000840306FA04F4D3F8640803689847A543E0
:1098A000F1D1F8BD003C014028190020038A2DE9C0
:1098B000F047B0F80C901FFA89F919EA03092BD088
:1098C00005460E464FF000474FF00008B9FA89F3FD
:1098D00027FA03F2D24391B21B3B298209EA02091B
:1098E000042B16D8DFE803F0352C231A0300B36AE3
:1098F000002B37D003F1FF3A1FFA8AFAC6F8288006
:10990000746A34B123682046514698476468002C35
:10991000F8D1B9F1000FD9D1BDE8F0877068696B53
:10992000036889B29847B9F1000FCFD1F4E7B06866
:10993000A96B036889B29847B9F1000FC6D1EBE76C
:10994000F068E96B036889B29847B9F1000FBDD19F
:10995000E2E73069296C036889B29847B9F1000FD2
:10996000B4D1D9E7E96A1FFA81FAC9E70A4608B50E
:10997000054920B9054847F097FD034808BD04484C
:1099800047F092FD004808BDB0220020401B0608A9
:10999000681B060810B5044C04480A46214647F0E7
:1099A00083FD204610BD00BFB0220020901B06089A
:1099B00010B5044C04480A46214647F075FD204680
:1099C00010BD00BFB0220020A41B060810B5044C37
:1099D00004480A46214647F067FD204610BD00BFF7
:1099E000B0220020B01B060838B590F82830012BB3
:1099F000044604D0407F40B10023637738BD406AFD
:109A000003681A7B92B9637F0BB9012038BD0A4DF8
:109A10000A49022305F688220EF098FD95F8893A46
:109A200003F0010383F001006377E7E71B6A002B73
:109A3000E9D0002038BD00BF2819002060020020B6
:109A40002DE9F0410446154E90F82800637F144F2D
:109A500006F68828012805D00BB100236377012082
:109A6000BDE8F081606A05682A7B82B9002BF6D0D8
:109A70000223424639460EF069FD96F8893A03F012
:109A800001036377002BEAD094F82800E2E72A6A02
:109A9000002AE8D1002BE2D0EAE700BF2819002015
:109AA00060020020F0B511F0010583B00AD190F8F2
:109AB0002860012E044607D0C368B3F1807F01D926
:109AC0000123237703B0F0BD0A4B476AD3F85C0843
:109AD0000EF02EFEE368B880B3F1807FF2D9B72193
:109AE0008DF80410267733462A46384601A90EF031
:109AF0002DFDE7E7281900202DE9F047089F88464B
:109B000015460021202204461E4650F0BAFA4FB1F5
:109B10003B68E3811B0C23827B687A89E3821B0C00
:109B20006282238340464DF0BBFFEB0619D4431EEF
:109B3000B8B108EB000701E0013B12D317F801CDE3
:109B4000BCF12E0FF8D1C01A421E032AA8BF03226F
:109B5000082B03F1010AA8BF08239146C2441A4604
:109B600006E008280246C246A8BF08224FF00009B6
:109B70004FF0203341462360636004F1080720461C
:109B800050F01CFA174B23815146BB704A463846A9
:109B900050F014FA611EE31D11F801CFACF1610E13
:109BA000BEF1190F9CBFACF1200C81F800C08B42B4
:109BB000F2D1384604F10B0110F8013BA3F1610228
:109BC000192A9CBF203B00F8013C8842F4D118239D
:109BD0002373330CA382E572099B6683E361BDE8BE
:109BE000F08700BF2020200008B548F02DF80C4B6E
:109BF00093F8911D29220129A3F8EA2AA3F8F22A51
:109C000001D0012008BD0748C3F8940D00F12001E0
:109C10004C304BF0BFFB044B002083F8230008BD01
:109C2000281900206402002000ED00E02DE9F04F2B
:109C3000DFF88894D9F80408C9F8080887B0002B21
:109C400000F0DA8001F5FE781344DFF874B4039372
:109C5000164601F12007C24621E0002E64D0D9F853
:109C60003438B34200F0CC80D9F83038B34200F039
:109C7000FF80D9F83838D9F83C18B3424BD8B142F4
:109C800000F29981711A20464BF032FB039B01369A
:109C90009E4207F500770AF5007A00F0AD80D9F80A
:109CA0004058B542A7F12004D7D8751BD9F8508881
:109CB00005F00702EB080492D8F8302002339342F3
:109CC00003D3D8F8382093420BD941461846059360
:109CD0004BF0DEFA059B8046002800F08C81C9F825
:109CE000500898F80420002A40F03481D8F8285011
:109CF000002D00F07981D8F830209B1A049A02EBED
:109D0000C303D8F80C20204602EB43224FF4007125
:109D10004346A847BAE7B142B4D920464FF400728F
:109D2000002150F0AEF9B1E74FF400723146204601
:109D300050F0A7F9802387F89E310C2387F8A231D1
:109D4000D9F83038D44AD9F82818C4F8C631934223
:109D5000C4F8CA1100F33481D04AD14C82FB03020B
:109D60001A44D817C0EB621284FB0254CD4D85FB18
:109D700003C5C0EB2530C2EB821587F8A1015B1B40
:109D8000801020F03F0001330343144487F8A031D2
:109D9000D317C3EBE4142244BF4B87F89F214A1E1C
:109DA0009A4200F31981BD4BBD4883FB0231114437
:109DB000D317C3EB611180FB0140BA4C84FB025402
:109DC000C3EB2433C1EB811487F8A531121B9B1020
:109DD00023F03F0301321343084487F8A431CB1723
:109DE000C3EBE010014487F8A311552387F8DE3157
:109DF000AA2387F8DF3149E7002007B0BDE8F08FDC
:109E00004FF0FF3384F8EC3184F8ED3184F8EE3113
:109E100084F8EF31D9F84838C4F8E8315223237078
:109E200063706123A37084F8E73141230025E37058
:109E300084F8E631722384F8E43184F8E5314FF494
:109E4000F0722946A7F11C0050F01BF95523C7F802
:109E5000D051C7F8D451C7F8D85184F8FE316FF00B
:109E6000550384F8FC5184F8FD5184F8FF310DE767
:109E700000214FF40072204650F003F98A4A03CAC9
:109E800047F81D0CEB2007F8200C582007F81F0C92
:109E9000902047F8191C07F81E0C00230222082105
:109EA000F820E372227307F8131CA273E37307F818
:109EB000102C07F80B0CD9F8300884F82C20D9F8AE
:109EC00028286376121A2262D9F83808D9F83C2873
:109ED000E376121A3F2020764FF0FF30A0763E2026
:109EE000207701206377A377E37784F82D3084F817
:109EF0002E3084F82F30626284F8300084F83130DC
:109F000087F82610802187F82010292187F8221051
:109F1000942187F823100E2187F824100D21634A1D
:109F200087F82510552187F8DE11AA2187F8DF115F
:109F300003CA5F4BC7F82700C7F82B1003CB138861
:109F4000A7F82F309378C7F83200C7F8361087F893
:109F500031309BE64FF400720021204650F091F81A
:109F6000049B002B4ED1D8F84030002B00F0AA8083
:109F7000049AD8F830304F49CDE90022204611220A
:109F8000FFF7BAFDD8F840301A6C002A00F0AD8017
:109F9000049A1B6BCDE90022474911223846FFF78E
:109FA000ABFDD8F8448007F120044FF4E075B8F118
:109FB000000F3FD16AE6F11A20464BF099F965E6A9
:109FC000FF2387F89F3187F8A13187F8A031324B02
:109FD0004A1E9A427FF7E7AEFF2387F8A33187F83E
:109FE000A53187F8A43100E7294620464FF40072D6
:109FF00050F047F84AE6A7F1240343F804BF9A4516
:10A00000FBD143E6D8F84030049AD8F84480002BBE
:10A010000CBF01230223C3EB02154346002B3FF480
:10A0200035AE013D9B6CF9D198464FF40075002B7D
:10A030003FF42CAE25442034234620354446049674
:10A0400098460EE05CF81C1B236BCDF800C0002680
:10A050000196FFF751FDA46C08F12008CCB1A8458A
:10A0600017D02379A44604F11C0E1122A8F1200078
:10A07000002BE7D162792669236B216842F0210227
:10A08000CDE900E6FFF738FDA46C08F12008002CAC
:10A09000E5D1049EFAE500BFFF03FB0083200882A0
:10A0A0008180808097554541C81B0608D41B06084F
:10A0B000E01B0608C01B0608C41B06082819002060
:10A0C000DEADBEEF049BD9F82C18CDE90033204655
:10A0D0000822FFF711FDD8F84480B8F1000F3FF4D3
:10A0E000D5AD3C464FF4F075A4E7049BCDE90033B1
:10A0F00052E700BF144B154910B5044618681B7988
:10A10000206284F82430152204F1250050F00AF86A
:10A110000F4B93F8982D4FF0010E84F83AE012B9E6
:10A1200084F83B2010BD03F69C5CBCE80F00206067
:10A130006160A260E360BCE80F0084F83BE020614E
:10A140006161A261E36110BDEC1B0608F41B060807
:10A1500028190020084B10B5D3F8BC3D18440C4614
:10A16000807D0EF09BFD18B1828803680CB11A83C4
:10A1700010BD5A83FCE700BF2819002010B42A49FB
:10A180002A4A91F804367BB3D2F8AC48A04239D0C1
:10A19000012B29D0D2F8C448844239D0022B23D0D5
:10A1A000D2F8DC48A04235D0032B1DD0D2F8F448B9
:10A1B000A04231D0042B17D0D2F80C49A0422DD0A8
:10A1C000052B11D0D2F82449A04229D0062B0BD060
:10A1D000D2F83C49A04225D0072B05D0D2F85449EB
:10A1E000844208BF07230ED003F1010C81F804C696
:10A1F00003EB430102EBC1025DF8044BC2F8AC086B
:10A20000184670470023DBB218465DF8044B7047D0
:10A210000123F8E70223F6E70323F4E70423F2E738
:10A220000523F0E70623EEE70400001028190020BC
:10A2300038B5424C8C2303FB004393F88B3003B9B1
:10A2400038BD94F8DCC494F8DD349C450ED003EBA3
:10A25000430204EBC20292F8E0E40EF1FF35012D57
:10A260004FEA430246D9BEF1030F3ED08C2202FBD7
:10A270000042A2F87C10EFF31181902383F312883F
:10A28000B2F87C5092F87E3043EA45030025C9B20B
:10A290009BB282F87E5081F3118829491A090D7802
:10A2A00082EA13225A4005B1D2431B019BB202F04D
:10A2B0000F021A4391F808365BBB8C2303FB004462
:10A2C000D1F8283AD4F8040101219847D4F80011B4
:10A2D000B4F888508A8AD4F8FC302A438A825860BD
:10A2E0001A6842F001021A6038BD5D1C05F00305D2
:10A2F0006545BBD0134404EBC303034493F8ED144A
:10A300000029B3D08C2303FB0043012283F87E2075
:10A31000ACE78C2303FB0044D1F8285AD4F88430EE
:10A32000D4F800115B79086903F0FC031844042198
:10A33000A847D4F800318000988138BD2819002042
:10A340000400001043680B4A23F0407323F4807329
:10A3500043F48073436083681A4042F002028260D3
:10A36000C36A0139CAB223F4700141EA0251C162E1
:10A37000704700BFFDF7FFC0704700BF0020FDF72A
:10A3800051BE00BF0120FDF74DBE00BF0220FDF70A
:10A3900049BE00BF10B1036882881A83704700BFAE
:10A3A00010B1036882885A83704700BF10B40469F3
:10A3B0008269E468416814604024D46044690023E1
:10A3C0000C31C2E90433C2E90633C2E90833C2E9F9
:10A3D0000A33C2E90C3393609363516084B1C2695C
:10A3E000E0689363C2E90233C2E90433C2E9063389
:10A3F000C2E90833C2E90A33C2E90C33C2E90001F9
:10A400005DF8044B704700BF436800221A60037D6B
:10A410001F2B08D9203B2022016802FA03F343F0E6
:10A420001803CB6070472022016802FA03F343F05F
:10A4300018038B60704700BF0268136A11B1D969B5
:10A4400001B3143330B49C681D689169DDB14FF4D9
:10A45000806088618D60104640690C6180B15968E8
:10A46000D369D9B10A464FF480619A609961224359
:10A4700012F0010F14BF00224FF400521A621C6147
:10A4800030BC704770478D61064D4FF0FF0C85F86A
:10A4900044C105F5A27500688D60DDE7024A9A6047
:10A4A0009961E4E788010020E82600200168F8B5FA
:10A4B000D1E9042304465568002B49D09861107DEA
:10A4C0005E681F2831D81768202202FA00F040F099
:10A4D0001800B8601A7D1F2A32D91868203A202344
:10A4E00003FA02F242F01802C26000232B603360CC
:10A4F0003368896943F010033360284646F0BEFD97
:10A5000023683046D96946F0B9FD2B68226843F0CC
:10A5100001032B603368526843F001033360938872
:10A520009BB243F003039380F8BD176820382022C4
:10A5300002FA00F040F01800F8601A7D1F2ACCD80B
:10A540001868202303FA02F242F018028260CCE776
:10A55000137D90611F2B1CD81068202202FA03F390
:10A5600043F01803836000232B602B68896943F054
:10A5700010032B60284646F081FD2B68226843F0CB
:10A58000010352682B6093889BB243F002039380CF
:10A59000F8BD1068203B202202FA03F343F01803B1
:10A5A000C360E0E72DE9F0417F4D804E07463C68EF
:10A5B00097F888806368B888012284F824201A8874
:10A5C00022F040021204120C1A802289824223D007
:10A5D000198821F038010904AB424FEA114100F01B
:10A5E000BF80734A934200F0BB800246B2F5807F81
:10A5F000A8BF4FF48072022AB8BF0222002A92FA42
:10A60000A2F2B2FA82F208BF4FF0FF32013A41EAF9
:10A61000C20292B21A802081397BA27A8A420CD07F
:10A620001A8822F003021204120C1A801A8892B2BD
:10A63000002900F092801A80A1721A8892B242F02A
:10A6400040021A80226A9168002900F0A3804FF02E
:10A65000000C1432E64652F8100C8E4400EA060153
:10A6600020B1B1F1805F23D0616909B352F8140CB5
:10A67000143200EA060110B1B1F1805F18D052F82F
:10A680000C1C0CF1010C0029E5D1227B82B1B8F140
:10A69000000F0DD0BCF1010F6FD8BEF1070F6CD8C1
:10A6A0000CEB8C018900226A11440A7B002A64D0D9
:10A6B000226A92684FF00008002A53D0B8F1000FC8
:10A6C00002D098F80C2022B1BA6812B111689288B1
:10A6D0004A83226AD2F800E0226A5168226A9268AC
:10A6E000501E9AB1BEF1000F23D01EF801CB1A897B
:10A6F0009207FCD5A3F80CC01A89D207FCD59A8919
:10A7000092B209B101F8012B0138EBD2236A1B7B0D
:10A71000E3B9236A1B697BB1236AD7F894001B69EC
:10A72000984701280DD0022806D100232362BDE8F6
:10A73000F0814FF0FF0CDAE7D4F82080236A14335D
:10A740002362236A9B686BB16368B7E7BB68002B21
:10A75000DFD01A689B881383DBE742F003026AE7C5
:10A76000420843E7236A1B68DBB1236AD3E900721E
:10A7700022620022C3E9002219E700213846FFF7D0
:10A780005BFEBB6813B11A689B8853833846BDE8EB
:10A79000F0418BE6227B002A8AD0B8F1000F82D1EB
:10A7A00086E72362C3E700BF003800400000FFFFD8
:10A7B000003C004038B5D0F8E0102B4B04465A68F6
:10A7C000D0F8D80071B1131A99420BDC94F8D0304C
:10A7D000C4F8D820012B10D0D4F8D4300133C4F8F9
:10A7E000D43038BDD4F8E430C4F8D8200344C4F8D9
:10A7F000DC3094F8D030012BEED16168201D04F1DB
:10A80000E805EFF3118C102383F3128863681B6A49
:10A810000BB3D4F8F0302A461BB1D3691432002BA5
:10A82000FBD10B6A6BB1996839B9934209D01968A9
:10A8300029B15B6899680029F7D01433F3E7C3E9BD
:10A8400000055FFA8CFC8CF31188D4F8D430013306
:10A85000C4F8D43038BD0D625FFA8CFC8CF31188DB
:10A86000FFF7A0FEB8E700BF001000E02DE9F041BF
:10A87000826992F8DC30012B8AB005464CD0023B4D
:10A88000012B54D892F84C31D2F89C202E4C63F016
:10A890007F0313708669D6F8A030D6F8108003F1D4
:10A8A000010E0FCCEC46ACE80F00D6F89C30CDE999
:10A8B000003E0FCCACE80F0094E8030006F110074F
:10A8C0008CE80300EFF31180102383F312883369BF
:10A8D0001B6A002B2FD0029B6A461BB1D36914322E
:10A8E000002BFBD1D8F8203073B1996839B9934265
:10A8F0000AD0196829B15B6899680029F7D0143328
:10A90000F3E71F60C3F804D0C0B280F31188AA69CE
:10A9100011690B6A002BFCD1D2F8A0305A8852BAC8
:10A92000EA819A8852BA2A82DB885BBA6B8201205C
:10A930000AB0BDE8F081C8F820D0C0B280F3118819
:10A940003846FFF72FFEE2E784AF05082DE9F04116
:10A9500090F8DC30D0F8A050012B8AB0044672D0B9
:10A9600016D8D0F89C304FF0FF321A605A609A60C7
:10A97000DA60D0F8E0300522B3F57A7FC0F8F02035
:10A980007CD8032380F8DC3001200AB0BDE8F081D8
:10A99000023B012BF8D890F84D31D0F89C20524E54
:10A9A00063F07F031370D0F8A030D0F8108003F16B
:10A9B000010E00F110070FCEEC46ACE80F00D4F802
:10A9C0009C30CDE9003E0FCEACE80F0096E80300C6
:10A9D0008CE80300EFF31180102383F312882369BE
:10A9E0001B6A002B73D0029B6A461BB1D3691432D9
:10A9F000002BFBD1D8F8203073B1996839B9934254
:10AA00000AD0196829B15B6899680029F7D0143316
:10AA1000F3E71F60C3F804D0C0B280F31188226945
:10AA2000136A002BFCD16B885BBAA4F8D030AB88DA
:10AA30005BBAA4F8D230EB8801205BBAA4F8D4301A
:10AA40000AB0BDE8F08190F84C2190F84D319B1A86
:10AA50005B100133DBB205EB430235F813305BBA10
:10AA6000A0F8D03053885BBAA0F8D23093885BBA94
:10AA7000A0F8D43001200AB0BDE8F08103691A7B48
:10AA800072B35B6963B390F898304BB390F84C3174
:10AA9000D0F89C20C4F8A40063F07F03137090F8F2
:10AAA0004C1190F84D31D0F8A0201048C4F80401A2
:10AAB0005B1A07330121C4F8FC30D4F89C3084F8C9
:10AAC00000110A44C4E93D3284F8DC105CE7C8F8A0
:10AAD00020D0C0B280F311883846FFF763FD9EE7AF
:10AAE000022384F8DC304FE784AF050801800008BA
:10AAF000D3B2012B23D870B502EB4202114C4FEABE
:10AB0000820E4FF0000C22460EF10805634604E069
:10AB10000133152B11D012F81CCF6045F8D192F8F3
:10AB200001C08C45F4D15659002EF1D0C3EBC303BC
:10AB30000EEB83030433E01870BD002070BD0020CD
:10AB4000704700BFACAF050810B40C4C002304F6EE
:10AB5000C45C01E0152B0CD003EB430201331CF85D
:10AB600002108142F6D122445DF8044B92F9C60DE1
:10AB700070474FF0FF305DF8044B704728190020F4
:10AB8000D3B2022B21D830B502EB4202104D114C4A
:10AB90004FEA820C0CF10C0E2A46002304E001332C
:10ABA000172B10D052F82C4FA042F8D114798C42B8
:10ABB000F5D152F80E40002CF1D02C2202FB03C339
:10ABC0000833E81830BD002030BD0020704700BFBA
:10ABD0004CA1050800000140002838D030B51C4DBC
:10ABE00090F804C0002305F6C45401E0152B2CD0C6
:10ABF00003EB43020133A15C6145F7D12A440468A9
:10AC000092F9C63D90F805E0DAB2022A1DD803EBAE
:10AC10004303104810494FEA830C02460CF10C051F
:10AC2000002304E00133172B0FD052F82C1F8C4265
:10AC3000F8D111797145F5D151590029F2D02C2262
:10AC400002FB03C30833184430BD002030BD7047F9
:10AC5000281900204CA10508000001400348D0F845
:10AC6000583113B100F5A4701847704788010020CF
:10AC70000348D0F87C3113B100F5B670184770471F
:10AC8000880100200348D0F8A03113B100F5C87046
:10AC900018477047880100200348D0F8C43113B129
:10ACA00000F5DA7018477047880100200348D0F893
:10ACB000E83113B100F5EC701847704788010020A7
:10ACC0000348D0F80C3213B100F5FE7018477047F6
:10ACD000880100200348D0F8303213B100F5087025
:10ACE00018477047880100200348D0F8543213B148
:10ACF00000F5117018477047880100200348D0F80C
:10AD0000783213B100F51A70184770478801002097
:10AD10000348D0F89C3213B100F5237018477047F0
:10AD2000880100200348D0F8C03213B100F52C7020
:10AD300018477047880100200348D0F8E43213B167
:10AD400000F5357018477047880100200348D0F897
:10AD5000083313B100F53E70184770478801002092
:10AD60000348D0F82C3313B100F5477018477047EB
:10AD7000880100200348D0F8503313B100F550701B
:10AD800018477047880100200348D0F8743313B186
:10AD900000F559701847704788010020094B0A4A8E
:10ADA000013800EBC00003EB8000116BD0F8483194
:10ADB000064883420CBF4FF400134FF480030B434B
:10ADC0001363704788010020003802400060024091
:10ADD00070B501383C4C3D4D00EBC00C04EB8C0CC5
:10ADE0009646DCF848613A4AAE420CBF4FF4001573
:10ADF0004FF48005166B35431563CCF85811CCF829
:10AE000060313449DCF84C318B424FEAC0023ED00D
:10AE100001F580618B423AD0A1F57A718B4247D01F
:10AE200001F580618B4243D0A1F57A718B4241D00C
:10AE300001F580618B423DD0A1F57A718B4235D00E
:10AE400001F580618B4231D0A1F57A718B4233D00C
:10AE500001F580618B422FD0A1F57A718B422DD004
:10AE600001F580618B4229D0A1F57A718B4227D000
:10AE700001F580618B4223D0A1F57A718B4221D0FC
:10AE8000154D01F580618B4218BF002500E0134D80
:10AE9000104404EB8003CEF38711C3F8685193F894
:10AEA0005D01BDE8704000224CF0D4B80C4DEFE7D6
:10AEB0000C4DEDE70C4DEBE70C4DE9E70C4DE7E7EA
:10AEC0000C4DE5E7044DE3E78801002000600240F7
:10AED00000380240106002400080002820800010EE
:10AEE00000800018008800100080201020800020C2
:10AEF0000088002000802020800AA0F580105228C1
:10AF000008D8054B184490F8F4330D2B02D8034AA7
:10AF1000D0567047002070474CA10508881C0608D1
:10AF20000120FEF7A5BC00BF0220FEF7A1BC00BFB8
:10AF30000420FEF79DBC00BF0820FEF799BC00BFAF
:10AF40001020FEF795BC00BF4FF47870FEF790BC60
:10AF50004FF47C40FEF78CBC30B50C4683B0054600
:10AF600018B3036803F13F4303F57E039B0A104ABD
:10AF7000134413F84C0C4AF0E9FCA988009104F042
:10AF80000303C4F381028DF8043028688DF805208E
:10AF9000C4F300136946C4F341148DF806308DF8EC
:10AFA000074045F027FF03B030BD4FF0FF33DEE729
:10AFB00044B2050800B1CFE7704700BFF8B5CB78C1
:10AFC00013B900252846F8BD00F110070C460646C7
:10AFD000897838460DF0D6FB05460028F1D0E07898
:10AFE0000DF05CFEB06123780133DBB210B1C371A8
:10AFF000222383710921FFF7DDFFB069FFF7CAF94A
:10B000000C4AD2F80438632BFBD90B480DF090FBA7
:10B01000B082384640F038FD074620B9E0780DF0A0
:10B020009DFE3D46CEE7306986F8D8704CF05AFB5D
:10B03000C8E700BF2819002040420F000B4B10B595
:10B04000D3F8BC3D03440446987D0DF027FE60B163
:10B050002E228271621CC2710121FFF7ABFF2046D4
:10B060000021BDE81040FFF775B810BD2819002079
:10B0700070B50E4CD4F8246A002E15DD04F58164F9
:10B08000002503E0B54204F120040DD0237F0135F3
:10B09000002BF7D0E0680028F4D0217DFFF75CFF9B
:10B0A000B54204F12004F1D1012070BD040000106C
:10B0B000F8B5037D85691F2B04464DD90168A3F1BE
:10B0C00020024E6820209040064234D01023934046
:10B0D000C860CB604B68D340DE0700F18380EFF39C
:10B0E0001183502282F312882A6C1168C9075AD43E
:10B0F000516889B271B9D5E90960864250D0AF690B
:10B100000744D76073D9301A80B25060AE62002114
:10B1100085F86410116841F00101DBB2116083F31E
:10B12000118895F86430002B44D1237D1F2B27D93B
:10B130002168A3F120024C6808209040044200D00E
:10B14000C8604C68042000FA02F2224203D0203B7F
:10B1500000FA03F3CB60F8BD02682020166898401F
:10B16000064219460ED010219940906091601168F6
:10B17000D940C807B3D5012101FA03F39360AEE7C4
:10B1800022681946106808238B40184200D093604B
:10B190001068042303FA01F10142DCD09160F8BD8C
:10B1A000012285F86420DBB283F3118895F86430BE
:10B1B000002BBAD095F87C30002BB6D195F87100F1
:10B1C0000DF06CFD2A6E938923F008031B04012106
:10B1D0001B0C938185F87C100028A6D02021FFF756
:10B1E000BBFEA2E7012303FA02F2CA6077E72E69E9
:10B1F000301A80B25060A96289E700BF70B50C4672
:10B2000082B015460646002839D0036803F13F4353
:10B2100003F57E039B0A1B4A134413F84C0C4AF0B7
:10B2200095FBB2880092B2FA82F304F003028DF823
:10B230000420C4F3810230688DF80520C3F11F0398
:10B24000C4F30012C4F341148DF80740C3F3CC04D7
:10B2500000EB840403F007038DF806209B00226AAC
:10B260000F269D4006FA03F322EA03032362226AB3
:10B2700015436946256245F0BDFD02B070BD4FF033
:10B28000FF33C8E744B2050800B1B7E7704700BF15
:10B290002DE9F043774D05EB001683B0D6F8043E58
:10B2A000002B00F0938004464FEA001896F80C0E2D
:10B2B0004AF04CFB96F80C3E590903F01F02032993
:10B2C0004FF0010303FA02F300F09880042900F024
:10B2D000858002297DD005EB0803013493F8080E20
:10B2E0000DF0DCFCE4B2814610B112238371C4710D
:10B2F00005EB080393F8090E0DF0D0FC074610B1DA
:10B300001323C471837105EB080393F80A0E0DF043
:10B31000C5FC064610B11423C471837145444846E8
:10B3200095F80B2E01924A21FFF7AEFF019A38469D
:10B330002A21FFF7A9FF019A0A213046FFF7A4FF4F
:10B34000D5F8042E4C4B9A425DD04C4B9A424AD0D1
:10B350004B4B9A4262D04B4B9A426AD04A4B9A422C
:10B3600072D04A4B9A427AD049499088B1F88A43C0
:10B37000B1F88833B1F892532343B1F88C43234397
:10B38000B1F88E4320F003002343B1F8904300044A
:10B39000000C2343B1F8944390802B43108823433F
:10B3A000B1F89643B1F8981300F441502343034396
:10B3B0009BB21380938B23F400631B041B0C9383B9
:10B3C000118213889BB243F04003138003B0BDE8A1
:10B3D000F083304A516A0B4353627CE72D4A11696E
:10B3E0000B43136177E703F50033196A41F4804199
:10B3F0001962196A21F480411962B5E7254A116A78
:10B400000B43136267E703F58433596A41F48051B3
:10B410005962596A21F480515962A5E703F5FE3358
:10B42000196A41F400411962196A21F40041196254
:10B430009AE703F58233596A41F400515962596A17
:10B4400021F4005159628FE703F56843596A41F4CA
:10B4500080115962596A21F48011596284E703F519
:10B460006443596A41F400115962596A21F4001188
:10B47000596279E728190020003001400038004067
:10B48000003C0040003401400050014000540140A5
:10B490008801002000380240431C00F0A8802DE9FC
:10B4A000F04F00EB8003C44FDA0087B057F80290EA
:10B4B00081000546019107EBC303B9F1000F04D0E9
:10B4C0009C68002C4BD0A17911B107B0BDE8F08F7A
:10B4D000D3F80CA0BAF1000F00F095819AF806306D
:10B4E000002BF2D11832B818D9F80480BB50691C6F
:10B4F000C0E90133C3601523A371C9B21623E171FA
:10B500008AF807108AF8063099F818004AF01EFAEF
:10B51000B8F804302268A18823F440731B041B0C84
:10B52000A8F80430DAF800301183BAF804201A833E
:10B5300011212046FFF710FD11215046FFF70CFDA9
:10B5400009264FF0330B24B12268A188106901420B
:10B5500031D1BBF1010B45D04BF0C0F9F3E7D3F883
:10B560000CA0BAF1000F00F0A4819AF80630002B6D
:10B57000ABD11832BB18D9F80480BC50C3E90144E0
:10B58000DC6016238AF806306B1C8AF8073099F8BD
:10B5900018004AF0DBF9B8F80430BAF8042023F4B4
:10B5A00040731B041B0CA8F80430DAF800301A832F
:10B5B000C2E7A188226851834BF034F92368A2883E
:10B5C0001A834BF02FF9013EBBD1332624B12368F7
:10B5D000A28819690A420DD1013E00F0FB804BF0B0
:10B5E0007DF9F3E7002CE4D14BF01CF9E9E7704753
:10B5F000A28823685A834BF015F9BAF1000F00F0C6
:10B600002481DAF80030BAF804205A834BF00AF9A2
:10B61000002C00F0EE802368A2881A834BF002F918
:10B62000DAF80030BAF804201A834BF0FBF82368EC
:10B63000A2881B691A4240F0A080019B2B4407EBB3
:10B64000C3039A7C002A40F095801A7C1221204680
:10B65000FFF7D4FD019B2B4407EBC3039B7C002B1E
:10B6600000F08F803221BAF1000F07D0019B2B44EC
:10B6700007EBC30350465A7CFFF7C0FD4F4B98457C
:10B6800000F0EF804E4B984500F0F6804D4B98450A
:10B6900000F0FD80019B2B4407EBC3074FF47A7346
:10B6A000BC8A03FB04F4B8F8043023F440731B0491
:10B6B0001B0CA8F80430B8F800309BB243F001032B
:10B6C000A8F80030B8F8045002A845F0DDFB25F0DA
:10B6D0003F0504993C4B2D04A3FB01232D0C45EAA7
:10B6E0009345A8F80450B8F8002022F00102120493
:10B6F000120CA8F80020354A980C9442034642DC0C
:10B700006200B1FBF2F292B20133042A38BF042284
:10B71000A8F82030A8F81C20B8F800309BB243F0FD
:10B720000103A8F80030B8F8003023F4816323F057
:10B7300002031B041B0C4FF4804143F48063A8F800
:10B740000030A8F80810B8F8003023F080031B047C
:10B750001B0C0022A8F8003099F81A0011464BF093
:10B7600079FC002299F81900114607B0BDE8F04FA6
:10B770004BF070BC1A7C322169E7DAF800301B69A3
:10B780005BE712216FE704EB4404B1FBF4F18AB2EA
:10B79000C1F30B0109B942F001020D494FF4967350
:10B7A00000FB03F3A1FB03139B09013342F40042A6
:10B7B000A8F82030AEE700BF281900200054004050
:10B7C00000580040005C004083DE1B43A08601005F
:10B7D000D34D6210002C7FF40BAF4BF023F8BAF17D
:10B7E000000F5FD0DAF80030BAF804205A834BF02B
:10B7F00019F84BF017F8DAF80030BAF804201A8379
:10B800004BF010F826E71832BB18D9F8048047F837
:10B8100002A0C3E901AAC3F80CA01523A371431C1D
:10B82000E37199F818004AF091F8B8F80430A2884A
:10B8300023F440731B041B0CA8F804302368112167
:10B840001A832046FFF788FB7AE64AF0EBFF23686D
:10B85000A2881A834AF0E6FF4AF0E4FF23681B69D6
:10B86000EBE603F5F2331A6A42F400121A621A6A1E
:10B8700022F400121A620DE703F5F0331A6A42F45B
:10B8800080021A621A6A22F480021A6202E703F541
:10B89000EE331A6A42F400021A621A6A22F40002B3
:10B8A0001A62F7E64AF0BEFF4AF0BCFF4AF0BAFF60
:10B8B000D0E61832BB18D9F8048047F802A0C3E9D3
:10B8C00001AAC3F80CA099F818004AF03FF8B8F89C
:10B8D000043023F440731B041B0CA8F804302FE63B
:10B8E0002DE9F84307460EF03DFFDFF84C8007EBEB
:10B8F0008709044608EBC90542F20F7604E00EF012
:10B9000031FF031BB3420ADC6B7E002BF7D108EB3F
:10B91000C90898F8180080F00100BDE8F883B8F86D
:10B92000343E013338469BB2A8F8343EFFF7B4FDED
:10B930000020BDE8F88300BF2819002070B500EB97
:10B940008003274D05EBC30255F833305C68A38AAA
:10B9500084B09BB20393039B13F4706F1CBF01234D
:10B960001376039B13F4E06F4FEA80060CD1A38A91
:10B97000304423F4706305EBC0051B041B0C00224C
:10B98000A3826A7604B070BD238BA38823F48063FE
:10B990001B041B0CA380039B9A05E8D423889B05FA
:10B9A000E5D42388D9050FD52388DA05FCD423886C
:10B9B0009BB243F40073238023889B05FCD4019041
:10B9C000FFF76AFD0198D2E723889BB243F4007326
:10B9D0002380A38823F440731B041B0CA380C6E7B9
:10B9E000281900200020A9E70120A7E70220A5E7E9
:10B9F0002DE9F84F2F4F00EB800407EBC404D4F877
:10BA00000480B8F1000F04D09A46637E03F0FF096A
:10BA100023B14FF000094846BDE8F88F0E46934623
:10BA200005460EF09FFE0A9B7600F6B2C4E9083385
:10BA30000123A67684F81BB084F81D90A37784F8C0
:10BA40001CA0637684F81890B8F804209105064687
:10BA500022D4B8F80030DA0512D442F20F7404E0B0
:10BA60000EF080FE831BA3421ADCB8F800309B0561
:10BA7000F6D4B8F800309BB243F48073A8F80030D5
:10BA8000B8F804309BB24FF0010943F44073A8F8B2
:10BA900004304846BDE8F88F99464846BDE8F88F1F
:10BAA000B7F8343E01339BB22846A7F8343EFFF77F
:10BAB000F3FCB0E728190020F8B590F871301C09A4
:10BAC000013C052C0FD81B4E06EB4402054632F80C
:10BAD000440C03F00F0340FA03F2D20703D595F8A4
:10BAE0007C70012F01D00120F8BD07FA03F3013B60
:10BAF000184034444CF000FD14F8382C0E4C10441F
:10BB000054F8302004EBC0041069A3881840EBD02F
:10BB1000EB6E002285F87C2093F82120204602213C
:10BB2000FFF76CFB2A6E93899BB243F008033846FB
:10BB30009381F8BD44B20508B4230020094BD3F823
:10BB4000382ED3F83C1E40F22A40002350604B624E
:10BB50000B889BB243F001030B80136843F0010391
:10BB600013607047281900201D4B1E48196C1E4A8F
:10BB700010B441F080510124196404625321FF2460
:10BB8000CA205462506251625B6FDB0085B017D4EB
:10BB900016480423002102910290029A1A4402924C
:10BBA000029A04331C2B1160F5D103910390039B7F
:10BBB0000393039B0E4A1A6005B05DF8044B70476F
:10BBC0000A4B002201920193019B0193019A084BB9
:10BBD00012689A42DCD105B05DF8044B704700BF93
:10BBE0000038024000000E4200280040502800406B
:10BBF0003166654210B5174C84B00139002389B213
:10BC0000A042ADF80C30ADF806308DF80E30029140
:10BC100013D0114B984210D003F5804398420CD0BA
:10BC200003F58063984208D003F58063984204D0FE
:10BC30000A4BD3F8AC375B0802E0084BD3F8AC37BB
:10BC4000B3FBF2F201A9013AADF8042045F0B8FACD
:10BC500004B010BD0004014000000140281900207C
:10BC600030B50446006EA268838923F400531B0498
:10BC70001B0C8381637995B013F0040F4FF0000122
:10BC8000019214BF4FF480520A46ADF808201A03FF
:10BC90001B0203F48063ADF80C302379ADF80E106D
:10BCA00002F40052ADF80A20DA0744BF0422ADF8CE
:10BCB0000E209B07ADF8101005D5BDF80E3043F0EF
:10BCC0000803ADF80E3001A945F08CFB6279236EB4
:10BCD000D50700F18B8012F0080F9A8A48D092B2F3
:10BCE00042F008029A829A8992B242F400529A81F2
:10BCF0002279D00732D5E06B002800F0898000233C
:10BD0000E26D0893CDE90C33CDE91033CDE9123360
:10BD10004FF480750A936369E1680E950692079364
:10BD2000626C05924FF480634FF480350B93099158
:10BD30000F9545F00DF905A9E06B45F09FF9E26B11
:10BD4000216E136843F0010313608B8A9BB243F0AA
:10BD500040038B82536822799BB2636591070DD4AF
:10BD6000226E93899BB243F40053938115B030BD8A
:10BD700022F008021204120C9A82B4E7206C002808
:10BD800052D02369A26D0993A36CCDE905324023FB
:10BD900000254FF4803108934FF480630B930F918B
:10BDA000CDE90C55CDE91055CDE9125507950A9509
:10BDB0000E9545F0CDF8206C05A945F05FF9236C90
:10BDC000226E586940F080005861186840F01600F3
:10BDD00018605D60938A9BB243F0800302F10C010E
:10BDE00093820B6843F040030B60BAE71E498B4215
:10BDF00024D0A1F54C418B421ED001F580618B42CD
:10BE00001ED102200121FEF7A5F96279236E62E7B7
:10BE10004FF6DF711980D96841F02001D960D968E7
:10BE200041F01001D96099E7226ED36843F0800396
:10BE300002F10C01D360D4E70120E3E70020E1E741
:10BE400001F580618B420AD001F580618B4208D0F8
:10BE500001F544418B427FF43EAF0520D2E7032039
:10BE6000D0E70420CEE700BF001001402DE9F84FD5
:10BE70004D4C04EB8004D4F82C4A002C7DD0E56EA8
:10BE8000002D76D01F46EB6A6361AB6AA3616B8EAF
:10BE9000E3602B8E23616B682366444B2360444B25
:10BEA000A160A3660646204690460DF021FF94F857
:10BEB00071000CF0F3FE814695F8200094F870B004
:10BEC000A24600284ED10223390784F87C3036D4AC
:10BED00018F0020F10D0B9F1000F0DD00B2389F824
:10BEE0000630731C89F807303B0648D495F82120AA
:10BEF00048462221FFF782F918F0010F04D1E26BC6
:10BF00009AB15046BDE8F88F58460CF0C7FE00289D
:10BF1000F5D00C220136C671827195F821202221BC
:10BF2000FFF76CF9E26B002AEBD195F8241095F835
:10BF3000220089094BF08EF85046BDE8F88F013693
:10BF4000F6B2B9F1000FDAD00B237A0689F8076050
:10BF500089F8063009D595F8212042214846FFF797
:10BF60004DF9CCE749F0F2FCADE795F8212012211C
:10BF7000F4E7AA465046BDE8F88FA246C1E794F818
:10BF800071000CF08BFE226E938923F008031B04D2
:10BF900001211B0C938184F87C100028ACD0202157
:10BFA000FEF7DAFFA8E700BF0400001014B205088E
:10BFB000B9BA0008BFF34F8F0549064BCA6802F4AF
:10BFC000E0621343CB60BFF34F8F00BFFDE700BFBC
:10BFD00000ED00E00400FA0508B50021032045F05B
:10BFE000CFF872B6FFF7E6FF08B5184CD4F8402E2C
:10BFF00094F8460E4AB11168938809690B40F8B964
:10C00000003B18BF0123002BF4D1142010F0D8FE00
:10C0100000BFD4F8403E63B11A689B88116994F858
:10C02000462E0B4042B9003B18BF01230BB1FFF76E
:10C03000D3FFFCF761FEEBE7B3FA83F35B09F5E7A7
:10C04000B3FA83F35B09002BD4D1DEE72819002073
:10C0500008B572B6FFF7AEFF00B583B00D490022F8
:10C0600000920091009B0C330093009B1B68012BF6
:10C0700002D003B05DF804FB01920191019B0649D7
:10C080000C330193019B1A600B6883F308884B689B
:10C090009847FEE7502800400000FF1F38B5FFF723
:10C0A00063FDFFF7D9FF012045F07AF8704A9368E5
:10C0B00023F003039360936813F00C0FFBD1136814
:10C0C0006B49002840D143F00103136041F28833EB
:10C0D0000A6895075BD4013BFAD1664C664D644B08
:10C0E000664AEA60664A596FAA60596B654821F052
:10C0F00080015963596F41F080715967196B41F4A0
:10C10000CE0119635A6B5A639A6B9A631A6C024395
:10C110001A64596C5C4A0A435A640EF0DBFAD4F88C
:10C12000AC375A4AA2FB03239B09013BB3F1807F42
:10C1300009D24FF0E022F02053610021072385F857
:10C1400023009161136138BD43F4803313600A68A2
:10C15000940341F2883304D4013BBED00A689403AF
:10C16000FAD5444C4A4A4B4BB0FBF3F3B0FBF2F028
:10C17000B3EB400F18BF18464FF48002B3FBF0F347
:10C18000C4F85C2EC4F8480EC4F84C3E09E0394CA3
:10C19000002108220223C4F85C1EC4F8482EC4F80B
:10C1A0004C3E022044F0FCFF03280FD83A4BD4F851
:10C1B0004C1E03EBC0008588C2884388C4F8545ED7
:10C1C000B3FBF1F3C4F8582EC4F8503E284B334962
:10C1D0001A6C42F080521A640A6842F440420A60C3
:10C1E0009A689A609A6842F400429A609A6842F4A7
:10C1F000A0529A60D4F85C0ED4F8482ED4F8501EA1
:10C20000024342EA8112D4F8541ED4F8580E490869
:10C2100042EA0062013942EA01425A601A6842F079
:10C2200080721A601A689201FCD51D4A40F20571AD
:10C230001160996821F003019960996841F0020149
:10C24000A2F580629960936803F00C03082BFAD181
:10C25000D4F84C0E1349D823B3FBF0F39B0143F001
:10C2600000530120C2F884308866FCF7ADFB35E747
:10C27000003802402819002000ED00E00005FA0512
:10C2800000000020FFC9FE36335F0700D34D621067
:10C2900080841E0040420F0044B205080070004038
:10C2A000003C02400000474210B584B00023044621
:10C2B000ADF80C300068ADF806308DF80E3003F1A3
:10C2C0008043013903F5823389B29842029114D038
:10C2D000A3F58063984210D003F5804398420CD0B8
:10C2E00003F58063984208D003F58063984204D038
:10C2F000204BD3F8AC375B0802E01E4BD3F8AC37C9
:10C30000B3FBF2F301A9013BADF8043044F058FF50
:10C310002168194A0B8819489BB243F001030B802E
:10C32000002301E050F83320914208D001330E2B56
:10C33000F8D1002004B0BDE81040FCF7B9BA104AAB
:10C3400002EBC30393F84D4D2046FCF7B1FA1B2CCA
:10C3500005D1192004B0BDE81040FCF7A9BA2E2C75
:10C3600008BF2C2004D104B0BDE81040FCF7A0BAEF
:10C3700004B010BD281900200000014094AE05084B
:10C380004CA1050870B50468A30AA3F58013522BCD
:10C3900051D83C4D2B4493F8F4530D2D4BD8407994
:10C3A0008608002954D005EB850305EB4303B4F858
:10C3B0000CE04FEA900C33440220334E00FA0CF0AC
:10C3C00040EA0E0006EB830C80B2CCF84815CCF89E
:10C3D0005825A081EFF3118C502383F312882C236E
:10C3E00005FB03F3F118D1F8442562B3274BC1F8DC
:10C3F0006825043226482C2105FB01F1084414313C
:10C400000B4453F8041B19B1116053F8042C043287
:10C410009842F6D100235FFA8CFC13608CF31188EC
:10C420002C2303FB0565D5F868352BB1A3899BB296
:10C4300043F00103A38170BDA38923F001031B0412
:10C440001B0CA38170BD03F12402104B1A44D1E7E9
:10C45000B4F80CC005EB8503304605EB43034FF001
:10C46000020E33441FFA8CFC074E0EFA00F02CEA41
:10C470000000A08106EB8300C0F84815C0F85825DD
:10C48000A8E700BF4CA10508281900206C1E002059
:10C49000901E002001490248FDF708BA6C1E0020DA
:10C4A0000000014010B5064C064804F24451FDF767
:10C4B000FDF904F5DA610448BDE81040FDF7F6B96E
:10C4C00028190020000001400044014002494FF0BB
:10C4D0008040FDF7EBB900BF981E002001490248DB
:10C4E000FDF7E4B9C41E00200004004001490248E1
:10C4F000FDF7DCB9F01E00200008004001490248A9
:10C50000FDF7D4B91C1F0020000C0040014902486F
:10C51000FDF7CCB9A01F00200004014010B5064C67
:10C52000064804F5CF61FDF7C1F904F254710448DF
:10C53000BDE81040FDF7BAB92819002000040140F9
:10C54000001C004001490248FDF7B0B9CC1F002093
:10C550000040014001490248FDF7A8B9242000200D
:10C560000048014001490248FDF7A0B950200020D1
:10C570000018004001490248FDF798B9A8200020A2
:10C580000020004010B50C2937D8DFE801F09736BD
:10C59000363666363636373636360700038C5488DC
:10C5A000B2F80CE023F480531B041B0C0384038CAF
:10C5B000B0F804C0818B21F4E6414EEA040E090470
:10C5C000148823F40053090C41EA04211B04754C20
:10C5D0001B0C43EA0E33A0421FFA8CFC9BB289B2BB
:10C5E00000F0AE8004F58064A04200F0A98092685B
:10C5F000A0F804C081830264038410BD038CB2F8E8
:10C600000CC0548823F480731B041B0C0384038C1C
:10C61000B0F804E0818B23F400731B044CEA040C93
:10C6200021F073011B0C43EA0C230904B2F800C08B
:10C63000090C41EA0C0C5B4988421FFA8EFE9BB242
:10C6400068D001F58061884264D09268A0F804E067
:10C65000A0F81CC0C263038410BD038CB2F80CC0E8
:10C66000548823F010031B041B0C0384038CB0F8C4
:10C6700004E0018B23F020031B044CEA040C21F49A
:10C68000E6411B0C43EA0C130904B2F800C0090C84
:10C6900041EA0C211FFA81FC424988421FFA8EFEB2
:10C6A0009BB269D001F58061884265D09268A0F89C
:10C6B00004E0A0F818C08263038410BD038C548882
:10C6C000B2F80CE023F001031B041B0C0384038C61
:10C6D000B0F804C0018B21F073014EEA040E090486
:10C6E000148823F00203090C1B0421432D4C1B0C5E
:10C6F00043EA0E03A0421FFA8CFC9BB228D004F53B
:10C700008064A04224D09268A0F804C001834263F0
:10C71000038410BDD189548A23F4006343EA0121C4
:10C72000138A2EF4405E23434EEA031E94884FF68C
:10C73000FF330B4043EA04231FFA8EFE9BB284E7CB
:10C74000148A2CF4804C4CEA841C1FFA8CFC4EE7B3
:10C75000D489B2F810E023F008032343548A2CF460
:10C76000407C4EEA040E948823F004034CEA0E0C3D
:10C770001FFA8CFC2343C6E7D189548A23F0800337
:10C7800043EA0111138A2EF4406E23434EEA830ECE
:10C7900094884FF6BF730B4043EA04131FFA8EFED2
:10C7A0009BB283E7000001402DE9F04FA24BDFF878
:10C7B000A49293F8723EA14EA14F8FB0CDE90139FA
:10C7C000013BDBB200930025DFF88CB2DFF88CA2CE
:10C7D0005B46D3469A464FEA9A23A3F58013522B21
:10C7E0004CD8334493F8F4330D2B47D8FC56019BB7
:10C7F000012B40F00181012C35D14FF0000841465A
:10C80000204610F0E5FE10F071FF037813B1542BB1
:10C8100040F0F98008F104081FFA88F8B8F1100F09
:10C82000EDD14FF0000E8DB3494600200CE03344AB
:10C8300093F8F4330D2B0ED8FB56A3420ED00130E3
:10C84000A84201F580711EDA8A6813689B0AA3F575
:10C850008013522BEBD90023A342F0D153799BF8DC
:10C8600005209A42EBD1774B5B454BD05BF81CAF70
:10C870004FEA9A23A3F58013522BB2D9009B012BC8
:10C88000F1D90024B9E7BEF1000FECD15846FBF70F
:10C8900079FDC3B2022B9BF805C000F23483431C20
:10C8A0005BB203EB43034FEA830E644B664903F527
:10C8B000727004E0984200F0268353F82C1F514513
:10C8C000F8D11A796245F5D153F80E40002CF1D019
:10C8D0005E4800234268A24203F1010300F0898010
:10C8E000102B00F12400F5D14FF0FF33584A03EB31
:10C8F000C30302EB830393F86431002BB3D1029B93
:10C90000C3F808B0029B013503F58073042D029330
:10C910007FF45AAFDFF848B10BF59E730027ABF5F3
:10C92000816A9846DAF8243ABB425FDDDBF80C50A6
:10C93000002D5BD09BF81030A88802932B68DAF8A2
:10C940000460019303F13F41B0FA80F301F57E01E9
:10C950000393002EC3F11F034FEA9121009340F38C
:10C960008480002302E00133B3427BD01C0259F8DB
:10C9700004208A42F7D14C440099029B8BF8103076
:10C9800003260137CBF80410CBF80C50CBF8184035
:10C99000AE71EF71636CE26C0D4649008E401E4330
:10C9A000012303FA01F111439AF800206664E1645F
:10C9B0007AB303FA05F11A46236D0B432365019BF5
:10C9C00089B21883D4F8A000FBF718FD2046FBF7C6
:10C9D0006BFE0123082F8BF81C308BF81D3088F874
:10C9E00011300BF1200B08F118089BD10FB0BDE8F6
:10C9F000F08FDBB2013B79E7022B7FF4FEAE082C0F
:10CA00003FF4FBAE2FE74FF0010E002D7FF40CAF8B
:10CA100029E70399C1F12F05009903FA05F58B4029
:10CA200099B2236D2B432365019B5883D4F8A00052
:10CA3000FBF7E4FCCAE700BF281900204CA1050859
:10CA4000881C060844B3050800000140D0020020FD
:10CA5000880100200C0000100004014064B20508A9
:10CA60000C040010032B00F31F820AEB0623320292
:10CA700018690492002800F03F8299600131CAB21F
:10CA800083F805210692542283F8042101360268B6
:10CA900005924479CAF80460FBF774FC934AC3B268
:10CAA000022B92F889EE844600F22D82461C76B263
:10CAB00006EB46068E498F48059AB600002305E02E
:10CAC0000133172B00F01F8251F82C0F8242F7D14F
:10CAD0000879A042F4D188590028F1D02C2101FB1B
:10CAE00003F30CEB4C0C03EB8C0C814B6344196986
:10CAF000049B5344C3E906017F4B00211E461C469C
:10CB00006368984216D00131102904F12404F7D14A
:10CB10007A4B93F84021002A00F0E7817849794A5E
:10CB2000794BCAF8681ACAF8602ACAF8703A0FB086
:10CB3000BDE8F08F01F1010C5FFA8CFC6F4B07969A
:10CB40000CF1FF3C0CEBCC0C03EB8C0C9CF864312F
:10CB50000593002BE2D1049E069B8CF86531F311FE
:10CB600003EB262000EB001368488C2400EB8300C5
:10CB70003112674B04FB01F103EB41010AEB0603A1
:10CB8000C3E93C145421019E8CF864113321C3F88D
:10CB9000AC10DE60C3F8A8005E4B04999A4209EB22
:10CBA000010400F07681534B9A4200F0728103F544
:10CBB00080439A4200F06D8103F580639A4200F051
:10CBC000688103F580639A4200F06381474BD3F894
:10CBD000AC07BEF1060F4FEA500000F061814E4BEA
:10CBE0004E49BEF1070F18BF9C464D4B08BF8C46FF
:10CBF0004C4918BF1946B0FBF1F1B0FBFCFC1046E4
:10CC0000049A01390AEB020389B20CF1FF3CA3F844
:10CC1000B0C0A3F868104FF000060193A16500238F
:10CC200002F154014944A4F85C60636544F0C8FA19
:10CC3000019B3D4A1B690193186803889BB243F02E
:10CC400080030380038809920A210B914FF48072BC
:10CC5000022123F00103CDE90C121B04ADF828607A
:10CC60001B0C019E0380717909AAFFF78BFC3079B8
:10CC7000002840F02281049B079E0AEB0302002358
:10CC80001069D2F818C001680A8892B242F0010215
:10CC90000A807268944503F1010300F00A81102BA9
:10CCA00006F12406F5D14FF0FF33144A1F4E03EB73
:10CCB000C30302EB83031E4AD3F84831B3420CBFCF
:10CCC0004FF400134FF48003166B33431363427920
:10CCD00018480C2A9BBF184B03EB42030026B3F8FD
:10CCE0001C61049B53449E8200232EE028190020DF
:10CCF0004CA1050800000140D0020020880100205E
:10CD000065730108617301086D730108B427002081
:10CD1000E42A002000040140449508001055220038
:10CD2000D0DD060040771B0060000100006002407B
:10CD3000003802401406001044B20508914200F089
:10CD4000E0800133042B00F0E18050F83320002A0A
:10CD5000F4D1DAF80C260132CAF80C260AEBC30229
:10CD6000DB00C2F8101603446A499A8805981643F6
:10CD70009E80049B0AEB030690222346FEF728F8C8
:10CD8000B0690268002342F010020260C4E9253352
:10CD9000A367C4F88830C4F89C30F26962664FF427
:10CDA0008062E26704214FF40032C4E9232140226B
:10CDB0002267D6F8AC206267F268049B1832A2663C
:10CDC0004FF48052C4F88020D6F8A820E26603F120
:10CDD00064014FF480424944C4F8842044F04EF981
:10CDE000B069049BD0F800E0C4F81CE0D0F814E06F
:10CDF000C4F820E0D0F804E0C4F824E003F1AC016A
:10CE0000D0F808E0C4F828E00023D0F80CE0C4F81B
:10CE10002CE0C4E93733C4F8B830C4F8C030C4F8E3
:10CE2000D030C4F8E430F369C4F8AC304FF4806318
:10CE3000C4F8C4304FF4403C0423C4E935C3D6F8E9
:10CE4000F430C4F8BC30F3681033C4F8B0304FF499
:10CE50000063C4F8C830D6F8F030C4F8B4304FF4EA
:10CE60008042C4F8CC20494444F008F9B369A8884A
:10CE70001A6822635A6962635A68A2639A68E26315
:10CE8000DA6822641A6842F010021A602B68019373
:10CE900072E5214BBEF1060FD3F8AC077FF49FAECD
:10CEA000DFF87CC01D49A6E61B4A032382F8883EB2
:10CEB00034E6DBB20593013BF7E60BF0EFFE06909C
:10CEC00038B1019B0221DA79FEF798F9069B5422CA
:10CED000DA80019B1A68B2F844306FEA43436FEA84
:10CEE00053439BB2A2F84430C5E6542283F8402154
:10CEF000069A83F8412111E6074A022382F8883E08
:10CF00000CE6DB002FE700235B68FFDE00239B8835
:10CF1000FFDE00BF4584000828190020A0BB0D00DB
:10CF2000882A11000C2911D8DFE801F02310101015
:10CF300019101010111010100700838B23F40063D8
:10CF40001B041B0C43EA022292B282837047838B3C
:10CF500023F008031B041B0C1A4382837047038BC6
:10CF600023F400631B041B0C43EA022292B20283E7
:10CF70007047038B23F008031B041B0C1A43028326
:10CF8000704700BF2DE9F04FDFF870B29BF800400A
:10CF900087B024B90124204607B0BDE8F08F934E36
:10CFA000D6F804580DF00CFC9BF8B43A0390002B13
:10CFB00000F058828E4AA2FB05328E4B5209A3FB29
:10CFC0000213DB0803EB8303A2EB4303DAB2049200
:10CFD0000BF23C6202EB830300930BF61C1306F189
:10CFE000DC0401934FF00009924635E03B68029360
:10CFF000009B5C330093019B30461433019343F054
:10D00000A7FF7A4B02988C2202FB0933002583F894
:10D01000D05079792A46FFF785FF22467979FFF7C4
:10D02000B1FA79790822FFF77DFF402344F83C3CB0
:10D03000A4F14801304644F021F8336843F010036E
:10D0400033609BF8B43A09F1010999450AF15C0A89
:10D0500004F18C0480F2D480DBF83836039AD31ABA
:10D0600004D454F8082C9342C0F2AB815F4B54F8BF
:10D07000587C266A8C2202FB093393F8D030002BAF
:10D08000B4D03968736834F8542C02911FFA83FEC7
:10D090008B89CEF1160E9BB223EA0203BEF1070F75
:10D0A0008B81A5D9DBF824390133CBF82439A36A65
:10D0B00005939C4600225CF8045B012190461BE02E
:10D0C000DCF80000B8F1140FA0EB05031DDC13F130
:10D0D000080548BF03F117052B1108EB2518054675
:10D0E000581E013102FA03F3012282408E4542EAC2
:10D0F00003020CF1040C08D38E45E1D8C8F11503E6
:10D10000DCF800504FF01508EAE7B8F1150F60D1D0
:10D110003948C2F38423C2F3441100EB830300EBCC
:10D120008101D3F83831D1F838111B0243EA0113D9
:10D1300002F01F0100EB8101C2F3C43200EB820256
:10D14000D1F83811D2F838210B4343EA023383EA8D
:10D15000132282EA121202F00F020F2A39D1C3F30E
:10D160000F134FF6FF72934233D0B3F5606F00F0A8
:10D170003681019A93819AF85820049DAA4211D0D1
:10D180000098DAF800208168521ACAF80020016B72
:10D19000DAF80420521ACAF80420002282600263DE
:10D1A0008AF85850DAF8002000990132CAF80020B5
:10D1B0008A6801328A604FF6FF7293427FF418AF9B
:10D1C000DAF804300133CAF804300B6B01330B6317
:10D1D0000EE7DBF820390133CBF82039B9F1000F25
:10D1E00000F0E5804FF6FF73C5E700BF2819002067
:10D1F0001F85EB51CDCCCCCC44B205080400001007
:10D2000001228BF8202ACBF83856002B3FF4C2AE0F
:10D21000974890F88C10890700F1BE80D0F88410F0
:10D22000086849798A40018C92B289B221EA0201E8
:10D230000184018C89B20A43012B02843FF4AAAE17
:10D240008B4991F81821970700F1C080D1F810217F
:10D2500010685479018C012289B2A24092B221EA6D
:10D2600002010184018C89B20A43022B02843FF43B
:10D2700091AE7F4991F8A421960700F1C180D1F8C1
:10D280009C2110685479018C012289B2A24092B28B
:10D2900021EA02010184018C89B20A43032B028432
:10D2A0003FF478AE724991F83022950700F1B180D1
:10D2B000D1F8282210685479018C012289B2A24049
:10D2C00092B221EA02010184018C89B20A43042B43
:10D2D00002843FF45FAE664991F8BC22940700F1E6
:10D2E000A180D1F8B42210685479018C012289B24E
:10D2F000A24092B221EA02010184018C89B20A4360
:10D30000052B02843FF446AE594991F84823900713
:10D3100000F19180D1F8402310685479018C0122EA
:10D3200089B2A24092B221EA02010184018C89B241
:10D330000A43062B02843FF42DAE4D4991F8D423C5
:10D34000920700F18180D1F8CC2310685479018CC8
:10D35000012289B2A24092B221EA02010184018C29
:10D3600089B20A43082B02847FF414AE404A92F833
:10D3700060349B0771D5D2F8582404231168507982
:10D380000A8C83409BB292B222EA03020A840A8C7E
:10D3900092B213430B84FDE5354AD2F8842010681D
:10D3A0005479018C0422A24089B292B23EE70599D9
:10D3B000304858224CF002FE3B6802934FF6FF7350
:10D3C000D9E60024204607B0BDE8F08F284AD2F8FD
:10D3D000102110685479018C042289B23DE7244958
:10D3E00091F8DD2402EB420201EBC2024A4492F8BA
:10D3F000ED240D2A7FF4BDAE019980228A77BAE62A
:10D400001B4AD2F89C2110685479018C042289B2FD
:10D410003CE7174AD2F8282210685479018C04227C
:10D4200089B24CE7124AD2F8B42210685479018CC0
:10D43000042289B25CE70E4AD2F84023106854797E
:10D44000018C042289B26CE7094AD2F8CC23106817
:10D450005479018C042289B27CE7054BD3F8582417
:10D4600001238BE701228BF8202ACBF8383692E58E
:10D4700028190020CC0900102DE9F04F002299B0A6
:10D480002F21074610F088F900B3BE4ED0F8008077
:10D49000C6F83C8E0446FDF79FFB0246B0B1D0F8BB
:10D4A00004C0C6F838CEBCF1000F0FD0B64D002333
:10D4B00029464868844501F1240103F101030FD096
:10D4C000102BF6D1B14B93F8400118B1002019B0E0
:10D4D000BDE8F08F2F2283F8402183F84101F6E761
:10D4E000DBB2DFF8A892013B03EBC30309EB830334
:10D4F00093F864A1BAF1000FE8D138469768DFF8D5
:10D50000C0B22F22A3F864210BF0C8FB2F220346E0
:10D51000CBF8280520B1DA80E2792A21FDF76EFEEA
:10D520009B4A9C49002301E051F83320904500F0CC
:10D53000228101330E2BF7D1002048F007FAD6F8EC
:10D540003C0E954A038823F001031B041B0C9042F8
:10D55000038000F070818E4B984216D003F5804313
:10D56000984212D003F5806398420ED003F5806391
:10D570009842D6F8AC270AD08849B1EB520F4FEA4F
:10D58000520340F2528100210AE0D6F8AC27834BC7
:10D590009A4280F017814FF0010C0021B2FBFCF39E
:10D5A0007F4AADF804101B0A7E49A2FB03231A0927
:10D5B000A1FB021252084FF000081B09ABF8262508
:10D5C00001A952000293ABF82425ADF80C80ADF808
:10D5D00006808DF80E8043F0F3FDCDE90688CDF886
:10D5E0002080A379ADF81480602204929A0740F15C
:10D5F000AF80DB0003F00803ADF81E300423ADF864
:10D600001430D6F83C0E617904AAFEF7BBFF6179AD
:10D610000822FFF787FCB0F84430D6F8388E6FEA5E
:10D6200043436FEA53439BB2A0F8443003889BB254
:10D6300043F080030380A3796179028C9B074CBF80
:10D64000042301238B409BB292B222EA030202849C
:10D65000028C92B21343038403889BB243F001030C
:10D6600003802A4600235168884502F1240203F111
:10D6700001037DD0102BF6D14FF0FF3303EBC30332
:10D6800009EB8309484AD9F8483148498B420CBF15
:10D690004FF400134FF48003116B0B43136300230B
:10D6A0006A68904505F1240503F101035DD0102B54
:10D6B000F6D13F49602200235046FDF789FB4046E2
:10D6C00043F046FCD6F8380E036823F0010300252A
:10D6D000036043F03DFCCDE91455CDE91655D6F86D
:10D6E0003C3E0E9512956279D6F8380E0997343380
:10D6F0001344304A0B9240220A930C924FF4804319
:10D700004FF48052CDE9102340F22A414FF44033C8
:10D710000D91139309A94FF480630F9343F0AEFC6E
:10D720006379D6F83C1E0C2B04D8234A02EB430342
:10D73000B3F81C518B89D6F8382E9BB21D438D81CE
:10D740001368012043F01003136019B0BDE8F08F97
:10D750005B0003F00203ADF81C300123ADF812307A
:10D760004FF48073ADF820304BE75FFA83FAA0E7FF
:10D77000DBB2013B82E7114A02EBC30393F84C0D85
:10D78000DBE600BF28190020D0020020880100201D
:10D790000000014094AE050800040140006CDC026A
:10D7A000598B4F01ABAAAAAA003802400060024080
:10D7B000FD8600082C89002044B205084CA105080C
:10D7C000202A0020254B98420BD003F58043984235
:10D7D00007D003F58063984203D003F58063984235
:10D7E00022D102F1B7731E4903F55853A1FB03136D
:10D7F0009B0D013B99B2194B984201F1010C3FF48A
:10D80000CDAE03F5804398423FF4C8AE03F5806384
:10D8100098423FF4C3AE03F5806398423FF4BEAE36
:10D820005308B3FBFCF3BBE6530803F1B7730C4991
:10D8300003F55853DAE7D6F8AC270A4B9A42FFF4BF
:10D84000AAAE074902F1B77303F55853A1FB0313BE
:10D850009B0D013B99B201F1010C9FE600000140D4
:10D86000819F5E16006CDC02F0B50C4689B03C4925
:10D87000BDF838609DF83C70013B054620689BB2BE
:10D88000049388424FF00003ADF81430ADF80E3029
:10D890008DF8163013D0334B984210D003F58043E7
:10D8A00098420CD003F58063984208D003F580635A
:10D8B000984204D02C4BD3F8AC375B0802E02A4BDB
:10D8C000D3F8AC37B3FBF2F203A9013AADF80C2060
:10D8D00043F076FC20686179A3790FB183F00103EE
:10D8E0000022CDE90622ADF81020602203929A07AB
:10D8F00029D5DB0003F00803ADF81A300423ADF896
:10D90000103003AA01910596FEF73CFE019908220A
:10D91000FFF708FB2268B2F844306FEA43436FEA2E
:10D9200053439BB2A2F84430138811469BB243F094
:10D93000010321F8343B63796A60C818002228602B
:10D94000CA5009B0F0BD5B0003F00203ADF8183017
:10D950000123ADF80E304FF48073ADF81C30D0E7E2
:10D9600000040140000001402819002070B5384C27
:10D9700094F8345584B00DB904B070BD94F83535C1
:10D9800084F8543528460BF089F9C4F8440508B1E9
:10D990003823C38094F82C656EB3012EECD1314648
:10D9A000FDF708FB94F85435002B49D1D4F84435E1
:10D9B00013B11A689B881383264D4FF4E072D5F893
:10D9C000B831C4F8502503A8012284F840250393F8
:10D9D00043F0A8FAD5F8BC31029302A843F0A2FAAA
:10D9E0001D491E4C0B6C1E48002243F030030B6493
:10D9F00022850285C0E72846324638210FF0CCFE4A
:10DA000005460028B8D0C279D4F844050221FDF7B4
:10DA10003BFC144A94F85435D2F8AC2712480193D1
:10DA20005208802329460096FFF71EFFD4F84815B8
:10DA300080230122C4F850350B6084F840259BE711
:10DA4000D4F84435002BB7D01A689B885383B3E7CA
:10DA5000202A002044B2050800380240001000408F
:10DA60000014004028190020682F00200B4B93F869
:10DA70005425D3F844353AB113B11A689B885383BF
:10DA8000074B00221A827047002BF9D01A689B8836
:10DA90001383034B00221A82704700BF202A002004
:10DAA000001000400B4B93F85425D3F844353AB19D
:10DAB00013B11A689B881383074B00221A827047A0
:10DAC000002BF9D01A689B885383034B00221A82DB
:10DAD000704700BF202A0020001400402DE9F041CB
:10DAE0005C4CDFED5D7AB4F82E35DFED5C6A94F8BE
:10DAF0002C5504EB400007EE103AB0F83635B4F878
:10DB000032056422B8EEC77A02FB03F327EE277AC8
:10DB100007EE903AF8EEE77A02FB003327EE277A19
:10DB200007EE903AF8EEE77A002687EE270A0F46CE
:10DB3000C4F8586520EE260A55B3012D01D0BDE882
:10DB4000F081D4F8508507EE908AF8EE677A27EED8
:10DB5000800A4BF0BBFC002832D194F85435002BDE
:10DB600066D0D4F8443513B11A689B881383B4F88F
:10DB7000300538440FF024F994F85435002B5FD069
:10DB8000D4F84435002BDAD01A689B885383D6E743
:10DB9000D4F8503507EE903AF8EE677A27EE800A0F
:10DBA0004BF094FCD4F848252D4B1060D3F8043882
:10DBB000B4F8301519443944C4F85C15BDE8F08157
:10DBC000284A294B5062C2F82C805E62C3F82C8030
:10DBD000EFF31181502080F312881580C9B21D80A7
:10DBE00081F3118895811E4A9D81D2F80438B4F8DA
:10DBF000301519443944D2F804389942FBD81949F0
:10DC0000194A0B88D4F8440523F001031B041B0CAC
:10DC10000B80138823F001031B0400241B0C1380CA
:10DC20008C81948100288AD0036882881A8386E7D1
:10DC3000D4F84435002B9AD01A689B88538396E712
:10DC4000D4F84435002B3FF47AAF1A689B881383CD
:10DC500075E700BF202A00200AD7233CCA269B3E36
:10DC6000281900200010004000140040034B93F8D6
:10DC7000402512B1042800D830E77047202A002040
:10DC80001648174A174938B5174C184D121A4CF058
:10DC900095F9D4F88820164B164842F47002C4F85F
:10DCA00088201A68002142F001021A6099601A68FF
:10DCB00022F0847222F480321A6058601A6822F4CA
:10DCC00080221A600C4AD960521B28460B494CF03E
:10DCD00075F9A560BDE83840FAF776BE000000107F
:10DCE0000400001021CB060800ED00E00000002039
:10DCF0000038024010300024880100200000000895
:10DD00000548D0F8C03723B1DB6A13B100F5F860DD
:10DD100018470248704700BF2819002004B40508BE
:10DD200038B5184CD4F860351B8843B9164D00231C
:10DD300084F86C3585F8B837C5F8B43738BDD4F8F1
:10DD40006425002AF2DD012A09D0D4F86835598803
:10DD50000D4DA4F86E15012384F87035E7E7D4F86B
:10DD600068158A8849880132521A9A42F0D1064DC4
:10DD7000D5F8C03700221B69C5F8EC2705F5F86017
:10DD80009847D4E7202A0020281900200748D0F817
:10DD9000BC371BB1064B93F870350BB100207047B0
:10DDA000D0F8C03700F5F8605B68184728190020E4
:10DDB000202A002030B4154A154D92F8B83705F2E4
:10DDC00074542344036095F86C35446092F8B807A6
:10DDD000834292F8B80712D8834204D3002030BCA3
:10DDE000C1E90000704792F8B827002BC2F1800209
:10DDF0000CBF0120022030BCC1E9002370471B1A70
:10DE00000022012030BCC1E90032704728190020EF
:10DE1000202A00200E4B0F4A93F8B81792F86C0591
:10DE200093F8B827904293F8B8270CD8904238BF9F
:10DE300093F8B827D3F8B4373ABFC2F180028018FC
:10DE4000002018447047D3F8B437801A184470473C
:10DE500028190020202A002030B51C4C1C4D94F8B5
:10DE6000B83794F8B81785B005F27452134402938A
:10DE700095F86C3503928B421DD894F8B8279342DD
:10DE800011D294F8B8170193C1F180010091D3B970
:10DE9000012208B93F2906D90023694602A849F0A2
:10DEA000ADFD95F86C3594F8B807C01AB0FA80F05B
:10DEB000400905B030BD94F8B8170022591A0192F4
:10DEC00000910122E5E719440222E2E72819002027
:10DED000202A00202DE9F043164685B0002936D0CF
:10DEE000441E254D254F04EB01084FF0000901E0C9
:10DEF000A0452CD095F86C0514F8013F411C28442E
:10DF0000C9B280F874350B0648BF002097F8B837BF
:10DF100085F86C154ABF0146084685F86C958B421A
:10DF200097F8B8378ABFC3F18003C01AC0183F28DA
:10DF3000DED997F8B8378B42DAD0114B93F8C4305A
:10DF4000002BD5D00020FFF787FFA045D2D169462E
:10DF500002A8FFF72FFF20B1DDE9003213443F2B69
:10DF600002D805B0BDE8F0830246334602A849F066
:10DF700045FD05B0BDE8F083202A002028190020C7
:10DF80008801002030B585B0694602A8FFF712FF6E
:10DF900058B9094C04F5F865D4F8C03728465B68D1
:10DFA00098470028F8D005B030BD0246012302A8EA
:10DFB00049F024FDEDE700BF2819002070B5124E8E
:10DFC0001546D6F8BC370A46411999420F4988BF11
:10DFD0001D1A91F86C1596F8B837994282B004462C
:10DFE00003D00192FFF7CEFF019AD6F8C017084878
:10DFF0000023C6F8EC372B468D6A2146AC4602B0AA
:10E00000BDE87040604700BF28190020202A00208A
:10E01000E82000208C461346014662461846CDE7AC
:10E0200038B52448244C0023C4F8BC370246117884
:10E03000022902F106022CD00133062BF7D11F4D25
:10E04000D4F8C0370022C5F86825F3B1DA6AE2B126
:10E050001B489047D5F86835C5F86005A3B19A8884
:10E060005B88D21A436802FB0333C4F8BC37FAF763
:10E0700011FE95F86C2594F8B8379A42054601D000
:10E08000FFF780FFC4F8B45738BD0E4BC5F86035B4
:10E0900038BD0A4DD4F8C02703EB430300EB43031C
:10E0A000C5F8683512B1D26A002AD1D10548C5F841
:10E0B0006005D4E71430002028190020202A002011
:10E0C000E820002004B405082DE9F04F41F69462E1
:10E0D0008BB00021BD484BF0D4FF042043F060F822
:10E0E0000446052043F05CF850EA040340F05C81EC
:10E0F000B74B03934C220021B4484BF0C2FF4C2293
:10E100000021B2484BF0BDFF039BB049D3F8CC339C
:10E11000B04A0A600124C1E907334B620C7148F030
:10E1200039FCFFF77DFF002108460AF049FEFAF7A7
:10E13000B1FDB0F1000B40F30881A74BA74D01934F
:10E14000A24BA74E0024029403F14C092746A04697
:10E1500005F5C36A04E008F50068C34540F3AE80E6
:10E16000019AD2F80438C2F80838FAF7C5FD20221F
:10E1700051464046FFF722FF9A49122250464BF083
:10E18000BDFF0028E7D1B84522D00299964BCDF8C3
:10E19000149001EB410203EB82004A1C9349029266
:10E1A000049001F097FDDDE90403D9F81C2043F841
:10E1B0004C0BC9E908228E4AC9F80C70C9F828200E
:10E1C000A8EB07070122C9E90477C9F80820994696
:10E1D000039BD3F8CC33C9F81C3047461222A91848
:10E1E000335D91F81816994202F101020BD0002418
:10E1F000202AF4D12037BB455146384654DBFFF77F
:10E20000DDFE0022EBE70134152CF1D1D01979495C
:10E210002022FFF7D3FE00230A2209A97548CDF872
:10E2200024A001F005FF04900998002301300A2280
:10E2300009A9099001F0FCFE07900998002301301C
:10E240000A2209A9099001F0F3FE0690099800231B
:10E2500001300A2209A9099001F0EAFE0590099807
:10E2600009A9013000230A22099001F0E1FE0746C6
:10E2700009980023013019460A22099001F0D8FEBE
:10E28000049989B1DDE9063243EA4212059B7F0118
:10E2900047EAC323A1F2BC7143EA600342EA412288
:10E2A00043EA0243C9F81C30029B642B00F0EC8067
:10E2B000474608F50068C3453FF752AF029A642A03
:10E2C00000F0E280B84500F0E380474C4749484EF3
:10E2D0000C2303FB0244531C1A462046A8EB0705F7
:10E2E000029301F0F7FCD9F81C30C9F80040C9E9E5
:10E2F0000375C9E908330123C9F81450C9F8286027
:10E30000C9F80830029B5D1C4C22304F02FB05F51A
:10E310007B19002118464BF0B4FE4C2200214BF033
:10E32000B0FE039A3449D2F8CC237951029C426260
:10E33000C0E904BBC0E90722012202348662826080
:10E340004FEA4B03B3F1805F1EDA4C221F4D02FBF4
:10E3500004F42B19184600214BF093FE4C220021A7
:10E360004BF08FFE0399CBF10062D1F8CC1303463A
:10E37000520022482851C3E90422C3E907110222AE
:10E380005A71012259629A60104A95682DB9137921
:10E390001BB11368002B40F08980002108460BB0A8
:10E3A000BDE8F04F0AF00CBD4FF47A72002321460D
:10E3B0004AF03AF8124B40F26D11A3FB00231B0CFC
:10E3C000022440F2B2720D4625E000BFA464002092
:10E3D000880100200CA7060828190020202A002008
:10E3E0002C1C0608081C0608583000201C1C0608B7
:10E3F00015E0000838300020441C0608541C0608AC
:10E4000007452EC2013212F00304A3EB01030CBF37
:10E410004FF4B77129469942F4DD7B49002C3FD077
:10E4200003910399D1F89C138B4272DB774D012441
:10E430005B1A55F8041F994204F10104F8DD013319
:10E4400043EA4413A2F2BC7243EA4223704A039D9A
:10E45000B0FBF2F102FB11024FF461603C24B2FB0D
:10E46000F0F100FB11221C20C5F8A003B2FBF4F070
:10E4700004FB1022521042EA401242EAC12242EA50
:10E480000343C5F8CC3335E66423624E029339E783
:10E49000029B01245D1C002B3FF452AF5D4E33E71D
:10E4A0000C4603911D21C4F8A013BAE7C2E9115527
:10E4B0001564D56329462E46D46C02F14C0354B33F
:10E4C0009C681E64481E8442C3E91166DE6312D054
:10E4D000481C844216D08C427FF45FAF0846002867
:10E4E0003FF45BAF116CCC6B0134CC631964936463
:10E4F00001461A46E0E700293FF44FAF884253F83F
:10E500000C2CECD1117900293FF447AF53641A6405
:10E51000EEE7012493E740490222264613E0CB6B45
:10E520000A635B011DBF03F6FF7702F1FF3303EBC4
:10E5300017331346C1E90466C1E90D3351F84C0F96
:10E540005A1C0135C8B10B79002BE8D10F690A6359
:10E55000002F4BD14F691046531E4863002F4ED0F9
:10E5600007F6FF7703EB1733201A8B63C41851F8B3
:10E570004C0F5A1C01350028E5D128492848C1F81C
:10E5800054583E220D46C1F830283F22013BC1F8C5
:10E5900034284022C1F838280191C1F84438C1F824
:10E5A00048489A00990FC5F82C0853B340F2FF1061
:10E5B000121841F10001520A42EAC152019C02F1D3
:10E5C00040010A4402EBC303C4F84028C4F83C18D5
:10E5D000144A1149C4F84C18C4F850185802D90DFF
:10E5E000C4F82838C4F820085160D6E607F6FF774B
:10E5F000531E03EB17304F694863002FB0D1134609
:10E60000B2E70122DAE700BF8801002024050020DC
:10E610008051010015E00008A464002028190020A2
:10E62000601C06084821002010B50A4CD4F8C037F9
:10E630005B6A13B104F5F8609847074AD4F8B43719
:10E64000D2F860255288013B134452421340C4F86B
:10E65000B43710BD28190020202A00202DE9F043EE
:10E66000DFF8E890374F93B0FFF75AFBFFF7D8FC7D
:10E6700099F8B83797F86C259A4201D0FFF782FCD9
:10E68000D9F8BC870025C9F8B457B8F1000F11D0EC
:10E690002D4E6C462A463146204601F01BFB204693
:10E6A00049F0FEF92035014601222046FFF712FC11
:10E6B000A845EFD899F8B83797F86C259A4201D059
:10E6C000FFF760FCD7F860359B7B012B33D099F8BE
:10E6D000B83797F86C259A4201D0FFF753FC002712
:10E6E000C9F8B477B8F1000F28D0DFF85C903D4648
:10E6F0006C462A46494609A801F0ECFA212200217D
:10E7000020464BF0BEFC202221462846FFF756FC4F
:10E710002022064609A9204615444BF0EFFC08B913
:10E72000202E00D00137A845E3D8B7FA87F040097A
:10E7300013B0BDE8F083FFF777FFC8E7012013B0FF
:10E74000BDE8F083202A0020681C06082819002054
:10E75000032108B50546084642F012FD72B6104B7B
:10E7600053E9022352EA03010AD10024214604207E
:10E7700042F006FD2146052042F002FDFDF71AFC9D
:10E780000848D0F8044829B24EF6602000FB01F199
:10E79000A41843F100030C1943EBE171E7E700BF54
:10E7A0001035002028190020084B09498B420246E9
:10E7B0000AD2184602E01C30884205D20388C3F30F
:10E7C0000B039A42F7D170470020704744A906080E
:10E7D00078B106088388C3F30B039342A8BF13469E
:10E7E00070B51A461D460C46064680684BF0E6FB9F
:10E7F00062199442B569074B08D0074814F8011B09
:10E8000000FB03F3A24283EA0103F7D12B6001204E
:10E8100070BD00BFC59D1C819301000100230370E2
:10E8200043708370C370704700230370437083701C
:10E83000C370704700220123027042708270C27060
:10E84000037143718371C371704700BFFF2303706D
:10E8500043708370C3707047002306214FF47A72AF
:10E86000C0E9012301700373704700BF10B5002396
:10E87000411CFF2200F8132001F8132001330B2B59
:10E88000F8D10B4B4FF0FF3103F10F0400228C46FF
:10E8900005E093F904C093F9051013F8032F00F86D
:10E8A00012C000EB420E9C428EF80110F1D110BD57
:10E8B00098BD05084FF0110C00B580F800C04FF06E
:10E8C000100C80F803C04FF0120C0022022180F8D7
:10E8D00006C04FF0130C012382704271C1710272A5
:10E8E00080F809C04FF0180E4FF0FF0C8172C17410
:10E8F000C2724F2137224370037180F80CE04373DA
:10E900008373C173037480F811C0827480F814C0DB
:10E910005DF804FB03230370704700BF0A44914273
:10E9200019D000B501F1FF3C02F1FF3E41F2210197
:10E930001CF8012F082380EA022010F4004F81EA1E
:10E9400040020ABF400090B280B2013BF5D1E645DB
:10E95000EED15DF804FB7047704700BFD0ED007A40
:10E96000D0ED016A30EE677AE6EE877AB0EE670A9C
:10E97000C0ED007A704700BFD0ED017AD0ED026A99
:10E9800030EE677A90ED000AE6EE877A37EEC07ACD
:10E99000C0ED017AA6EE870A80ED000A704700BF3D
:10E9A00090ED017AD0ED036AD0ED027A30EE470A9D
:10E9B000A6EE807A90ED000A80ED017A37EE676A64
:10E9C000E6EE867A37EEC07AC0ED027AA6EE870AC6
:10E9D00080ED000A704700BFDFED277AB4EEE70A4A
:10E9E000F1EE10FA0CDDDFED256A9FED257AF0EEF1
:10E9F000407AF4EEC77AF1EE10FA30EE660AF6DCF1
:10EA0000DFED207AB4EEE70AF1EE10FA0CD5DFED77
:10EA10001B6A9FED1D7AF0EE407AF4EEC77AF1EEB4
:10EA200010FA30EE260AF6D4DFED187AB4EEE70AD3
:10EA3000F1EE10FA14DDDFED107A37EEC00A60EE69
:10EA4000006A9FED136A9FED137ADFED137AA6EE4D
:10EA5000867A20EE266AE6EE877AA6EE270A7047C7
:10EA6000DFED0E7AB4EEE70AF1EE10FA44BFDFED07
:10EA7000057A37EEC00AE2E7DB0F4940DB0FC940F9
:10EA8000E4CB1641DB0F49C0E4CB16C1DB0FC93F15
:10EA900092E741B99730083C15A82ABEDB0FC9BFE1
:10EAA000D0ED056AD0ED017A90ED007A90ED066A1E
:10EAB000D0ED025A90ED035A80ED050A66EEA77A72
:10EAC000C0ED066AE7EE007A90ED077AE5EE867A09
:10EAD00090ED086AD0ED045A80ED087AE5EE477AA9
:10EAE000E5EEC67AB0EE670AC0ED077A704700BF60
:10EAF000D0ED057A90ED006A90ED067AD0ED035ADC
:10EB0000E6EE007A90ED016AF0EE406AA6EE267A13
:10EB1000B0EE670AD0ED047A90ED026A67EEC07A33
:10EB2000A5EEC07AE6EE267A80ED057AC0ED067A8B
:10EB3000704700BF2DE9F047089F3C460E4614F889
:10EB4000011B002B054614BF4FF030094FF0200980
:10EB500041B3002A2CDD234600E0B2B113F8010BCB
:10EB60009046013A0028F8D1A8F102086AB1C246DD
:10EB700049462846B0475346002B0AF1FF3AF7DCD6
:10EB8000397828EAE872013249B1D71B2846B047E4
:10EB9000E01914F8011B0029F8D1BDE8F0871046F0
:10EBA000BDE8F087002A02F1FF38E0DC0846F4E710
:10EBB0000022EAE703685A1C02601970704700BF20
:10EBC000024B186803681B68184700BFD4990020DF
:10EBD000884210B54FF001043ED301FB04F4B0FBB2
:10EBE000F4FC8C45F9D2CCB122BB08E0A14203F879
:10EBF00001EBB4FBF1F211D8B0FBF2FC1446BCF10E
:10EC0000090F0CF1570E0CF1300204FB1C00EDDC77
:10EC1000A14203F8012BB4FBF1F2EDD900221A70E6
:10EC200010BDA14203F801EBB4FBF1F2F6D8B0FB42
:10EC3000F2FC1446BCF1090F0CF1370E0CF1300256
:10EC400004FB1C00EDDCA14203F8012BB4FBF1F244
:10EC5000EDD900221A7010BD8446002AEAD1CEE711
:10EC60000028BEBF2D23404201F8013B092870B5A2
:10EC70004FF00103864607DD03EB83035B00B0FB27
:10EC8000F3F2092AF8D8EBB1104CBEFBF3FCA4FB5D
:10EC90000320C008BCF1090F0CF130060CF1570538
:10ECA000024607D8092B01F8016B03FB1CEE09D9BA
:10ECB0000346EAE7092B01F8015B03FB1CEE01D9CF
:10ECC0001346E2E700230B7070BD00BFCDCCCCCC67
:10ECD0000378202B024600F10100F9D0092BF7D070
:10ECE0002D2B28D02B2B03BF5378B7EE000A0246FA
:10ECF000B7EE000AA3F13001C8B209289FED567A99
:10ED000010D8F2EE046A07EE901AF8EEE77A12F8DD
:10ED1000013FE7EE267AA3F13001C8B20928B0EE30
:10ED2000677AF0D92E2B5ED003F0DF03452B07D096
:10ED300020EE070A70475378BFEE000A0246D9E773
:10ED400010B451782D2978D02B296AD0A1F1300345
:10ED5000092B02F101026BD80024002303EB83038B
:10ED600001EB430312F8011FA1F130000928A3F1C0
:10ED70003003F3D9B3F59A7F1A4628BF4FF49A723D
:10ED8000072B66D9DFED356A1346F7EE007A083BAC
:10ED9000072B67EEA67AFAD802F00702DAB1F2EE94
:10EDA000046A012A67EEA67A15D0022A67EEA67ACF
:10EDB00011D0032A67EEA67A0DD0042A67EEA67A50
:10EDC00009D0053A67EEA67A05D067EEA67A012A41
:10EDD00018BF67EEA67A6CB387EE277A5DF8044B0E
:10EDE00020EE070A70475378A3F13001C8B2092812
:10EDF00002F1010298D8F2EE046AF0EE665A07EECC
:10EE0000901AF8EEE77A12F8013F87EEA66AA3F1AE
:10EE10003001C8B2092866EEA56A37EE067AEED947
:10EE200082E79178A1F13003092B02F1020293D914
:10EE3000F7EE007A27EE277AD0E79178A1F1300338
:10EE4000092B02F1020288BFF7EE007AC4D8012430
:10EE500083E7F7EE007AA1E70000000020BCBE4C7B
:10EE6000F0B5067906F0E003402B03D145794FF069
:10EE7000FF3406E0602B4FF00105F8D1447905FA24
:10EE800004F40023012006F00706AB4200D1F0BDD8
:10EE9000052E0FD8DFE806F00308101D242448B122
:10EEA000C85CD75C78400FE020B1C856D756C71B66
:10EEB000784278410133E8E70028FBD031F81300AD
:10EEC00032F81370784080B220420CBF012000203D
:10EED000F0E70028EED031F9130032F91370E6E7BD
:10EEE0000028E7D051F8230052F82370DAE7F8B58C
:10EEF0000C4E337905468BB9F8BD25B12388C3F391
:10EF00000B039D4204D0D4E90201A2884BF056F8CD
:10EF10001C34BC42F1D300233371EDE7024C034FA4
:10EF2000F7E700BFD499002044A9060878B1060885
:10EF3000037903F01803102B1CD004D82BB1082B35
:10EF400006D000207047182BFBD1B0F80B0070479B
:10EF5000104BB0F80B0093F90030591C06BF0E4B54
:10EF60001B78DBB203EB830203EBC20300EB8300ED
:10EF700080B27047074BB0F80B0093F901305A1C70
:10EF800006BF054B5B78DBB2C3EB031300EB43001A
:10EF9000EEE700BF940500202435002070B505463B
:10EFA000B0F80900FFF700FC054B1E79044628461F
:10EFB000FFF7BEFF16B1E368184470BDA368FBE716
:10EFC000D499002038B505460C46FFF7E7FF2B79AA
:10EFD00003F0E002602A03F007032AD1052B0CD8C6
:10EFE000DFE803F0030B0F0B1B1B6A79012393402F
:10EFF000DBB2027814B11343037038BD22EA030375
:10F00000FAE76A79012393409BB2028814B1134353
:10F010000380F2E722EA0303FAE76A79012303FA9D
:10F0200002F2036814B113430360E6E723EA020324
:10F03000FAE7052BE1D8DFE803F00303050507072E
:10F040000470DAE70480D8E70460D6E7092900D025
:10F0500001B9704701394B0003F00802930001F039
:10F060000301A3EB9203C1EB0111C3EB0313C1EB4B
:10F07000011100229B00890002608180438070475B
:10F0800010B50021382204464AF0FBFF0D490E4A14
:10F090000E482061C4E905120D480E4AE0610123C3
:10F0A00041F61E614FF0090CE18484F808C0A37397
:10F0B00084F82130A26221460748BDE810402DF0B7
:10F0C00059BE00BF1A046C07001975036400DC0503
:10F0D00043080E001E7D01019C1C0608B5EEC00A07
:10F0E000DFED337AF1EE10FACCBF30EE270A30EEC6
:10F0F000670ADFED307A20EE270A70B5FDEEC07AA0
:10F1000086B017EE904A054684EAE470002303A90E
:10F11000A0EBE470CDE90033029343F065FB002CD3
:10F12000ACBF20232D2303A88DF8003048F0B8FC95
:10F1300001286E4626D0022830D0032803BF302392
:10F1400003A9304603A914BF30468DF801304AF0B8
:10F15000A0FF304648F0A4FC0338C4B22246314632
:10F1600028464AF02BFF00232B55284648F098FCF0
:10F170002E232B540130311928444AF0A6FF28468B
:10F1800006B070BD43F23002302303A93046ADF81B
:10F1900001208DF803304AF07CFFDAE743F23003B8
:10F1A00003A93046ADF801304AF073FFD1E700BF44
:10F1B0006F12033A00007A4409F0B0B813B568B191
:10F1C0004C1E14F8011F21B902B0BDE8104009F02F
:10F1D000B9B8019009F0A2F80198F2E702B010BDA9
:10F1E00008B520214AF064FF034620B11A78202A8E
:10F1F00000F10100F8D0184608BDF8B5B8B10E4BC3
:10F200000138C70003EBC000CA43067B457B02F010
:10F21000010282EA0604A54209D0806828B18588E7
:10F220000068B24214BF058345833B445C73CB073F
:10F2300001D4FCF70DFFF8BDD49900202DE9F3416E
:10F24000124D134F002305F8283F044600EB8106BA
:10F25000B44203D10F4802B0BDE8F08139462846D8
:10F260004AF017FF214668464AF02FFF4FF000088A
:10F27000202168464AF01CFF28B9694628464AF012
:10F2800008FF0434E4E780F80080F1E7D499002017
:10F29000C9620608FC990020014BD86C38F042BACC
:10F2A000D49900202DE9FF471E46C368BDF8307091
:10F2B000DDF8348004468946924643B3CBB20D2B29
:10F2C0009ABF1A4AD5560025BAF1FF3F21D02368CC
:10F2D000174A3146CDE9005A3846C0475246207990
:10F2E0005FFA89F1FBF704FC024600B10288D3B251
:10F2F0000393C2F30323120BCDE9005202930D4A8C
:10F30000236831463846C04704B0BDE8F0874D1C3D
:10F31000DAE77B06F8D42368074A0C95314638466D
:10F32000C44604B0BDE8F047604700BF881C06082B
:10F33000BC600608C9600608ED6006082DE9F041CA
:10F34000154686B06A1C8846BDF830600D9F194688
:10F3500023D0030900F00F044033CDE90045164ADD
:10F3600005933046B847A8B198F80510D8F80000C2
:10F370002A46FBF705FC68B1028801780391C2F3C5
:10F380000321120BCDE900420291059B0B4A00219B
:10F390003046B84706B0BDE8F0817306FAD40309D9
:10F3A000074A00F00F000C9040333046BC4606B0D0
:10F3B000BDE8F041604700BFFC6006080E6106082A
:10F3C000376106082DE9F04188B01E4603090E9FFB
:10F3D0009046403300F00F0451B307930EF096F8B7
:10F3E000C279079BCDE900420546164A41463046A0
:10F3F000B847D0B12868FBF77FFDA9796A79DFF8B3
:10F4000054C0ED79079B009411F0020F4FEA92026D
:10F410000D4902F1010208BF6146CDE90102CDE9C3
:10F4200003150A4A00213046B84708B0BDE8F0810C
:10F43000074A0E9441463046BC4608B0BDE8F0414C
:10F44000604700BF4B610608EC6406085D61060872
:10F450007F6106084576060870B585880B46044628
:10F46000C5F30B052A46002118464AF00AFE6169D9
:10F47000084A9142034602D3074A914205D319B183
:10F48000BDE870401846084770BD2A46BDE8704088
:10F490004AF094BD78B1060885B3060838B5064C25
:10F4A000064DAC4206D2A16820461C34FFF7D4FFBB
:10F4B000AC42F8D338BD00BF44A9060878B10608AD
:10F4C0004840082310F0800F82EA40010ABF400044
:10F4D000C8B2C0B2013BF5D1704700BF30B5056876
:10F4E0008D4219D901F1FF3E6C1E00231EF801CF99
:10F4F000082183EA0C0313F0800F82EA430C0ABF51
:10F500005B005FFA8CF3DBB20139F4D17445EDD1C5
:10F510006A1C02602B7030BD00236A1C02602B70D5
:10F5200030BD00BF07EE901AB8EE677ADFED7C7A47
:10F5300027EE000A60EE277ABDEEE77A17EE103A62
:10F540002033402B00F2DB809FED767AB4EEC70AC1
:10F55000F1EE10FAB0EE677A0CDDDFED735A9FED35
:10F56000736AF0EE476AF4EEC66AF1EE10FA37EE0F
:10F57000657AF6DCDFED6E6AB4EEE67AF1EE10FA4B
:10F580000CD5DFED695A9FED6B6AF0EE476AF4EE39
:10F59000C66AF1EE10FA37EE257AF6D4DFED666A28
:10F5A000B4EEE67AF1EE10FA00F39D80DFED636AC7
:10F5B000B4EEE67AF1EE10FA44BFDFED5D6A36EEA6
:10F5C000C77A27EE075ADFED5E5A9FED5E6ADFEDE0
:10F5D0005E6ADFED5E4AA5EE256A27EE054AE5EE96
:10F5E000066AF7EE005AA4EE267AF0EE656AE7EEB8
:10F5F000646AE7EE245A86EEA54A9FED4F7A77EECD
:10F60000877ABDEEE77A17EE103A2033402B6FD899
:10F610009FED4F7AB4EEC70AF1EE10FA0CDD9FEDC4
:10F62000426ADFED426AB0EE677AB4EEE67AF1EE56
:10F6300010FA77EEC67AF6DC9FED3D7AF4EEC77AE3
:10F64000F1EE10FA0CD59FED386ADFED3A6AB0EEB4
:10F65000677AB4EEE67AF1EE10FA77EE867AF6D4AF
:10F660009FED357AF4EEC77AF1EE10FA4CDD9FED9E
:10F67000397A77EE677A67EEA74A9FED317A9FED88
:10F68000315ADFED316AA4EE875A67EEA43AE4EE10
:10F69000856AB7EE006AE3EEA67AB6EE007A36EE39
:10F6A000676AB8EE005A67EE857A26EE077AB7EEFB
:10F6B000005AC5EE256A0023836143610362C3617A
:10F6C00080ED044A26EE877A26EE866A66EEA77AF1
:10F6D00080ED095A80ED007A80ED016A80ED027AB2
:10F6E000C0ED037A7047DFED1B6A36EEC77A68E734
:10F6F000DFED197AB6EE007AB7EE006AD7E7B7EE1B
:10F70000004AF0EE445A78E79FED0C7AF4EEC77A9F
:10F71000F1EE10FA44BF9FED067A77EE677AAAE71A
:10F7200027D4D2360024F448DB0FC940E4CB16417D
:10F73000DB0F49C0E4CB16C1DB0FC93FDB0FC9BFEC
:10F7400092E741B99730083C15A82ABEF304353F2B
:10F7500000247448DB0F4940000000009FED2E7A22
:10F7600070EE077AFDEEE76A16EE903A2033402BF2
:10F770004FD8B4EEC70AF1EE10FA0CDD9FED276A00
:10F78000DFED276AB0EE677AB4EEE67AF1EE10FAB2
:10F7900077EEC67AF6DC9FED237AF4EEC77AF1EEC7
:10F7A00010FA0CD59FED1D6ADFED1F6AB0EE677A87
:10F7B000B4EEE67AF1EE10FA77EE867AF6D49FEDA3
:10F7C000167AF4EEC77AF1EE10FA1DDC9FED177A87
:10F7D000F4EEC77AF1EE10FA44BF9FED127A77EE9D
:10F7E000677A27EEA76ADFED125ADFED126A9FED06
:10F7F000127AE6EE256A67EE865AA6EE267AE5EEDE
:10F80000877AB0EE670A70479FED0C7A77EE677AD9
:10F81000E7E79FED0B0A7047DB0FC93FDB0FC940DD
:10F82000E4CB1641DB0F49C0E4CB16C1DB0FC9BFE7
:10F8300092E741B99730083C15A82ABEDB0F494032
:10F8400000000000F0EEC07AB0EEE07AB4EEE77AA5
:10F85000F1EE10FAB4BFB0EE676AB0EE476AB5EEEB
:10F86000406AF1EE10FA46D0B4EEE77AF1EE10FA03
:10F870008CBFF0EE675AF0EE475AC5EE866ADFEDB0
:10F880001F2ADFED1F3ADFED1F4A9FED1F5A9FED44
:10F890001F3A9FED1F4ADFED1F5AE6EEE23AA6EE51
:10F8A000834AE6EEA34AB7EE006AA6EEA45AA6EE95
:10F8B000846AE6EE855AC5EE866AB4EEE77AF1EE22
:10F8C00010FA48BFDFED147AF5EEC00A48BF77EEB4
:10F8D000E66AF1EE10FA48BFDFED107AB5EEC00A25
:10F8E00048BF77EEE66AF1EE10FA48BFF1EE666ABD
:10F8F000B0EE660A7047DFED076ADEE739094E3D74
:10F90000E3B59E3E88FA163E45FE7F3F99FB243FB5
:10F9100069A2163EA7DFA834DB0FC93FDB0F4940C1
:10F9200090ED005A9FED4C0A35EE000A08B5FDEE49
:10F93000C07A17EE903A2033402B7BD8FFF74CF873
:10F94000F0EE403AFDEEC57A17EE903A2033402BA8
:10F950007FD8B0EE450AFFF73FF8B0EE405AD0ED41
:10F96000014A9FED3D0A34EE800AFDEEC07A17EEA3
:10F97000903A2033402B69D8FFF72EF8F0EE405A2A
:10F98000FDEEE47A17EE903A2033402B5BD8B0EED0
:10F99000640AFFF721F8F0EE404A90ED023A9FED3D
:10F9A0002E0A33EE000AFDEEC07A17EE903A2033AD
:10F9B000402B45D8FFF710F8B0EE404AFDEEC37A71
:10F9C00017EE903A2033402B37D8B0EE430AFFF7BA
:10F9D00003F8F0EE407A24EE233A27EEA36A24EEF1
:10F9E000057A67EE856AB0EE462AF0EE432AA7EE66
:10F9F000242AE6EEE42AA6EE247AE3EE646A24EEF4
:10FA0000254A65EEE77A25EE655A65EEA35A81ED43
:10FA1000004AC1ED017AC1ED024A81ED032AC1ED30
:10FA2000042A81ED055AC1ED066A81ED077AC1ED20
:10FA3000085A08BDDFED093A84E7DFED087ACAE726
:10FA40009FED064ABAE7DFED054AA6E7DFED035A68
:10FA500096E79FED025A82E7DB0FC93F00000000E6
:10FA60002DE9F04389B0541C03941478002C00F065
:10FA700000810025074688461E46A94609E0214622
:10FA80003846C047039A0135531C03931478002C61
:10FA900040D0252CF3D1931CCDE903395078302880
:10FAA00002BFD31C03939078A0F13003DBB20CBFEC
:10FAB00001240024092B40F292806C2838D0782849
:10FAC00022D857282AD9A0F15803202B1CD8DFE8C8
:10FAD00003F0AA1B1B1B1B1B1B1B1B1B1B8B931B42
:10FAE0001B1B1B1B1B1B1B1BA51B1B1B1B111B9D64
:10FAF0001B1BAA0056F8043B049A009300234146BE
:10FB00003846FFF717F80544039A531C03931478FB
:10FB1000002CBED1284609B0BDE8F0830028F9D0FA
:10FB20002528F1D125213846C0470135039AABE796
:10FB3000039B5A1C039219787829A5D8572949D9CB
:10FB4000A1F15803202B9FD801A050F823F000BF4B
:10FB50003FFC000889FA000889FA000889FA0008C1
:10FB600089FA000889FA000889FA000889FA000869
:10FB700089FA000889FA000889FA0008E9FB0008F8
:10FB800057FC000889FA000889FA000889FA000879
:10FB900089FA000889FA000889FA000889FA000839
:10FBA00089FA000889FA00081FFC000889FA000891
:10FBB00089FA000889FA000889FA0008F5FA0008AD
:10FBC00089FA000863FC000889FA000889FA00082D
:10FBD0003FFC000800299DD02529A3D054E704AAA2
:10FBE00003A945F053FE68E756F8041B3846C9B22E
:10FBF000C0470135039A47E756F8040B05A9FFF7FC
:10FC00002FF805AB0093049A234678E756F8040BC7
:10FC100005AB00220A21FEF7DBFFF2E7039A56F854
:10FC2000043B1D6030E7A0F15802B2FA82F256F8A8
:10FC3000040B520905AB1021FEF7CAFFE1E7A1F161
:10FC40005802B2FA82F256F8040B520905AB1021A1
:10FC5000FEF7BEFFD5E756F8040B05A9FFF700F83D
:10FC6000CFE756F8040B05AB00220A21FEF7B0FFE0
:10FC7000C7E725464EE773B5114C01920646206D45
:10FC80000D46A0B10F49FFF799FA206D3146FFF7F5
:10FC900095FA0D49206DFFF791FA0C49019B206DF3
:10FCA0002A46FFF7DDFE0A49206DFFF787FA94F830
:10FCB000543013B1012384F8553002B070BD00BF39
:10FCC000D4990020916106082E670608B9F1000852
:10FCD0009E6106080EB400B584B005AB019053F8E0
:10FCE000042B0649039301A8FFF7BAFE019B0022EB
:10FCF0001A7004B05DF804EB03B07047B5EB000870
:10FD00002DE9F043002483B00646048021463046A6
:10FD1000013434F0E3FE082CF8D10023DFF86880CA
:10FD200086F8EA30C6F8EC30C6F8F030C6F8F430A1
:10FD3000C6F8F8301F46FC3699463A46414601A8B7
:10FD4000FFF7C8FF3546032401AA12F8013B6BB147
:10FD5000013C05F8013BF8D10137082F85F80090E8
:10FD600006F10406E9D103B0BDE8F0832846224637
:10FD70002021254401374AF084F9082F85F80090A6
:10FD800006F10406D9D1EEE7A81C0608F7B5114E16
:10FD900007463046002300F8563F0C460E4B0F49ED
:10FDA000002F08BF194615464AF073F90C4F04EBB3
:10FDB00045055636AC4202D10A4803B0F0BD39467B
:10FDC00034F8022B6846FFF785FF694630464AF053
:10FDD00060F9EFE7D4990020AB610608A26106083C
:10FDE000B46106082A9A0020F7B50C4E0C4F002388
:10FDF00006F8873F044600EB4105AC4202D10948B2
:10FE000003B0F0BD394634F8022B6846FFF762FFB5
:10FE1000694630464AF03DF9EFE700BFD49900202B
:10FE2000996406085B9A0020F8B5084F4E1E0546F7
:10FE300001F11F0416F8012F28463946FFF74AFF43
:10FE4000A64205F10205F5D1F8BD00BFB96106086B
:10FE50000246531C084605D1034B1A681B790A60F9
:10FE60000B717047014935E7F76006089A64060888
:10FE700010B5013114460DF049FB28B9054B1A683D
:10FE80001B792260237110BDC27903492046BDE869
:10FE900010401FE7F76006085861060803685A1CFF
:10FEA000026019700368090A5A1C026019707047D1
:10FEB00002681146531C036011F802CB0160D31C89
:10FEC0005178036093781B0443EA0123111D0160FC
:10FED000D07843EA0C0343EA00607047A0F1300396
:10FEE000092B07D920F02000413819288CBF0020A9
:10FEF0000120704701207047303809288CBF00204E
:10FF000001207047413819288CBF0020012070471C
:10FF1000613819288CBF002001207047202805D0A7
:10FF2000093804288CBF0020012070470120704749
:10FF3000A0F14103192B98BF20307047A0F1610355
:10FF4000192B98BF2038704710B500F100440246C5
:10FF5000013C04E0B3EB0E0015D1A24214D012F81C
:10FF6000013BA3F14100192811F8010BA0F1410C4C
:10FF700098BF2033BCF1190F00F1200EEAD91B1AEB
:10FF800004D10028E9D110BD002010BD184610BDD5
:10FF900002B310B58446841804E0B3EB0E0014D10C
:10FFA000A44513D01CF8013B11F8010BA3F1410249
:10FFB000192AA0F1410298BF2033192A00F1200E1E
:10FFC000EBD91B1A04D10028EAD110BD002010BDC6
:10FFD000184610BD1046704770B5044608460D46D9
:10FFE00047F05EFD064602E014F8013F43B12046AB
:10FFF00032462946FFF7CCFF0028F5D1204670BDD8
:020000040801F1
:100000001C46204670BD38B507490546FFF7E4FF9A
:100010000649041E284618BF0124FFF7DDFF08B17A
:1000200044F00204204638BDBE610608DA790608AD
:100030002DE9F041044686469EF800C0BCF1200F31
:100040007046ACF109050EF1010EF5D0042DF3D97F
:10005000BCF12B0F5BD0BCF12D0F3BD1102A4FF020
:10006000010600F1010E58D19EF800C0BCF1300F1E
:100070005FD04FF010086FF070450F2742460EF129
:10008000010E00200DE0ACF1300C5FFA8CFC9445C1
:100090000FDA854274462DD32AD008FB00C01EF823
:1000A00001CBBCF1390FEED94CF0200CBCF1600F44
:1000B0000BD801B10C600EB323B1B0F1004F28BFD3
:1000C0004FF000404042BDE8F081ACF1570C5FFAC0
:1000D0008CFCDCE7102A864649D04FF0FF35B5FB93
:1000E000F2F502FB05F7FF43FFB290460026C6E794
:1000F0006745D2D21E404FF0FF30D0E7002BE2D050
:100100006FF00043984228BF1846BDE8F081102ADE
:100110004FF0000600F1010EA6D04FF0FF35B5FB01
:10012000F2F502FB05F7FF4390F801C0FFB29046DD
:10013000A5E79EF801C0ACF1410019280EF10104B9
:10014000624601D80CF12002782A4FF0100805D041
:10015000A6466FF070450F27424690E79EF802C012
:100160006FF070450EF1020E0F27424687E700261A
:100170007AE773B50E4611490546FFF7E5FE18B953
:100180003070012002B070BD2C78602C8CBF613CB7
:10019000413C072C10D8013501230A2201A9284629
:1001A000FFF746FF019B9D4206D00F2804D801347B
:1001B00040EA04143470E4E70020E3E7F76006083F
:1001C00001230A22002133E770B50D461446FFF7DC
:1001D00007F80646A0B1FFF7F3FF40F63403984254
:1001E000A8BF1846B0F5617FB8BF4FF46170A0F5A5
:1001F00061731920B3FBF0F32B7023780133237064
:100200003046FEF7EDFF0646A0B1FFF7D9FF40F6F6
:1002100034039842A8BF1846B0F5617FB8BF4FF4C9
:100220006170A0F561731920B3FBF0F36B70237854
:1002300001332370304670BD2DE9F04117461E464C
:1002400005464FF47A7200233846314648F0ECF800
:100250004349444A014482FB0143C8170B44C0EBA5
:10026000631382FB03021A44D8173F4CC0EB62129F
:1002700084FB02044FEAE27C3C48CCEBA40C80FBFC
:100280000C404FEAEC74C4EBE010C3EB0314A1EB99
:100290008401A971C2EB0211A3EB81036B710CEB1A
:1002A0004C03A2EBC30240F2B55303FB10CCBCF5E8
:1002B000896F2A714FEA800043DA40F2DA239C45C5
:1002C00046DCBCF5B77FB4BF00220122284B02EB0D
:1002D000420103EBC1034FEA42085B8D91B2254C0A
:1002E00008EB020E04EBCE0416344FF00B0E01E0C7
:1002F00034F8023D63451FDDBEF1010EF8D11C4B01
:10030000424403EBC2024FF0010E938A85F802E0EB
:1003100000F5FA600CF1010C0844ACEB030C2880EA
:1003200085F803C04FF47A7200233846314648F00E
:100330007BF82A81BDE8F0810EF1010E5FFA8EFE96
:10034000E4E7032140F296530A464FF00608C6E759
:10035000022140F229430A464FF00408BFE700BFDC
:1003600080BC92C789888888ABAAAA2A73B06D1608
:1003700098BD0508ACBD050808B50C4BD3E90023B2
:1003800052EA030C09D1002340F20112428083801B
:10039000837103800381184608BD054909688A18DE
:1003A00043F10003FFF748FF012008BD0835002096
:1003B0002C21002090422DE9F0410B4604461546C1
:1003C0000AD2B0FBF5F6134A05FB16441846135D36
:1003D00000F8013BBDE8F081B0FBF2F69642B6FBB7
:1003E000F2F706D20B4A05FB1767D15D03F8011B34
:1003F000EAE7BA42B7FBF2F807D9064A05FB1878D4
:1004000012F8081003F8011BEDE74046FFF7D2FF92
:100410000346F2E7B01C06087D4B9A88B3F808C083
:1004200058899989B2F57A7F88BF4FF47A7230B5CE
:1004300088BF9A80DA88774CB2F57A7F84BF4FF410
:100440007A72DA80BCF57A7F84BF4FF47A7CA3F8A5
:1004500008C0B0F57A7F88BF0020DA8988BF58814C
:10046000B1F57A7F84BF4FF47A719981B2F57A7FC2
:1004700084BF0022DA8184459CBF0020188191420C
:1004800098BF0022598B98BF9A819A8B914284BF62
:1004900000225A83604B1B8883B0002B43D06279C3
:1004A0005E4D012A63D9AA78062A97BF5C499FED61
:1004B0005D7A01EB820191ED1D7A2979002940F0E6
:1004C00084805949087807EE903A06EE900AF8EED3
:1004D000E77AB8EEE66AAB79C6EE276A002B6CD1F4
:1004E000B4EEE67AF1EE10FA1DDD67EE277ABCEE87
:1004F000E77A8DED017A9DF8042007EE102AB8EE18
:10050000C77AF4EEC77AF1EE10FAC4BF0132D2B264
:10051000002A6ED0102AA8BF1022D2B282421346FF
:1005200038BF03460B7063782278032B95BF3F4991
:100530003E49C3EB0313002394BF01EB43016370F7
:100540003B4B032AC3F8B8139DBF02EB820103F5AE
:10055000947302EBC102002294BF03EB820322706A
:10056000344A88BF03F59473136003B030BDAA7991
:10057000002A98D0AA78072A09D0B3F57A6F93D9C0
:10058000294908780228B8BF022008708CE70622A3
:10059000B3F57A6FAA702ED82A79002AC3D12249DE
:1005A0009FED257A087807EE903A06EE900AF8EE6D
:1005B000E77AB8EEE66AC6EE276A37EE077AB4EE57
:1005C000E67AF1EE10FAAEDD8FE7042A02D8002AAF
:1005D000A9D002E0053A032AA5D9B7EE000A80EEB9
:1005E000070A48F073FF2B88984228BF18462880D6
:1005F00099E7012291E70C490A78022AB8BF022242
:100600000A702A79002A8ED19FED0B7A5AE700BF33
:100610006C370020243500201C0F00108827002094
:1006200098BD05086F12033828370020849A0020EF
:10063000D49900203037002017B7D1382DE9F04F7A
:10064000B64B83B01B78A3F11702022A00AF05D97D
:10065000B34A12F83310002940F05B8243F0A0FF48
:10066000002800F02F83DFF8EC820024022088F8B5
:100670002C4411F05BFD98F83034022B00F0BE8260
:10068000002800F04783A74BDFF8CCB27B60A64B75
:1006900098F8899403F5247E4FF47A7C00254FF076
:1006A000640A5A88B2F57A7FB3F8462088BFA3F867
:1006B00002C0B2F57A7F9A8888BFA3F846C0B2F527
:1006C0007A7FDA8888BFA3F804C09988B2F57A7F68
:1006D00084BF0022DD809142B3F85A10B3F85C2049
:1006E00098BF9D80914293F86B2088BFA3F85A5021
:1006F000013A632A93F86C2088BF83F86BA001321B
:10070000D2B2092A88BF83F86C5003F166011A46F9
:100710000326947A11F8010B844238BF01F8015C7A
:10072000013E02F10602F4D1B9F1010F18BF83F8BE
:100730008560A4337345B4D17C4B9B78042B00F0C7
:10074000C8823BB9794A1388B3F5F07F84BF4FF470
:10075000F0731380764CFFF75FFEE17904F1080037
:10076000FEF774FC617D04F11600FEF76FFCB8F82B
:10077000A224B8F8A0341343B8F8A42413431BB23E
:1007800013B10123A8F8A6347B686A4A1B681A4093
:10079000002A00F0D782DA0700F117825D0440F1E9
:1007A000C28165497A680B401360DBF800200A407B
:1007B000CBF8002013F4004200F0DD81002288F81D
:1007C000BB2488F8CB24D90440F1DF8198F8EB34BE
:1007D000DFF86891022B04BF012388F8EB3409F19C
:1007E00078044B4602E00633A3420CD01A78072A5D
:1007F000F9D19978DA78914202D35A79002AF2D065
:10080000072021F00BFE00234FF4806088F82C3481
:1008100011F08CFC002800F07182484DAA469AF82D
:10082000051079B19AF8000050B14B4602E006334A
:10083000A34207D01A788A42F9D15A79002AF6D011
:1008400021F0ECFD0AF1060A5445E8D1374B93F844
:100850000290B9F1080F00F0C68198F88A1498F850
:100860008904374BDFF8F4C0DBF80020A1F1010167
:10087000B1FA81F14909A0F101001971B0FA80F0D3
:100880009CF80110400918700329C2F3C030987019
:1008900084BF00238CF801302A4B2B49987B7B685E
:1008A0001B680A400B407968CBF800200B600028D9
:1008B00000F0FA81DFF8A8B0BBF80430002B40F05C
:1008C000C181224A136813F07F4F1CBF00231360BD
:1008D000936823F4007323F0020313B140F2022360
:1008E00093601379013B042B88BF0123A9F105090B
:1008F00088BF1371B9F1030F40F25A81144B93F87A
:1009000000A0BAF1000F42D000237B60074A6FF0CD
:100910000703A3EB020B02F1080928E0D9350020F8
:100920005CB50508CC3B0020FC9A002088270020FD
:100930008036002009600002F6DFFFFDC49E002023
:100940008464002024350020DEDDCDFD3437002016
:10095000C00D0010D4990020603500206C370020B5
:10096000986400200BEB09039A4540F2E08019F8E7
:10097000010B0028F6D00CF0F3FD0028F2D08379AB
:100980009B07EFD57A680123002A40F0D580B24B4F
:100990009B7913B1B04A00239371B04BDA8812F0FF
:1009A0000C0F03D1C2F30312022A02D94FF42062C2
:1009B000DA801A8912F00C0F03D1C2F30312022A53
:1009C00002D940F601221A8198F8753598F8692500
:1009D0009A4298F8683505D9002288F8692553B1FC
:1009E000A8F86C2598F874259A423EBF002388F831
:1009F0006835A8F86C3598F85E3698F86A25DFF8FF
:100A00009CC29A4284BF002388F86A350CF1780BA7
:100A10001CF8012C924902EB42020A44634692F808
:100A200090A092F8919092F892E000201A785245A6
:100A3000A8BF524603F8012B59799A784945A8BFB7
:100A4000494601307245A8BF7246032859719A7011
:100A5000ECD10CF11E0CDC45DAD1D8F8DC24002AEC
:100A600000F02A81002001212B78282B07D16B78F8
:100A7000043301FA03F313421CBF9A4301200635E5
:100A8000AC42F1D108B1C8F8DC24764D05F1080478
:100A90002B4613F8012B072A5BD89C42F9D1EA4672
:100AA00088B0E9462022FF21484649F0EAFA6D4A1B
:100AB00012F8013B59F82310013151D1944249F801
:100AC0002330F5D1B8F88224B8F880349A42D5465C
:100AD00002D3654BC8F88034644B654CFF2288F81C
:100AE000902603F16C0093F90420142A04D01968AD
:100AF00034EA010100F0EA800C338342F3D15D4B0C
:100B00005A79022A01D100225A710C37BD46BDE83C
:100B1000F08F02EBC3035B68002B7FF49FAD564A56
:100B2000172313709AE51C0758D554493AE67A689A
:100B30000023002A3FF42BAF47494A7C002A7FF468
:100B40002CAF4A79012A3FF422AF002B7FF41FAF6C
:100B500023E7EA4688B02022FF21684649F091FA4F
:100B600005F8016B0136082EACD005F8016B013693
:100B7000082EF5D1A6E798F8BB1400293FF423AE60
:100B8000D90488F8CB243FF521AE1A067FF51EAEB6
:100B9000394B1978182906D8394B01228A4013405D
:100BA000002B7FF413AEDFF8F89009F178042AE601
:100BB000294A00231371334B93F800A0BAF1000FB8
:100BC00000F0B78001237B60A0E62F497A680B40D4
:100BD0001360DBF800200A40CBF8002098047FF572
:100BE000E9AD2A49DEE51A469B79002B3FF435AE84
:100BF000537C012B04BF022353742EE600283FF4DC
:100C000042AD234D234B297890F904604FF0FF0C3F
:100C100003F16C0093F90820B24204BF01F1FF31E7
:100C200083F808C003F10C0304BFC9B20124834256
:100C3000F0D1194BDFF86CB07B60002C3FF427AD8E
:100C4000297024E59BF800000CF08AFC00287FF452
:100C500038AEABF8040034E688270020A43A002020
:100C600098BD05089B270020AE014A01909D0020F9
:100C700001000200B4260020D9350020FE9FFFFDB0
:100C800000410001C00D0010F79FFFFDF6BFFFFD02
:100C90006435002068350020CC3B0020879A002076
:100CA000C49E0020603500202C4978680B430A431D
:100CB0000360CBF80020FDE5282021F0AFFBD8F839
:100CC000DC24CFE6264811F0EDF9CCE488F8902634
:100CD00015E77A68136823F480531360DBF800305B
:100CE000204A23F48053CBF80030538CB3F57A7F3D
:100CF000BFF430AD4FF47A7353842BE57A681368F0
:100D000023F000631360DBF8003023F00063CBF8BE
:100D1000003082E51449DFF854B00A68DBF800308F
:100D2000796022F0800223F080030A60CBF8003063
:100D3000ADE4537C002B7FF430AE5379012B7FF46C
:100D40002CAE24E67A6843F008031360DBF8002039
:100D500042F00802CBF800201DE500BF00040500AA
:100D6000909D002088270020CC3B0020603500208B
:100D70002DE9F04FDFF80C82754BD8F80C2002F209
:100D8000DC52C8F80C20734A934283B080F0DC80B8
:100D900003F11C059B46704B704E4FF0010A9F1CDF
:100DA0006D4B5A88002A00F0B880BB18B34280F01F
:100DB000B4803C4608E01A881C461344002A00F020
:100DC000AC80B34280F0A980052A40F2A68035F8B5
:100DD0001C2C6188C2F30B029142ECD1627992071C
:100DE000E9D1238855F8141C94F8049001935846CF
:100DF000FEF732FB35F81C2CB9EB123F00F0958062
:100E00004FF0000A35F8181C55F8140CC1F30B010B
:100E100043F0AEFB55F8043C18604E4B0BF11C0B35
:100E20009B4505F11C05BBD34D4A4E4B4E4F1268F6
:100E30001A60FFF703FC3B784C4C4D4D7A784D4ED1
:100E400003EB830103EBC10304F5947101EB83030E
:100E50002B60C2EB021204F1B00303EB4202C4F8B0
:100E6000B82320F0FFFC4FF0FF33286873602BF0AD
:100E700017FA21F027FB04F59E6304F5AD6102E04B
:100E800006338B425BD01A78002AF9D19D78D87846
:100E9000854202D358790028F2D094F8E8343272AF
:100EA00003EB830303EB83039B00632BB4F8EC2475
:100EB000D8BF6423C8F80430642303FB02F2632A1A
:100EC000DCBF1A46C8F808304FF00003C8BFC8F8A6
:100ED0000820C8E90732284AA8F82430C8E90333B3
:100EE000C8E9053388F82630244B93622BF0FEFFC7
:100EF000B4F8940694F8961622F056F936F0B2FC3F
:100F000016F0DAFD1E4A1268C8F80C20012350467C
:100F100088F8253003B0BDE8F08F55F8141C58460A
:100F2000FEF79AFA4FF0000A6CE7019BA11D9A1F89
:100F30005846FDF74FFC00287FF464AF60E7FA7B6A
:100F4000003A18BF0122A8E74FF0010A6CE700BF82
:100F500044A9060878B1060800400008008000088F
:100F6000CC3B00206035002024350020D49900209F
:100F70003037002094050020AC140010749E00202F
:100F80002C2100204037002038B51C4B01220328BB
:100F900005461A7020D96A1CD2B252001848402A5D
:100FA00028BF4022002300F5D36102244FF0140E25
:100FB000CC54023301EB030C9A420CF801ECF7D845
:100FC000FF2D08BF02220244FF2382F89836BDE8B5
:100FD00038400E200CF03ABE05EB850309480A4A5A
:100FE00005EBC30300EB8300084B157018602BF072
:100FF00057F922F02FFC22F003FDCCE7E01400109B
:10100000D4990020FC9A002024350020303700209D
:10101000054BD3F8DC26012142F4001283F8D916DF
:10102000C3F8DC26704700BFD4990020F8B5164DF0
:101030006B78BE2B26D1022229464FF6FF70FDF7B2
:101040006DFC124FAC1C22884AB1A618BE4219D2C0
:10105000052A17D92146FDF761FC3446F3E72146FE
:101060000222FDF75BFC0222A118FDF757FC0634B3
:10107000074B641BA3F8E04641F60F53C31A5842CE
:101080005841F8BD0020FCE700400008008000083F
:10109000D4990020F8B50468C4F30D0406460F4641
:1010A0000CB335683F6840F017F8092840F0878096
:1010B000444C236923F440732361236943F4007390
:1010C0002361236943F0010323612F6040F004F89A
:1010D0002369092823F00103236170D133680433A5
:1010E0003360002034E0384B384A93422AD302F56B
:1010F0008042934225D302F58042934229D3344A59
:10110000934228D902F58032934226D902F5003263
:10111000934224D902F50032934222D902F50032DB
:10112000934220D902F5003293421ED902F5802263
:1011300093421CD9B3F1016F1BD345F0BFF844F0C3
:10114000FDFB08243FF0C8FF092814D04FF0FF3002
:10115000F8BD1024F6E71824F4E72024F2E7282449
:10116000F0E73024EEE73824ECE74024EAE74824AF
:10117000E8E75824E6E7134D2B6923F440732B610D
:101180002B6943F400732B612B6923F0F8032B6167
:101190002B691C4344F002042C612B6943F4803317
:1011A0002B613FF099FF2B6923F002032B612B6920
:1011B000092823F0F8032B613FF473AFC6E76FF003
:1011C0000100C5E7003C0240004000080040000864
:1011D000FFFF00082DE9F041574F3B78B12B8AB053
:1011E0006FD1FFF723FF80F00104E4B2534B544D5D
:1011F000B3F89F30534EADF8003004F00104B5420F
:1012000061D3002C00F096801022002106A848F03F
:1012100038FF4D4B0497DB1B05934C4B484F1A6925
:10122000002ABFBF4A4A5A6002F188325A6001223E
:101230008DF82420F322DA606946022204A80025F2
:10124000089546F063FA022269464FF6FF70FDF7F3
:1012500065FB0446B74243D3022201A904A8002536
:10126000ADF8045046F052FA022201A92046FDF7DB
:1012700055FB40BAC043ADF80800022204A802A9F9
:1012800046F044FA079868B106ABC0F1040229465B
:10129000184448F0F6FE089818B906A904A8FFF704
:1012A000F9FE08909DF82430089823B1274A136965
:1012B00043F000431361B0FA80F040090AB0BDE882
:1012C000F081012492E7A988A868C1F30B0143F0DB
:1012D0004FF9AB691B681C35834218BF01248EE7A8
:1012E000B7F804808DF80D50C8F30B0808F1060319
:1012F000ADF808303B88C3F30B02ADF80A201B0B96
:10130000062202A904A88DF80C3046F0FFF9062247
:1013100002A92046FDF702FBB9680446424604A82C
:1013200046F0F4F9B96820464246FDF7F7FA1C3753
:1013300004468FE70120C1E70040000898BD05087A
:1013400044A9060878B1060800800008003C024065
:101350002301674538B5184C184DFFF76FF9E3685E
:10136000012203F2DC53E36085F8E226FFF732FF47
:1013700010B9FFF72FFF50B1114B1B78B12B02D1E1
:10138000FFF754FE58B944F099FF44F0D7FAFFF73D
:1013900021FF0028F0D144F091FF44F0CFFA094A30
:1013A0000023116885F8E2360122E16084F82520E7
:1013B00085F8E33638BD00BF40370020D4990020BF
:1013C000004000082C21002008B50B490B4A0123DE
:1013D0000B709373FFF7BEFFFFF7CAFC084B41F297
:1013E0000241FF22A3F8981683F89A26BDE8084028
:1013F0000E200CF02BBC00BFE014001024350020A0
:10140000D499002090F88730DFED6A5A03EE903AC5
:1014100090F88B3006EE103A90F8893004EE103ACE
:1014200090F88A30F8EEE33A04EE903A90F88D3076
:1014300063EEA57AB8EEC66A03EE903A26EE256A08
:10144000B8EEC44AF8EEE44AF8EEE33A26EE276A2C
:1014500024EE254A64EEA54A63EEA53AF0B5564D52
:1014600024EE064A64EEA74A63EEA73A0021062658
:10147000F7EE002AA5F10C0C00F1660E06FB01F256
:10148000B7EE005AAC1890F886700244F0EE456A48
:1014900015E0012904F1060402F10602EED190F8EC
:1014A000883007EE903A90F8903006EE903AF8EED9
:1014B000E77AF8EEE66A27EEA55A66EEA56A237883
:1014C00007EE103A66EE867AB8EEC77A27EE277AEC
:1014D000FDEEC77A17EE903AFA2BA8BFFA2323EA5B
:1014E000E3731372637807EE103A66EE847AB8EE0F
:1014F000C77A27EE277AFDEEC77A17EE903AFA2BD5
:10150000A8BFFA2323EAE37353725CF8213007EE95
:10151000903A002BF8EEE77A49DDA37807EE103A0F
:10152000B8EE477A90F88C3037EE677A03EE103ACF
:1015300087EE272AB8EEC33AB0EE627A23EE253A58
:10154000A2EE037A64EEA77A66EEA36A67EE857A66
:1015500027EE877AFDEEE77ABDEEC77A17EE103AEE
:10156000FA2BA8BFFA2323EAE373937217EE903A9B
:10157000FA2BA8BFFA2323EAE3730EF80130A388FD
:1015800007EE903AF8EEE77A013167EEA67AFDEEC3
:10159000E77A17EE903AB3F57A7FA8BF4FF47A73E3
:1015A00023EAE3738F429381BFF673AFF0BDB7EECA
:1015B000007AC7E70AD7233C48BE050890F88E306A
:1015C0006BB3B0F85A308BB190F88F2002EB8203E6
:1015D0006421C3EB0313B3FBF1F3A0F85A30962355
:1015E00012FB03F3B3FBF1F3A0F85C3043884BB17B
:1015F00090F88F3003EB8303C3EB03136422B3FB38
:10160000F2F34380B0F846304BB190F88F30962219
:1016100013FB02F36422B3FBF2F3A0F846307047E9
:1016200090F821304BB3438B83B190F82230FA22EB
:1016300013FB02F203EB8303B3F57A7FA8BF4FF4E9
:101640007A7364218383B2FBF1F24283838843B1CE
:1016500090F82230FA2213FB02F36422B3FBF2F378
:101660008380C3884BB190F8223003EB8303B3F53A
:101670007A7FA8BF4FF47A73C380704770B50A4C65
:101680000A4E002594F8863013B12046FFF7BAFEC3
:101690002046FFF793FF01353046FFF7C1FF042DC9
:1016A00004F1A404EED170BDFC9A00206C37002038
:1016B000034BD3F8E40608B106F044BE704700BF00
:1016C000D499002008B50B4605490246D1F8E40636
:1016D00028B10449FEF7C4F9BDE80840E8E708BDB1
:1016E000D4990020B9F10008024B0146D3F8E40672
:1016F000FDF764BDD499002008B504460848FFF7FB
:10170000F3FFFFF7D5FF074BD86C15F04BF80BF044
:10171000FDFA012C01D144F011F9FAF799FC00BF50
:10172000C1610608D49900200048DDE74376060829
:101730000CB4C30607B500D561B9049805A9019199
:10174000FFF7C0FFFFF7F0FF012003B05DF804EBE7
:1017500002B070470020F8E70FB407B504A951F8AC
:10176000040B0191FFF7AEFFFFF7DEFF03B05DF85A
:1017700004EB04B070470349034801F521610EC929
:10178000EAE700BF0070FF1FCD61060810B57521A4
:1017900004462BF055FE01460948FFF7DDFF1A21EC
:1017A00020462BF04DFE01460648FFF7D5FF1B21D2
:1017B00020462BF045FEBDE8104001460248CBE72D
:1017C000E1610608F46106080762060838B50B4DAA
:1017D000E87810F0FD0405D10948FFF7BDFF204669
:1017E000FFF7D4FFEB78013B012B06D80548FFF744
:1017F000B3FFBDE838400120C8E738BD6C37002092
:101800001A6206082562060808B5FFF76DFFBDE8F5
:10181000084089E72DE9F04387B0FCF771FA0269C7
:10182000838901880292826801924288009242680C
:101830001B4EDFF880801B4FDFF87C9004461A486F
:10184000FFF78AFF002515B94046FFF7DDFF3B682B
:101850009D4213DA33781548052B96BF09EB8303B5
:101860000022D3F8C420B388009329467388013539
:10187000FFF772FF062D06F10606E4D144F02CF8BE
:1018800081884388CB1A616803FB01110591FCF73D
:10189000C1FA05990246064807B0BDE8F0435BE788
:1018A00014300020842F0020306206089A62060857
:1018B000A96206088E62060898BD050810B50446A0
:1018C0000348FFF711FF2046BDE810409CE700BF2A
:1018D000C662060808B5034610462AB1DB0600D5E5
:1018E00011B1FFF7EBFF002008BD2DE9F04F2DED02
:1018F000028B0A468BB000218246FFF7EBFF6F4D4B
:10190000814605F1800B00266D4B1C79AB7AB34202
:1019100000F395801035AB45F5D140F21620FCF769
:1019200043FFD0E902530CB12C461D460DF1100BBC
:1019300015220021584648F0A4FB00272E78002EDF
:1019400044D06978039130460BF0E0FD95F9023000
:1019500002935A1C534208EE100A5341002C00F027
:10196000A9800399002214F802C0B44504EB0200D8
:1019700040F09C8090F90280029A424540F09480A9
:1019800042788A4208BF012301220BF8072003F0A6
:1019900001034A4683F0010150460393FFF79AFF83
:1019A000039B81464CB1474A18EE101ACDE900A2BC
:1019B00030464246FDF7C2FC039B434A18EE101A1C
:1019C000CDE900A23046029AFDF7B8FC0137152F89
:1019D00005F10305B2D16CB33A4FDFF8EC8004F1A6
:1019E0003F061BF8013B02930BBB2078F8B194F93A
:1019F000022001321BD061780BF088FD4A46054673
:101A000001215046FFF766FF94F90220029B294608
:101A100081462078CDE900A7FDF790FC2078029B55
:101A2000CDE900A84FF0FF322946FDF787FC0334CB
:101A3000B442D6D10BB0BDEC028BBDE8F08FE88884
:101A4000FCF7B2FED0E902230CB114461A46297AFB
:101A50006B7A06FB013312F9038014B3E756B845DD
:101A60000CBF012300234A4614BF01210021504628
:101A70000293FFF72FFF029B814644B1114A314682
:101A8000CDE900A228463A46FDF70CFC029B0E4A1F
:101A90003146CDE900A228464246FDF703FC013657
:101AA00032E74FF0FF37DAE700236DE703323F2AD2
:101AB0007FF459AF4FF0FF386BE700BFA00500205F
:101AC000D49900203D1C01083117010808B50948C8
:101AD000FFF7F4FEFFF7ECFD074B002483F8E84620
:101AE000C3F8E84783F8EC4722F05AF82046FFF79E
:101AF00003FE00BFCB620608D49900202DE9F04F09
:101B00008BB0074640F216200391FCF74DFE039A76
:101B1000044600213846FFF7DDFE404AD4E902536F
:101B2000147906460CB12C461D461522002104A846
:101B300048F0A7FA05F13F03039395F80090B9F137
:101B4000000F31D095F801A0002C65D0224600236B
:101B50001178494558D128336B4492F8018001220D
:101B600003F8182CD045324614BF01210021384615
:101B70000CBF4FF0010B4FF0000BFFF7ABFE06461A
:101B800054B1B8F1000F07D0254B00935A463B469D
:101B900041464846FDF716FC224B00935A463B4609
:101BA00051464846FDF70EFC039B03359D42C4D1C8
:101BB0003CB3DFF86C90DFF86CA0651C0DF11008E9
:101BC000403418F8013BCBB915F8013CB3B116B15C
:101BD0003046FFF773FE297815F8010CCDF8009018
:101BE0003B460022FDF7EEFB002215F8010CCDF874
:101BF00000A03B461146FDF7E5FB00260335A54254
:101C0000DFD10BB0BDE8F08F0133152B02F10302D9
:101C10009ED14FF00008A5E7A046A3E7D499002085
:101C20003D1C010831170108034B0146D3F8E406B7
:101C300008B106F073BB7047D49900200CB407B507
:101C400010F020000BD079B92320FFF7EDFF0498A6
:101C500005A90191FFF736FDFFF766FD012003B0EE
:101C60005DF804EB02B070470020F8E72DE9F04F73
:101C7000914689B00C461A4600218046FFF72AFE9D
:101C8000DFF8ECB006464D460027B9F1000F6CD0E6
:101C900029460622204648F0CAF90028324614BFD9
:101CA0000121002140460CBF4FF0010A4FF0000A0D
:101CB000FFF710FE0646287815F0D2FE079010B305
:101CC000687915F0CDFE079BEA785B790793AB78CE
:101CD00095F801E04FF461714FF0190C1CFB0313F0
:101CE0001CFB0212297900B14079CDF804E0CDE95E
:101CF0000232079B0093CDE904103B465A465146F9
:101D00004046FFF79BFF207815F0AAFE079010B31E
:101D1000607915F0A5FE079BE2785B790793A378BD
:101D200094F801E04FF461714FF0190C1CFB0313A0
:101D30001CFB0212217900B14079CDF804E0CDE915
:101D40000232079B0093CDE904103B465A465146A8
:101D50004046FFF7EDFC0137142F04F1060405F1AE
:101D6000060592D109B0BDE8F08FCA46CBE700BFA7
:101D7000F26206082DE9F04F174689B01A460C4664
:101D800000218146FFF7A6FD3B4EDFF8F4B007F1D6
:101D90006C0380463D46079394F90410374A0023AC
:101DA00092F90800884263D00133092B02F10C023A
:101DB000F6D1079B0C359D4204F10C04ECD109B01F
:101DC000BDE8F08F29460C22204648F030F9002863
:101DD000424614BF0121002148460CBF4FF0010AC2
:101DE0004FF0000AFFF776FDEA7995F9043006EB2B
:101DF00082028046D2F8DC2004922A7A06EB820224
:101E00005146D2F8DC200392AA7906EB82024846BA
:101E1000D2F8DC2002926A7906EB8202D2F8DC204A
:101E200001922A6800925A46FFF708FFE27994F976
:101E3000043006EB82025146D2F8DC200492227A6A
:101E400006EB82024846D2F8DC200392A27906EB28
:101E50008202D2F8DC200292627906EB8202D2F88A
:101E6000DC200192226800925A46FFF761FCA0E74D
:101E7000002FA7D1BA46D9E798BD050868350020DC
:101E80000B6306082DE9F04F8BB00C460892002139
:101E90001A460746FFF71EFDDFF8B4B0089D09900B
:101EA00000264FF019094FF46178089B002B4BD0A6
:101EB00029460A22204648F0BAF80028099A14BF99
:101EC0000121002138460CBF4FF0010A4FF0000AF3
:101ED000FFF700FD2A890692EA8805922A79049282
:101EE000EA780392AA78099019FB028202926A7832
:101EF00019FB028201922A78009233465A465146D3
:101F00003846FFF79BFE22890692E28805922279E5
:101F10000492E2780392A27819FB0282029262781C
:101F200019FB0282019214F80A2B009233465A469A
:101F3000514638460136FFF7FBFB1E2E05F10A0518
:101F4000B3D10BB0BDE8F08FDDF820A0DBE700BF18
:101F5000286306082DE9F04F2DED088BDFF82CA142
:101F600095B0804691461F460C4616464FF0000B32
:101F700094ED008AB5EE408AF1EE10FA7FD0D4EDF0
:101F8000019A94ED029AD4ED038AB9F1000F49D079
:101F9000D6ED00BA96ED01BAD6ED02AA96ED03AAE7
:101FA000B4EE6B8AF1EE10FA6ED1F4EE4B9AF1EECC
:101FB00010FA69D1B4EE6A9AF1EE10FA64D1F4EE37
:101FC0004A8AF1EE10FA0CBF012100213A460D4673
:101FD000404681F00101FFF77DFCB0EE6B0A074639
:101FE00011A8FDF77BF8B0EE4B0A07900EA8FDF79D
:101FF00075F8B0EE6A0A06900BA8FDF76FF8B0EE20
:102000004A0A059008A8FDF769F80599069A079B02
:10201000039002910192009352465B462946404646
:10202000FFF70CFEB0EE480A11A8FDF757F8B0EE26
:10203000690A05460EA8FDF751F8B0EE490A069068
:102040000BA8FDF74BF8B0EE680A059008A8FDF75D
:1020500045F8069B059A0390CDE9005302925B4632
:102060005246002140460BF1010BFFF761FBBBF12B
:10207000080F04F1100406F110067FF479AF15B0D3
:10208000BDEC088BBDE8F08F00219FE74B6306088D
:102090002DE9F74F92460C461A4600218146FFF77C
:1020A00019FCDFF870B0804656460025BAF1000FE3
:1020B0002ED031460422204647F0B9FF0028424680
:1020C00014BF0121002148460CBF01270027FFF75C
:1020D00001FC738801933AF82530009380462B4623
:1020E0005A4639464846FFF7A9FD6388019334F8FC
:1020F000043B00935A462B46394648460135FFF7C4
:1021000017FB042D06F10406D0D103B0BDE8F08F13
:102110005746EAE75F6306082DE9F04F89468FB01E
:10212000174600211A460646FFF7D4FBDFF878A0D1
:10213000054600240DF1240B59F82430029359462A
:1021400002A840F0B3FA67B357F82430029A039319
:10215000934218BF01212A4608BF002130460CBF18
:102160004FF001084FF00008FFF7B4FB04A9054643
:1021700003A840F09BFA04A9009123465246414629
:102180003046FFF75BFD2346CDF800B0524641468E
:1021900030460134FFF7CCFA202CCDD10FB0BDE88A
:1021A000F08FB846EFE700BF706306082DE9F04FE7
:1021B000924685B00C461A4600218146FFF78AFBFD
:1021C000DFF874B0804655460026BAF1000F31D0D2
:1021D00029460422204647F02AFF0028424614BF21
:1021E0000121002148460CBF01270027FFF772FBA1
:1021F000EB780293AB7801932B88009380463346AB
:102200005A4639464846FFF719FDE3780293A3780A
:10221000019334F8043B00935A4633463946484606
:102220000136FFF785FA102E05F10405CDD105B072
:10223000BDE8F08F5746E8E77A6306082DE9F04FCE
:1022400087B0144603911A4600210546FFF742FB6A
:10225000DFF830B106464FF00008062303FB08F70D
:10226000C0374FF00009039BDB5D0493002C00F0A6
:102270008580E35D049A05939A4218BF0121324696
:1022800008BF002128460CBF4FF0010A4FF0000A9A
:10229000FFF720FB059B0646CDE900935A464346CF
:1022A00051462846FFF7CAFC049B5A46CDE90093E5
:1022B00051464346284609F10109FFF739FAB9F1B9
:1022C000060F07F10107CED108F10108B8F1060F9A
:1022D000C3D1DFF8B0B0E427039BA7F1E40913F8FA
:1022E00007A0002C4CD0E35D04939A45324614BFFE
:1022F0000121002128460CBF4FF001084FF00008D3
:10230000FFF7E8FA049B0646CDE900935A460623F8
:1023100041462846FFF792FCCDE9009A194A062368
:10232000414628460137FFF703FAEF2FD4D1039B2C
:1023300093F8EF70B4B194F8EF804745324614BF7C
:102340000121002128460CBF01240024FFF7C2FA16
:10235000002300930B4ACDF804800723214628462A
:10236000FFF76CFC00230093064A019707232146E0
:102370002846FFF7DDF907B0BDE8F08FA24693E7E6
:10238000A046C9E78C6306082DE9F04F89B00C46DA
:10239000079200211A460746FFF79CFA0026079D80
:1023A000DFF8A0B00690B2464FF019094FF46178FB
:1023B000079B43B329460622204647F038FE0028F3
:1023C000069A14BF0121002138460CBF4FF0010AC4
:1023D0004FF0000AFFF77EFA6A79069019FB028235
:1023E00005922A7919FB02820492EA780392AA786C
:1023F00002926A7801922A78009233465A465146F0
:102400003846FFF71BFC627919FB0282059222799C
:1024100019FB02820492E2780392A2780292627817
:10242000019214F8062B009233465A46514638461C
:102430000136FFF77DF90A2E05F10605B8D109B07E
:10244000BDE8F08FA06306082DE9F04F0F4689B074
:10245000144600211A460646FFF73CFA0546002CB2
:1024600000F0DB8022783B789A4218BF01210246B7
:1024700008BF002130460CBF4FF001084FF00008A4
:10248000FFF728FA23789B4A054641463046FFF776
:10249000D5FB3B78974A41463046FFF749F9002C77
:1024A00000F0BD8062787B789A4218BF01212A46ED
:1024B00008BF002130460CBF4FF001084FF0000864
:1024C000FFF708FA63788C4A054641463046FFF725
:1024D000B5FB7B78884A41463046FFF729F907F17A
:1024E000CA030493822304F1CA0B05934FF0020937
:1024F0004FF0000A3B78534500F39380002C00F026
:10250000F38097F8EA3094F8EA209A4218BF012144
:102510002A4608BF002130460CBF4FF001084FF09B
:102520000008FFF7D7F994F8EA30744A05464146A7
:102530003046FFF783FB97F8EA30704A4146304651
:10254000FFF7F6F807F1EC09002C00F0CF8004F15A
:10255000EC034A4604F1FC014FF001089A4633F8B7
:1025600002CB32F8020B844518BF4FF000088B42B3
:10257000F5D188F001012A46C9B23046FFF7AAF921
:10258000082105465046FDF72FFC5D4A03464146AB
:102590003046FFF753FB97F8EA104846FDF724FC56
:1025A000574A034641463046FFF7C2F8002C00F078
:1025B0009F804FF0FC094FF0010807EB090104EB85
:1025C0000900FDF7C1FC09F10409002818BF4FF00C
:1025D0000008B9F58E7FF0D188F001012A46C9B212
:1025E0003046FFF777F9082104F1FC00FCF726FEDE
:1025F000444A034641463046FFF720FB97F8EA106D
:1026000007F1FC00FCF71AFE3E4A034641463046FD
:1026100009B0BDE8F04FFFF78BB8A04639E7A046F8
:1026200057E7059B3B440693002C5BD0059B06981F
:10263000234419460793FDF787FC049B1A789BF8FF
:1026400000309A4206BFB0FA80F84FEA58184FF0AF
:1026500000084B4609F11002F85AE15A0233884249
:1026600018BF4FF000089342F6D188F001012A46C6
:10267000C9B23046FFF72EF9627804EB090105462E
:102680009BF81800FDF782FB02909BF80030019345
:10269000079B00931C4A0AF1010341463046FFF7AD
:1026A000CDFA049B7A78187E079307EB0901FDF7B2
:1026B0006DFB079B049A02901B7801930132069BE5
:1026C00004920AF1010A00930F4A534641463046EC
:1026D000FFF72EF8059B09330BF1010B09F11009E7
:1026E000059307E7A046DCE7A04624E7A04652E7AB
:1026F000A04683E7B9630608CB630608F9630608BA
:102700001164060828640608E06306082DE9F04F06
:1027100089B00F4691460021139A98460646FFF766
:10272000D9F887EA09096FEA0903DFF8849006936C
:102730000446002528460FF04BFC129B184230D06F
:10274000069BDFF870B0034014BF4FF0010A4FF052
:10275000000A049310EA070314BF4A465A46284663
:10276000059307920FF046FC079A039000904346AA
:1027700051463046FFF762FA049BB3FA83F12246D2
:1027800049093046FFF7A6F8059A039B00930446D3
:102790004346002A14BF5A464A4651463046FEF781
:1027A000C7FF0135182DC5D109B0BDE8F08F00BFB6
:1027B000596306083F6406082DE9F04F0A4687B0C2
:1027C00000210646FFF786F83B4C05903B4A2378EC
:1027D000608802EB8303D3F81CA2FBF7E5FF836854
:1027E0000493374BC1681A79002A4BD0DDF810806A
:1027F0000491002721796279049B07FB012213F8D9
:102800000290B8F1000F3FD018F80250059A4D45DC
:1028100014BF0121002130460CBF4FF0010B4FF0D7
:10282000000BFFF757F8013705907DB305F00F0255
:102830002D0940350292CDE90075224A534659468A
:102840003046FFF7FBF9B9F1000F2AD009F00F026B
:102850004FEA1919029209F14002CDE9007253467C
:10286000184A59463046FEF763FFA279012A38BF5D
:102870000122BA42BEDC144B0834A342A6D107B0F1
:10288000BDE8F08F9046B4E74546BFE7B8F1000FCA
:10289000D9D00E4A0097534659463046FFF7CEF935
:1028A000D1E77306E1D4094A0097534659463046AA
:1028B000FEF73EFFD9E700BFB4BE050898BD050886
:1028C000D499002046640608B4BF05085C64060875
:1028D0000FB407B504A951F8040B0191FEF7F2FEFD
:1028E00003B05DF804EB04B070472DE9F0410379C3
:1028F00003F0E002402A53D004D85AB1202A2BD04A
:10290000BDE8F081602A4ED0802AF9D182794179E0
:10291000274813E003F00703052B18D8DFE803F07E
:1029200012171217030AD0F805102248BDE8F0412B
:10293000FEF712BFD0F8052051421F48BDE8F04114
:10294000FEF70ABFB0F80720B0F80510F5E7B0F9B8
:102950000720B0F90510F0E74679184D184805EB47
:10296000C605FEF7C1FE95F8907300240123A74227
:1029700003D8BDE8F041FEF7D7BED5F88C6356F812
:1029800024204FEA84084AB113B90E48FEF7ACFE82
:1029900056F808100C48FFF79BFF00230134E6E7C8
:1029A00041790A48C2E7BDE8F0410948FEF7D4BEC4
:1029B000BF640608706406088664060898BD0508AA
:1029C0009D64060877670608637A0608AE64060801
:1029D000D6640608154B1B6870B533B31448154E02
:1029E000FEF712FFFEF764FEFBF79AF90025FBF7EE
:1029F000CDF9044648B113200BF028F9FEF794FEF8
:102A0000BDE870400C48FEF7FFBE3046FFF760FFA0
:102A1000782D06D80135FEF74BFE64200AF0D0F978
:102A2000E5E7FEF781FE2546F5E770BDE4200020CE
:102A3000EE640608868E0608086506082DE9F04F44
:102A4000784B79491A687948794BB2FBF3F299B01F
:102A5000FFF73EFF774BDFF854C20FCBDCF808409E
:102A60000CAF87E80F00744B0793A608734B0893CD
:102A700016F00206C4F3810418AB18BFDCF804504A
:102A800003EB840318BFC5F3805553F8301C002EA8
:102A900000F0C68018AB03EB850555F8442C684C54
:102AA0006848694E694FDFF80882DFF8CC91FFF77C
:102AB0000FFFB4F8EE274FF47A73B2FBF3F103FB88
:102AC00011220A20B4F9F03792B2B2FBF0F260485A
:102AD000FEF742FE5F4A60496048FFF7F9FEFEF7E5
:102AE00023FE5F4B5F4A997B5F4B604806EB810199
:102AF000D31AD1F85415B4F8E026FEF72DFE5C4841
:102B0000FEF7F2FD94F8F2175A48FFF7E1FE5A4833
:102B1000FEF7EAFD94F8F3175848FFF7D9FEFEF7E1
:102B200003FE5748FEF7E0FD00210A46FB7F0B41FC
:102B300013F0010F01F1010508D012B14846FEF76C
:102B4000D3FD29464046FFF7C3FE0122072D294643
:102B5000ECD14C4D95F86A1505F5EC7305F13C0286
:102B6000012918BF134693F8DC30032B02D04648E6
:102B7000FFF7AEFE454B95F86A15A3F5CE72012915
:102B800018BF134693F8DC30012B02D14048FFF701
:102B90009FFE3E4B95F86A15A3F5CE72012918BF2A
:102BA00013461B695B7B012B02D93A48FFF790FE65
:102BB000394FDFF800A1DFF800B1FEF7B5FDD4F81A
:102BC000F4370393002507F1200957F8041B002967
:102BD00074D0012303FA05F8039B18EA030F1DD0F4
:102BE00018F01F0F1AD01AF8050059F8252052F8CE
:102BF000202035B12948CDE90412FEF775FDDDE945
:102C000004125846FFF764FEB8F1020F06D1244BB8
:102C100093F8211011B12348FFF75AFE0135D4E78C
:102C2000214A3CE7D4200020166506081B650608EB
:102C300040420F00DCC20508386506083D650608FD
:102C4000D49900204265060898BD05086C3700201D
:102C50004A650608F0FF0010000800006B650608D2
:102C60002435002000800008004000088F65060819
:102C7000BE650608D0650608D8650608DA65060848
:102C8000E26506081C0F0010FB650608F410001032
:102C90000366060808660608F4C205087767060892
:102CA000E014001016660608457606080038024053
:102CB000F26506082006002010660608FEF734FDBF
:102CC0007F4B80481A68804B1978137A527A06EB4A
:102CD0008101D1F89015FEF73FFD7C497C48FFF754
:102CE000F7FD7C497C48FFF7F3FDFEF71DFD7B4BAC
:102CF0007B4819684FF47A73B1FBF3F1FFF7E8FDF5
:102D000009A8FDF739FB38B109A910A844F02CFE39
:102D1000744810A9FFF7DCFDFEF706FDD4F8802803
:102D2000002A00F0898007EE902ADFED6F6AB8EE86
:102D3000E77AC6EE877AFDEEE77A17EE903AB4F8B6
:102D4000380F58B107EE900ADFED676AF8EEE77AC0
:102D500086EEA77AFDEEC77A17EE900AD4F80058EF
:102D60005DB107EE905ADFED606AF8EEE77A86EE25
:102D7000A77AFDEEC77A17EE905A5C49B1F85C105D
:102D80006429A8BF6421CDE900055948FEF7E4FC99
:102D900094F83A3F94F83B2FB4F83C1F554806EBA3
:102DA0008303D3F8A435FEF7D7FC534B5348198857
:102DB00089B2FEF7D1FCFAF7A3FF016921B182685D
:102DC0004F48120DFEF7C8FC4E48FEF78DFC4E4BE7
:102DD0001B681B0660D594F8683F032B8CBF4B48DB
:102DE0004B48FEF781FC94F83034022B26D1494839
:102DF000FEF77AFC94F8683F042B44D84648FEF767
:102E000073FC94F8783F002B44D006EBC303D3F84F
:102E1000BC154248FFF75CFDFEF786FC4048414F79
:102E2000FEF762FCD4F8DC460125002C38D1FEF711
:102E30007BFC19B0BDE8F08F134680E702200FF04D
:102E400097F9054608B93848D2E734F0F1FC95F90E
:102E5000041006EB80000131D0F8DC203348FFF786
:102E600037FD94F83334012B04D13148FEF73CFC94
:102E70003048BDE7AB79304806EB8303D3F8DC106C
:102E8000FFF726FDF4E794F832340BB92B48B6E788
:102E90002B48B4E72B49BCE72B48FEF725FCBBE7E2
:102EA00094FAA4F3B3FA83F305FA03F206EB83036F
:102EB0003846D3F8F01524EA0204FFF709FDB4E719
:102EC000283B00201A660608263B00202C660608D0
:102ED0004D6606085B660608616606082C21002020
:102EE000676606088166060800247449E01400102D
:102EF00094660608DA6606085C2700200167060863
:102F0000106706082B670608603500203167060841
:102F10003D6706084D670608029F06089567060884
:102F2000B1670608A1670608536706085D670608CB
:102F30007167060876670608246306087A6706083C
:102F40008A6706080E650608A56706082DE9F04F92
:102F5000DFF8788198F8033099B0002B00F0988062
:102F60005148524EDFF868B1DFF86891DFF868A188
:102F7000FEF74AFC00252F460BA9E8B214F0E8FF43
:102F80009DF83430002B53D0139C54B107EE904A77
:102F90009FED470AF8EE677A80EE270A46F096FA28
:102FA00004460B9A29465846FFF792FC109A002ACD
:102FB00070D002FB04F04FF47A73B0FBF3F3099383
:102FC000DDF848C0BCF1000F66D00CFB04F142F202
:102FD0001073B1FBF3F198F80330082D18BF7F1878
:102FE000002B5BD0179807901598069016980590BF
:102FF0000A2311984FF47A7EB0FBFEFE0998CDF8B3
:1030000010E0B1FBF3FE03FB1E11CDE902E10999CB
:10301000B1FBF3F103FB1100CDE90010BCFBF3F3AE
:1030200021465046FEF798FB0023C6E90D33B362F4
:1030300001351D2D06F140069ED198F8033023B3CB
:103040001C4C1D48D4F8802FD4F87C1FD2084FF4B4
:103050007A73B1FBF3F3D4F8841FFEF77DFB0A22E9
:103060001648B7FBF2F102FB1172FEF775FB144B29
:103070001B78432B06D1D4F8882FD4F88C1F114825
:10308000FEF76AFB0023C4F8843F19B0BDE8F08F57
:103090000D4866E7099293E761469CE7214648465A
:1030A000FEF75AFBC0E700BFC7670608CCA10020A7
:1030B0008096184BD49900206E6806088E68060822
:1030C00094220020B26806082568060824350020EE
:1030D0002F680608716B06083E68060810B586B0B2
:1030E000104B0493104B0393104B0293104B01931E
:1030F000104B1149114A00930446114B1148FFF738
:10310000E7FBFEF711FB10491048FEF725FB3CB129
:103110000F4A1049104806B0BDE81040FEF71CBB2E
:1031200006B010BD1C690608216906082B6906084F
:10313000346906085B660608E6680608DC68060867
:103140002B350020F1680608406906084869060822
:10315000596906086A6906086F6906080120BDE713
:1031600037B52B4D2B48FEF7BFFA95F8CD34002B21
:103170004CD0294C2948FEF747FB94F8F4302BB18A
:1031800094F8F63013B194F8F53073B994ED400A21
:1031900023488DED010AFEF7A7FAB5F8383F9DEDFB
:1031A000010A33BB1F48FEF72FFBB4F8F8101E4886
:1031B000FFF78EFB94F8F43013B31C48FEF724FBA2
:1031C000B4F8FC101A48FFF783FB94F8F630CBB143
:1031D0001648FEF719FBB4F8FA101648FFF778FB0B
:1031E00094F8F53083B1114803B0BDE83040FEF7E4
:1031F0000BBB46F06BF981B20F48FEF7ADFAD4E78E
:103200000E48DBE70D48E4E70C48EDE70C48EBE738
:10321000D49900209C690608E0140010B2690608E1
:10322000B9690608D3690608E2690608026A060851
:10323000126A06082C6A0608DD6906080B6A060889
:1032400066A6060838B50C4B03EBC0050C4695F88E
:103250001C210A4803EB8203D3F81C12FFF738FB4A
:1032600095F8223133B1611C0548BDE83840C9B238
:10327000FFF72EBB38BD00BF98BD0508637A06086E
:10328000996406082DE9F04F6E4B1B7887B0002B30
:1032900000F0D1806C4D6D48A968DFF8F4A1FEF70D
:1032A0005BFA69686A48FEF757FA6A4B6A48D3E9DD
:1032B0000031C91A694BD3F8902FB1FBF2F2FEF737
:1032C0004BFAFEF731FA6648FEF79EFA6548FEF7BC
:1032D0009BFA4FF00008644B1B785FFA88F4A34216
:1032E00022D8624C624FFEF71FFA2646002556F898
:1032F000041B38460135FFF7EBFA162DF7D1FEF720
:1033000013FA5B4E0125234661681B683046C91AD3
:103310000135FFF7DDFA162D04F10404F3D107B0EF
:10332000BDE8F04FFEF700BA524B142603EB8403BE
:1033300006FB045693ED450AB6F80E9046F0C6F823
:1033400096F81EE01EF0010F14BF52222D221EF02F
:10335000020F14BF54232D231EF0040F07EE903AE2
:1033600014BF56232D231EF0080F14BF4FF0430C3B
:103370004FF02D0C81B21EF0800F4FF03C0BB1FBD3
:10338000FBF105914FF0640114BF4FF0530E4FF065
:103390002D0E80B201FB09F1671CCDE902E100931B
:1033A000049017EE903ACDF804C039465046FFF726
:1033B0008FFAB37FDB073AD55C232F4A6343D118DA
:1033C000D05891ED010A70B1DFED2C7AB8EE400AC9
:1033D00020EE270A07EE900AF8EE677A80EE270AB9
:1033E00046F074F800B2642290FBF2F102FB110285
:1033F0002348FFF76DFA142101FB075701FB045422
:10340000F988628A0491218B0391E18A0291A18B50
:103410000191A18A009102F0030319214B4319483D
:10342000218A9208FEF798F908F1010853E7164837
:10343000FEF75AF9DFE7154807B0BDE8F04FFEF791
:10344000E3B900BF04000010200900104C6A060810
:103450005C6A060834060010736A0608D4990020D6
:10346000A06A0608FC6A0608C00D0010CC0900100E
:10347000AC6B0608E01400104006001000401C462B
:10348000756B06088A6B0608816B0608B06B060828
:10349000586B06080EB403B503AA52F8041B019238
:1034A000FCF7E9FB064BD3F8E4261AB90549186D79
:1034B000FBF784FE02B05DF804EB03B0704700BF79
:1034C000D4990020437606082DE9F04798460B79F9
:1034D00003F0E004402C81460F46164631D1684D7A
:1034E000DFF8A081DFF8C091002422E03B7903F0EF
:1034F0000703013B042B04D8DFE803F006080B0E9A
:103500002000315D28460AE03157FBE736F81410F9
:10351000F8E736F91410F5E756F824104046FFF79F
:10352000D7F97B79013BA34202DD4846FEF7DCF880
:1035300001347B79A342D9DCBDE8F08756F824102A
:10354000E0E703F00703052B58D8DFE803F0030C8E
:10355000141619313578602C5ED045D8002C66D011
:10356000202C7CD0E8E796F90050602C54D03BD852
:10357000002CF5D148E03588EDE7B6F90050F4E7C6
:10358000D6F800A0202C554669D02BD8002CD3D1DA
:1035900051463C48FFF79CF9D7F805108A4518D8E2
:1035A000B8F1000FC8D03848BDE8F047FFF790B930
:1035B000202C356853D015D8002CBDD12946304871
:1035C000FFF786F9D7F80510A94202DB4B42AB4260
:1035D000E6DDFEF7A9F83A682C492B464846BDE8D7
:1035E000F04757E7602C17D0802CA5D13178284BB5
:1035F0002848002914BF31461946D5E7202C2DD084
:1036000007D8002C98D12546B7F90540B7F90760CF
:1036100011E0602CE8D100257B7945FA03F3DB0744
:10362000BDE8F0474CBF1C481C48FFF751B9B7F83C
:103630000540B7F8076012482946FFF749F9AC4240
:10364000C7DCAE42C5DBB8F1000F3FF475AF3246C0
:1036500021461348BDE8F047FFF73AB900257A79CB
:10366000104B03EBC20393F890239542B1DAD3F8E1
:103670008C3353F82500BDE8F047FEF735B800BF9E
:103680009A64060883640608CC6B0608D26B0608A9
:103690007E9F0608637A0608EB64060866A606089D
:1036A000C260060898BD0508D86506082DE9F04FE8
:1036B00085B0164601911A46824600213046FEF733
:1036C00009F9324C06F0100305464FF00009029349
:1036D000FDF7EEFF2379019A03F01803934203D01C
:1036E000002A48D1182B46D1284B4FF00D0B0BFB6D
:1036F0000933B3F80900FBF757F880462046FBF77B
:1037000017FCD8E902210746024401442046FBF792
:10371000A7FB80F001012A460390C9B23046FEF7AC
:10372000D9F8DDE90223054602B123BB174A0BFB9A
:1037300009FB52F80BB0B2060FD573B914480393C6
:103740005946FFF7C5F8D8F80820039B3A442146AC
:103750005046FFF7B9FEFDF7E7FF0E485946FFF761
:10376000B7F8D8F80C2000233A4421465046FFF71A
:10377000ABFEFDF7D9FF09F10109B9F5157F04F199
:103780000D04A5D105B0BDE8F08F00BFF4CB05084E
:10379000EC6B0608ED6B060813B50446084601926B
:1037A0000091FBF7FBFBDDE900130246204602B067
:1037B000BDE8104088E60EB403B503AA52F8041B16
:1037C0000192FCF758FA054B0549186DFBF7F6FC1A
:1037D00002B05DF804EB03B0704700BFD49900203D
:1037E000437606080049E6E7F76B060838B50C464D
:1037F000054615492046FCF7A7FB30B9FDF73EFF0B
:103800001248BDE83840FDF7FFBF11492046FCF7DC
:103810009BFBA8B90F4A82F8AE0182F8B60182F884
:10382000520282F85A0282F8F60282F8FE0282F808
:103830009A0382F8A203084A82F821000748E0E7C9
:103840002846BDE83840CDE7066C06080C6C060833
:10385000276C0608D49900206C3700202F6C0608CE
:1038600001490246A7E700BF4B6C0608F8B50646BB
:1038700008460C46FCF7A4FC20210546204646F0ED
:1038800017FC044618B93046BDE8F840E8E7114F88
:10389000114E3B7832789A4201D0FAF773FB0F4B06
:1038A00020461D6044F0FCF8012201462046FAF74C
:1038B00011FB3B7832789A4201D0FAF763FB20463D
:1038C00044F0EEF82A460146BDE8F8400448FDF70A
:1038D00043BF00BFE02000208C2F0020DC20002010
:1038E000626C06082DE9F041064688B008460D4690
:1038F000FCF766FC20210446284646F0D9FB20B997
:10390000304608B0BDE8F041AAE7FCF759FC224672
:10391000054601460F48FDF71FFF85B1202D2A46B9
:10392000694628BF20222046FAF748FBE8460646AB
:103930000027B74208DBAD1B3444002EEDD1FDF764
:10394000F3FE08B0BDE8F08118F8010BFEF76CF942
:103950000137EEE7786C06082DE9F043064687B09C
:1039600008460C4644F09CF8082843D1671E03AD76
:10397000073429463A46A84612F8010FFCF7DEFA4A
:10398000A24201F8010BF7D10023DFF87C908DF8FB
:10399000143017F8010FFCF7D1FAC1B205F8010B8A
:1039A0004846019146F084FB20B10199284646F033
:1039B0007FFB28B13046FFF715FF07B0BDE8F08365
:1039C000A742E6D10F49404629F0D4F90D480E49E7
:1039D000082310F8012B11F8014B18326A44013BFF
:1039E00002F80C4CF5D109488DF8143003A9FDF705
:1039F000B3FEE2E70028E9D0304607B0BDE8F04367
:103A00002EE700BF809E0020A42F0608906C0608B9
:103A100007B5009313460A460249FFF7CCFE03B0F0
:103A20005DF804FB976C060810B504460748FDF7DF
:103A3000EBFEFAF713FE20B1BDE810400448FDF795
:103A4000E3BE20460349BDE81040B4E6B06C06086A
:103A5000BA6C0608C26C06082DE9F04F8FB0044618
:103A600002AA0846AF4946F0DFFA064640B90346C7
:103A70000246AD494120FEF7E7FC0FB0BDE8F08FEC
:103A8000AA49FCF761FA074620BBA64902AA46F0FC
:103A9000CBFAFCF795FB0828054606D9A44908236C
:103AA0003A462046FFF7B4FFE7E7A24C94F8743596
:103AB000834202DC84F87455DFE7064604F274574B
:103AC0003146384631F00AF894F874350136B3427D
:103AD000F6DCEFE798493046FCF736FA0546E0B9E0
:103AE000904902AA46F0A0FAFCF76AFB08280646AD
:103AF00003D9924908232A46D3E78E4C94F87535AA
:103B0000834202DC84F87565B7E728463146013503
:103B10003EF0A4FD082DF8D1F4E789493046FCF7C2
:103B200013FA074600BB7F4902AA46F07DFA002837
:103B3000A3D0FCF745FB0828054603D98149082393
:103B40003A46AEE77B4C94F85E36834209DD014687
:103B500004F2745031F00CF8294604F2745031F03C
:103B600015F884F85E5688E777493046FCF7ECF99B
:103B7000054618BB6F4BDFF8AC9193F85E7606AE46
:103B800001461022304646F07CFAB046BD4202AAF9
:103B900080F20E814946002046F046FA10B96B4982
:103BA0003A460EE1FCF70CFB013528F8020BEDE775
:103BB00096E80F00664C84E80F005EE765493046E2
:103BC000FCF7C2F9054600283BD15A4B0DF1180805
:103BD00093F85E96464607464F45524902AA4FF073
:103BE000000080F2F28046F01FFA014610B95A49EF
:103BF0004A46E6E00322304646F094FAB2464FF0D9
:103C0000000B304643F04CFF584502D801370436CC
:103C1000E2E79AF80000FCF791F90BF1010B0AF8C2
:103C2000010BEEE74D494A46CBE0414620460322D0
:103C300030F03CFF0135043408F10408AF42F4D100
:103C40001BE747493046FCF77FF90546002840F05E
:103C5000AC80384F334997F8748502AA46F0E4F9EE
:103C600000283FF40AAFFCF7ABFA461E01D4B0457A
:103C700003DC3C494346012213E72A4902AA0020FB
:103C800046F0D2F9014600283FF4F7AE4FF00008A5
:103C9000082203A8CDE903888DF8148046F042FA83
:103CA0000DF10C0903A843F0FBFE40451CD81D494B
:103CB00002AA002046F0B8F900283FF4DEAE90F8E2
:103CC00000A097F87595DFF8ACB04FF000084D45AF
:103CD000144902AA4FF000007EDA46F0A5F9024628
:103CE00058B921494A466CE099F80000FCF726F9DA
:103CF00008F1010809F8010BD4E7002D40D1137831
:103D0000303B092B3CD919490192FCF71DF9019A66
:103D100090B310465946FCF717F9019A002838D09D
:103D200013494EE0C9620608489F0020C96C060886
:103D3000CF6C0608D4990020DA6C0608E36C0608FC
:103D4000F16C0608FD6C06080F6D0608FE6D06088E
:103D500034A00020396D06081E6E0608456D060861
:103D6000636D0608686D06083E6E0608A3610608C6
:103D70007B6D0608746D06084FF001084FF0FF35A3
:103D800010460192FCF71CFA0028019A03DA214937
:103D900017E0A846F2E70EAB03EB4503013523F825
:103DA000200C94E71C494A460BE01C49324608E0C7
:103DB0001B49002046F038F900283FF4F9AE1949B4
:103DC0003A462046FFF7F7FC57E646F02DF9002863
:103DD0007FF428AF144C31E746F026F90028E1D1F2
:103DE000124C06EBC6008230082203A9204430F0B2
:103DF0005DFE5046FCF7A2F837446A0087F83E069D
:103E000004EB061006A9023046F0D8F887F856866B
:103E100033E600BFB06D0608C56D0608E86D0608FC
:103E2000C96206081B6D060844A00020489F0020B8
:103E30002DE9F041144B1B6888B00446F3B11A68B1
:103E400004A9D56A18466A46A847064688B1DFF82D
:103E5000448004AC6D46002735F8022B34F8021B71
:103E600040460137FDF778FCBE42F5DC08B0BDE8FE
:103E7000F08106492046FFF79EFCF7E7044908B0A9
:103E8000BDE8F04197E400BF9C3700207D6E060836
:103E9000956E0608636E060813B504460846019140
:103EA00043F0FEFD024670B1102804D10199094883
:103EB00046F024F938B1074B074A0849204602B0BA
:103EC000BDE8104077E40349054802B0BDE8104062
:103ED000FDF742BC596906089C6E0608A76E0608E5
:103EE000D16E060813B504460846019143F0D8FD8B
:103EF0000199024668B1042803D1094846F0FEF84A
:103F000038B1074B074A0849204602B0BDE81040C7
:103F100051E40349054802B0BDE81040FDF71CBC60
:103F20006A690608DF6E0608A76E0608EF6E0608C7
:103F30002DE9F04306469BB008460C4643F0B0FD21
:103F4000002705461C22394602A8019746F099F839
:103F500025B3402D07D0394940232A4630461BB0AF
:103F6000BDE8F04327E40DF1040804F14009022202
:103F70002146684646F0D6F80023102209A9684673
:103F80008DF80270FCF754F8099B0DF10202934280
:103F900021D10234A14508F8010BE8D100213D22CE
:103FA0000AA8099109AC46F06CF8002D39D0244BD1
:103FB0001D78C5B12349202201A846F038F890B1F8
:103FC00020462049FBF730FF1F4A20492346304650
:103FD000FFF7F1FB04E01A781D493046FFF7EBFBD1
:103FE0001BB0BDE8F0831B4E3379D3B9CDB9154A68
:103FF00001AD2B4603CBA342106051601D4602F178
:104000000802F6D1012320460E4986F8943FFBF7BB
:104010000BFF1148FDF752FC10482146FDF79CFBB1
:10402000DEE70C4B93F8943F1BB9054B1B78002B34
:10403000F2D004492046FBF7F7FEEDE7026F0608D1
:10404000C0260020C4260020406F0608A76E060880
:10405000246F0608D49900204A6F0608596F060895
:104060002DE9F74F834608460D4643F019FD3A4FB8
:104070000446D7F80090B8B93848394D394FFDF7A4
:1040800033FB012655F8041B49B106FA04F313EA81
:10409000090F02D03846FEF71BFC0134F2E703B0EB
:1040A000BDE8F04FFDF740BB02462F492846FBF71D
:1040B0006FFF78B92D482A4C2D4DFDF715FB54F8AC
:1040C000041B0029EBD00B78002BF8D02846FEF714
:1040D000FFFBF4E72B782D2B214B03BF013504F1B7
:1040E000FF344FF0010A4FF0000A002653F8048B0A
:1040F000B8F1000F07D11F492A46584603B0BDE862
:10410000F04FFFF758BB2246414628460193FBF784
:104110003FFF019BF0B90123B3409A0505D516482E
:1041200003B0BDE8F04FFDF76FBBBAF1000F0CD044
:1041300029EA030311483B60FDF7D6FA0C484146D3
:1041400003B0BDE8F04FFDF707BB49EA03030C4895
:104150003B60F1E70136C9E7CC3B0020666F0608FB
:10416000F0C30508706F06082A680608746F060811
:10417000A16706087F6F0608906F06089C6F060807
:10418000A56F06082DE9F74F814608460E461746EB
:10419000984643F085FC0446E8B94048404DFEF798
:1041A00097FB20460DF014FF3B68184206D02046CE
:1041B0000DF020FF01462846FEF78AFB0134182C3B
:1041C000EFD13B6813B93748FDF78EFA03B0BDE86D
:1041D000F04FFDF7A9BA024633493046FBF7D8FE47
:1041E0000546A8B93148FDF77FFA2C46304D2046E8
:1041F0000DF0EEFE10EA080F06D020460DF0FAFE94
:1042000001462846FEF764FB0134192CEFD1DDE7A7
:1042100033782D2B48F0807303BF013604F1FF344F
:10422000012500254FF0000A019350460DF0E2FEF3
:104230002246834601463046FBF7AAFE00BB5046A5
:104240000DF0C6FE019B03421AD08DB1BAF1180FD2
:104250001CBF3B6840EA03081648C7F80080FDF71A
:1042600043FA1348594603B0BDE8F04FFDF774BA5E
:10427000BAF1180F1CBF3D6885433D600E48EEE75C
:104280000AF1010ABAF1190FCFD10C49324648465A
:1042900003B0BDE8F04FFFF78EBA00BFAD6F060860
:1042A000A0670608B76F06082A680608746F060834
:1042B000A16706089C6F0608A56F06087F6F0608B1
:1042C000014A40F202235DE73C370020014A6FF0CB
:1042D0007F4357E73437002008B50A4B93F8982FEF
:1042E000032A0AD193F8993F092B06D128F0CAFD79
:1042F000BDE808400448FDF72FBABDE8084003496F
:10430000FFF759BAD4990020BE6F0608C96F060896
:1043100070B5054608461646FBF752FF0C4B1A7857
:104320009042044605D201460A48FDF715FA204698
:1043300070BD2EB1FF2803D10748FDF70DFAF6E74F
:104340000649013A2846FFF736FA4FF0FF34EEE708
:10435000C00D0010D86F0608E96F0608FC6F06084C
:104360002DE9F04F074691B08248834D0E46FDF788
:10437000F3F98249C5F8B8DF002385F8BC3F06226F
:10438000012309783046402485F8BD4F08F086FCAB
:104390000A2008F015FD95F8BC3F0C2BDAB240F26C
:1043A000E4809DF80C50FE2D36D0FF2D0BBF152458
:1043B0000F2401260026944240F0D780611EC9B226
:1043C000684637F097FF04F140030DEB030414F83F
:1043D000413C834240F0C48006F1FF389DF80D3027
:1043E00067485FFA88F8B8F1010F8DBF03F01F0727
:1043F0009DF80E709DF80F4061378CBF5C091D461B
:10440000FDF772F9022E64D0013C042C5FD8DFE87E
:1044100004F005585A5E5C000226CCE75948DFF8E4
:10442000C091DFF8C0B1FDF7EFF95748FDF75CF92F
:104430006C464FF0000A14F8011B48460AF1010AC5
:10444000FEF746FABAF10C0F49D1FDF76DF9022ECD
:104450004FD06422B5FBF2F102FB11524B483B46B0
:10446000D2B2C9B2FDF778F9B8F1010F71D8484A54
:10447000484B9DF810104848484D002914BF11467C
:104480001946FDF769F99DF81110454B454800297B
:1044900014BF19462946FDF75FF9022E59D19DF840
:1044A00012404148FDF720F94CB3FF2C37D00A22C7
:1044B000B4FBF2F102FB11423C48D2B2FDF74CF9D9
:1044C00020E03B48ABE73B48A9E73B48A7E73B4830
:1044D000A5E700238DF83F300DF11F009FE7384B13
:1044E00003FB0AF2B2F1553FA5D85846FDF7FCF898
:1044F000A1E734483A462946FDF72EF9B7E72846A2
:10450000FDF782F99DF813402F48FDF7EDF844B10F
:10451000FF2C21D02D482146FDF71EF904E02C4840
:10452000EEE71E48FDF770F91C4E294FDFF870804A
:104530000DF11305002415F8013F7BB1FF2B0CBFD3
:104540003A464246214623480134FDF705F9042C3A
:10455000F1D111B0BDE8F08F1D48E3E73246F1E735
:104560001D493846FFF727F9F3E71C48FDF74CF9DA
:10457000EFE700BF42700608D4990020C00D00107C
:10458000537006085E700608847006089670060868
:10459000227006082B700608CD70060832700608D7
:1045A000AD790608E4700608EB700608FF7006088F
:1045B000657006086D700608757006080E650608B9
:1045C000ABAAAAAAB2700608077106089A64060880
:1045D000367006081771060822710608327106083F
:1045E000B96106087E9F06082DE9F84FDFF8A8801C
:1045F000DFF88890DFF8A4A007460C46204643F079
:104600004FFA064658B91D4B1D481A781D4B03EB4F
:104610008203D3F8D016BDE8F84FFDF79DB80246E7
:1046200041462046FBF7B4FC60B1DFF864B00025DA
:104630005BF8041BB1B9224638461349BDE8F84F70
:10464000FFF7B9B81148124C124DFDF74DF854F868
:10465000041B19B12846FEF73BF9F8E7BDE8F84F0F
:10466000FDF762B832462046FBF792FC0135002880
:10467000DED189F800505446C0E700BFD93500208C
:104680003B71060898BD05087F6F0608746F060821
:104690006CC40508A16706082A680608457606085E
:1046A00038B50D4604461A4905222846FBF770FC2A
:1046B00068B9184B93F8542022B9012183F854109B
:1046C00083F85520BDE838401348FDF79DB81349DD
:1046D00003222846FBF75CFCA0B90E4D95F8543038
:1046E00063B195F855304BB10D492046FFF763F89B
:1046F000002385F8543085F8553038BD0948FDF75A
:1047000083F8F5E720460849BDE83840FFF753B87D
:104710000B790608D499002045710608567A0608D8
:104720005B71060892710608A6710608F8B5194C67
:1047300094F8543005467BB194F8553063B116496E
:10474000FFF739F828461549FFF735F8002084F8B7
:10475000540084F85500F8BD94F8945FBDB1104B37
:1047600018780028F7D10F4B0F4A03F1200716469F
:1047700018685968144603C40833BB422246F7D16F
:10478000012386F83B3009F051F82846E3E7012081
:10479000E1E700BFD49900205B710608B5710608F7
:1047A000C0260020C42600202C3C002008B5FFF7BE
:1047B000BDFF50B1054B01229A73FCF7CBFD0448B5
:1047C000FDF77CF80020FCF797FF08BD243500209A
:1047D000D37106082DE9F74F064601AA08462E496F
:1047E000DFF8C480DFF8C490DFF8ACA045F01CFC13
:1047F0004FF0000B04465D46012714BBBBF1000FD0
:1048000027D1264C002D43D025482946FCF7A4FF8C
:1048100023790BB903F096FCFAF740FE002384F8E5
:104820005530FCF72BFF15B12846FAF760FB9FB116
:104830003046FFF77BFF78B1FCF78CFD0020FCF7DA
:104840005BFFBBF1000F0AD02046FBF7B9FC85B235
:10485000C5B93046FEF7C6FF03B0BDE8F08F41464C
:104860002046FBF7B9FB80B949462046FBF7B4FB6D
:104870000028EED05F4601AA5146002045F0D4FB47
:104880000446BAE74FF0000BF5E74FF0010BF2E7F3
:104890000448FDF713F8BFE7C9620608D499002061
:1048A000E371060806720608DA71060842790608FE
:1048B0002DE9F04F80468BB008460D4643F0F0F8E6
:1048C000024678B3A5492846FBF762FB044648BB7D
:1048D000FCF72AFFA248A34DA34FA44EDFF8D882CD
:1048E000FCF792FF14203DF0CDFEE11004F007022A
:1048F00001313846FDF7ECFF2B7F6A7F06EB83031F
:10490000D3F81C1252B19A48FCF726FF0134102C40
:1049100005F12405E9D10BB0BDE8F08F4046FCF766
:104920001BFFF3E72846934905AA45F07DFB0546A2
:1049300020B901464120FCF7D8FFECE78E49FBF790
:1049400003FB20B98D494046FEF735FFE3E78C4E67
:104950000827002431682846FBF7F6FA002808BF2C
:104960003446013F06F11006F4D154B98549284672
:10497000FBF7EAFA28B184492A464046FEF71BFFB6
:10498000C9E700207B498DF8130005AA45F04CFBD0
:104990000646002C3AD080B1FBF712FC451E09D424
:1049A000A37A9D4206DAE2684AB1012303FA00F0D5
:1049B000104204D175493246DFE7754EFAE7E088C8
:1049C000F9F7F2FE7349D0E902320979002908BFEC
:1049D0001A46217A637A05FB0133002712F903A0F6
:1049E000039702EB030B634905AA002045F01CFB6B
:1049F0008146A0BB6849012344B39BF900202046AF
:104A0000CDE900312946FAF74DFC84E768B10DF194
:104A10001301FBF7AEFB28B19DF81350284604F0B4
:104A20003DF920B95D493246A7E7594EFAE72846D5
:104A3000F6F78AF88246284608F054FD0390284687
:104A400008F08EFDA34607462546CCE7CDE90031A8
:104A50009DF8130052463946FAF770FC5BE7464969
:104A6000FBF772FA064658BBACB14D4FEDB2207958
:104A700072B22946F6F73CF800283FF44CAF0288A2
:104A8000037800933146C2F303233846120BFCF738
:104A900063FE0136EBE7424C7979386872B2F6F77B
:104AA0006FF800283FF437AF02880378009331464F
:104AB000C2F303232046120BFCF74EFE0136EBE750
:104AC00038494846FBF740FA10B34846FBF778FBF5
:104AD000064642B26CB12079E9B2F6F709F8C8B9D6
:104AE000CDF80090226830496B1C4046FEF763FE0B
:104AF00011E779793868F6F743F858B99DF813301B
:104B00002A49CDF800901A09403203F00F03ECE770
:104B10004FF0FF3606AF39463046FBF799F908A942
:104B20005046FBF795F9564548D076B24CB18BF814
:104B30000060009721681E4808AB6A1CFCF70CFE59
:104B4000E9E69DF81320039B1A489E70110900970F
:104B500008AB02F00F024031F0E700BF1C720608FC
:104B600021720608D00200203772060898BD050899
:104B7000AA730608C96206082A6806084872060869
:104B8000A00500205C720608607206086F720608B5
:104B900045760608D4990020311701087F7206086F
:104BA00091720608B96F0608B2720608D572060837
:104BB000FD72060820730608A167060834B1216853
:104BC000074808AB6A1CFCF7C7FDA4E69DF8132054
:104BD0000448110908AB02F00F024031F3E700BFAF
:104BE00048730608637306082DE9F04F80468DB0C0
:104BF00008460D4642F054FF024630B901460120F6
:104C00000DB0BDE8F04FFCF779BF0390B0492846DE
:104C1000FBF7BEF9039A30B9AE4940460DB0BDE886
:104C2000F04FFEF7C8BDAC492846FBF7B1F9044682
:104C300000285BD1FCF778FDA848A94FDFF8E0B267
:104C4000DFF8E082FCF7E0FD17203DF01BFD17F9CF
:104C5000015B002D3CD029465846FDF739FEDFF8B0
:104C60009C92DFF88CA200231A46910089B2284654
:104C70000593049208F0ACFC039008F037FD049A09
:104C80000178059B561CC9B11BB90490FCF74CFD7B
:104C90000498039B41789A79037802F0020208EBAA
:104CA0008303C1B10091D3F81C328E48002A14BF8F
:104CB0004A4652463146FCF74FFD0123042E324648
:104CC000D3D113B98848FCF79FFD01340E2CBED117
:104CD0000DB0BDE8F08FD3F81C328448002A14BF11
:104CE0004A4652463146FCF737FDE6E70024804944
:104CF0008DF81B4007AA284645F096F918B940469A
:104D0000FEF770FDE4E70DF11B01FBF732FA0546F3
:104D10000028F4D09DF81B60304603F0BFFF20B997
:104D200074494046FEF747FDD2E7DFF8FC91234681
:104D30004FF0FF3403EB430212F8092096420BD0E8
:104D4000611C02D1002A08BF1C460133152BF1D18A
:104D5000631C15D16849E4E71C46654907AA002091
:104D600045F062F90646002800F09E805849FBF79E
:104D7000EBF828BB614E624FDFF8B081044615E0C6
:104D80000025EAE7E97928680391F6F7B5F80246C5
:104D9000A8796B79039910F0020F14BF304638469A
:104DA0009B08009001334046FCF7D6FC01349DF887
:104DB0001B00214608F0AAFB05460028E2D187E740
:104DC000504902223046FBF7E3F80746002849D154
:104DD000B01CFBF7F5F99DF81BB00346BA46013746
:104DE00039465846039308F091FB039B38B94FEAC4
:104DF0001B12454900960BF00F0340323FE0C27989
:104E00009A42EBD1002D40D14FF0FF36BAF1FF3F6F
:104E10009DF81B5008BF002504EB440409EB040374
:104E20000AF101025A7009F80450FF220AAC9A7084
:104E30009DF81B0022465146FBF71AF808AA314696
:104E40009DF81B00FBF714F89DF81B20B2454FEAB4
:104E5000121120D12D4808AB02F00F024031FCF7AF
:104E60007BFC35E72A493046FBF76EF850B39DF8D6
:104E70001B30284900961A09403203F00F034046C0
:104E8000FEF799FC24E74FF0FF3A04EB44034B4450
:104E90005E78013EBAE72048009408AB02F00F02AA
:104EA0004031FCF759FC13E704EB44041B4B00931F
:104EB000A144024699F801109DF81B000123FAF75E
:104EC00081FA05E7002DDED14FF0FF36B246A3E7A9
:104ED0002A680608487206081C7206087F730608CE
:104EE000881C06089F730608C0730608B17306087D
:104EF000C9620608C6730608DD730608EC64060876
:104F00004576060806740608737406082F740608AA
:104F1000B96F0608097406084D74060831170108B0
:104F20009873060898BD0508EC260020F173060862
:104F30002DE9F04F2DED028B85B0064603AA0846F9
:104F4000924945F071F8074640B901464120FDF706
:104F500033FC05B0BDEC028BBDE8F08F8C49DFF867
:104F60006482FAF7F1FF044600283CD189488A4D53
:104F70008A4FDFF85492FCF747FC14203DF082FB87
:104F80002968AB79AA8801F13F4108EB830301F559
:104F90007E01B2FA82F2890A4131D3F81C32C2F1A1
:104FA0001F023846FDF794FCE97911B14846FDF738
:104FB0008FFC0134FCF7B8FB602C05F10805DFD14C
:104FC000724903AA002045F02FF87549FAF7BCFF93
:104FD0000028BED130466E49FFF706FE6C493046C8
:104FE000FFF766FCB5E7002508F58E7919F835302E
:104FF00008EB8303D3F81C120191084642F050FDE0
:10500000019902463846FAF7C3FF40B10135202D19
:10501000ECD164493A463046FEF7CDFB99E75B494F
:1050200003AA45F001F808EBC5080746FBF7C8F8E6
:1050300098F8223104464FEAC50A2BBB002825DC2C
:105040003B78002B00F09E80D144B9F80200F9F7BC
:10505000ABFBE3B2019399F8058099F80430019A0B
:10506000846802FB038804EB08013846FBF781F8EB
:10507000002800F0878014F808A0BAF1000F1CD1B6
:105080004948FCF7C1FB64E7002805DD012B1A46FF
:1050900038BF0122A24208DA012B444938BF01235C
:1050A00001223046FEF7B4FC53E7384903AA00203A
:1050B00044F0BAFF013C0746C2E7504603F0EEFD5C
:1050C000814600285ED04FEA1A13403308EE103AAA
:1050D0000AF00F03DFF8F48008EE903A002700266C
:1050E000B8F80200F9F760FB98F8042098F805304A
:1050F00006FB02338268D15C514523D1BD4204D105
:1051000001998E421ED00021D15418EE902A18EE3B
:10511000101A27485FFA86FBFCB2FDF7D9FB594607
:105120002046FEF78FF8BD4209D12248FDF7D0FB9B
:1051300020465946FEF786F81F48FDF7C9FB1F4871
:10514000FCF762FB98F80630012B06F1010638BF28
:1051500001239E42C4DB0137202F08F10808BED18D
:10516000D9F80010B9F80420154801F13F4101F5C4
:105170007E01B2FA82F2890AC2F11F024131FCF7C4
:10518000EBFAE6E63046FEF72DFBE2E6C9620608DA
:105190001C7206089F740608B4230020DD740608FC
:1051A000E8740608EC7406080E750608087506080B
:1051B000207506080565060844750608868E0608EB
:1051C0004E75060898BD050899640608B4BE050822
:1051D00020B10078B0FA80F0400970470120704794
:1051E0002DE9F34106460846FFF7F2FF0D46074654
:1051F00070B1002401A920463DF0F6FA01340146C1
:105200003046FFF7EDFF122CF4D102B0BDE8F0817B
:105210000846FAF7D5FFC4B2112C72D8681CF9F70A
:10522000DFFF3C4D8046E8B93B4B03EB440393F86A
:10523000C01F8A1E51425141374B03EB440393F880
:10524000C02FAA5C002955D093F8C13F192040F225
:10525000EE2100FB03133148214602B0BDE8F041C6
:10526000FCF77ABA0178284644F022FF70B1032C8B
:1052700094BF002201222A4902EB4202431B0A4446
:1052800052FA83F393F84077032F05D1304602B0EA
:10529000BDE8F041FEF7A6BA4046F9F7A1FF08B312
:1052A000022FF3D1FAF78CFF40F6CA0280B2904287
:1052B000194BA8BF104640F2EE22904203EB440384
:1052C000B8BF1046A0F2EE201922B0FBF2F083F82E
:1052D000C10FBB1E594259410F4B03EB440383F8E6
:1052E000C07FA9E7022FF4D1304602B0BDE8F041FB
:1052F000FEF7B6BA0B48214602B0BDE8F041FCF714
:105300002BBA094911233A46304602B0BDE8F041B4
:10531000FEF77EBBA0310608D49900206A75060806
:1053200098BD05087A750608877506082DE9F041CD
:10533000064686B00846FFF74BFF0F46054640B1CC
:1053400000235D491A46012006B0BDE8F041FCF794
:105350008DBC0846FAF734FF1328044600F3A380F7
:1053600006264643781C8DF81750F9F739FF534D40
:10537000074670B1FAF724FFC0B212F087FB40B1C4
:10538000AB19027983F8F0249DF8173001338DF8BA
:1053900017303846F9F724FF074668B1FAF710FFCF
:1053A0000D2809D8062303FB045383F8F1049DF864
:1053B000173001338DF81730DFF8FC80B11C0DF188
:1053C000170241443846FAF7FFFEF9F709FF07468E
:1053D00068B1FAF7F5FE012809D8062303FB045348
:1053E00083F8F4049DF8173001338DF817303846F0
:1053F000F9F7F6FE80B1FAF7E3FEC0B212F046FB11
:1054000050B1062303FB0453027983F8F5249DF879
:10541000173001338DF817309DF81720042A4FF00C
:1054200006032FD103FB04530022A3F8F4241DF03C
:1054300049F8062303FB04554FF4617695F8F00410
:1054400012F00EFB95F8F32495F8F27419238046B8
:1054500095F8F50413FB076713FB026612F000FBD7
:10546000437998F80520039395F8F4340097CDE933
:105470000163134895F8F1342146FCF76DF906B045
:10548000BDE8F081052A05D103FB0453002283F80F
:10549000F524CCE7062A1FBF08EB0602002348F8D4
:1054A00006309380C3E7074913232A46304606B0E7
:1054B000BDE8F041FEF7ACBAC49E0020D4990020AC
:1054C000F2620608087506082DE9F04380468BB0A5
:1054D0000846FFF77DFE40B100234D491A460120E2
:1054E0000BB0BDE8F043FCF745BCCDE907000990DF
:1054F00008464D1CFAF764FE44B220460CF0BCFD91
:105500000646002843D08DF8204001242846F9F7AC
:1055100067FE054638B100230A221946FAF788FDCE
:1055200001340790E4B2DFF8F09000272846F9F73D
:1055300057FE054618B3FAF743FE3649002251F8E4
:1055400004CB6045D3B203D00132102AF7D1002337
:1055500009EB8302D2F8DC20904210D1022F1DD03B
:10556000032F20D05A1E012FD2B212D00B2A03D8FB
:105570008DF821300134E4B20137042FD6D1052C47
:1055800017D840460BB0BDE8F043FEF769B90446B2
:10559000BCE7042AF0D88DF82230EBE7052BEBD8D6
:1055A0008DF82430E6E79A1E0D2AE5D88DF82330D1
:1055B000E0E707AB03CB9DF8232030601868164B5B
:1055C000716003EB8202B060D2F8DC2004929DF897
:1055D000242003EB82020021D2F8DC2003929DF804
:1055E000222003EB82020846D2F8DC2002929DF8CA
:1055F000212003EB8203094AD3F8DC300193079B97
:1056000000939DF92030FCF793F80BB0BDE8F083D0
:10561000909D002074BE050898BD05080B63060820
:105620002DE9F04F024691B00846FFF7D1FD0B4639
:10563000044628B1104611B0BDE8F04FFEF710B98E
:105640004FF0FF32CDE90820A64ADFF8E082D26CA5
:10565000DFF8DC9292F83810DFF8D8A2CDE90C1010
:10566000CDE90E02CDE90A009F4907AA184644F089
:10567000DBFC27460546049426464DB9089A0C9F44
:10568000BA4262D19948FCF767F811B0BDE8F08FD3
:10569000062F12D8DFE807F0041E2328454C5100DE
:1056A00051462846FAF798FC78B14FF480600CF028
:1056B0005FFD90F90430089301248B4907AA00206C
:1056C00044F0B2FC01370546D7E72846FAF778FDE3
:1056D0000890F2E72846FAF773FD0990EDE72846AF
:1056E000FAF791FC0A90E8E7284642F0D9F94146DA
:1056F000024605902846FAF74BFC18B3059A49462E
:105700002846FAF745FC06460028D6D02846FAF780
:1057100057FD04280646D0D901467548FCF71CF809
:10572000B3E72846FAF74CFD00230C900F93C4E72B
:105730002846FAF745FD0D90BFE72846FAF763FCC7
:105740000E90BAE701230493B7E7DFF8EC8151B27A
:10575000434613F9010B884208D00135092DF8D1D1
:10576000002164480131FBF7F7FF8EE76248012111
:10577000FBF7F2FF7AB2002318F9011B8A4200F00E
:105780000C810133092BF7D13A460121E9E7A7F152
:10579000140253425341059308AD002303F101085D
:1057A000EB68A3BB95F900B058460CF0A9FCD5F8FE
:1057B00004A020B1D0F80090B9F1000F5ED1BAF189
:1057C000000F19D14FF461436B604FF0010AAB68D1
:1057D0000BB90323AB600023D5F8049002932A7A17
:1057E0001946CDE9009258461A4610F061FFE8606C
:1057F00028B94248414691E74FF0000AE7E74A4698
:105800004146BAF1000F37D03D48FDF761F8B8F1D5
:10581000020F05F110054FF00103BFD1059BDDF824
:105820003C800B9D53B13748FBF7EEFFD8F80030B2
:105830001B6A1BB134492A4640469847049B002BFB
:105840004ED03249324B142F18BF19463148FBF75E
:1058500083FF142F09D1049B03B936B12B68DB6990
:105860001BB12D49324628469847002C66D10022AC
:10587000414628463CF06CFF2848C6E7C5F80C9026
:10588000BAF1000F25D0264841465246FDF720F8D0
:105890005146484601F076FDD5F808A0BAF1000F50
:1058A0000FD099F8042092450BD01E48534641462C
:1058B000FDF70EF8D9F800305FFA8AF19B69484687
:1058C0009847D9F82C30002BA1D00023C9F82C30F0
:1058D0009DE7D9F8082014484146FCF7F9FFDBE7BB
:1058E0000B49B3E7D4990020C9620608C5750608BC
:1058F000AD75060809770608DE750608EA7506081C
:1059000006760608BD760608857301088F750608B9
:1059100045760608E6760608FBF100082A760608B2
:10592000467606089876060873760608A775060870
:10593000B96F06089C75060850B5050803F078FA9B
:10594000052007F03DFA1A4FDFF86C9000264FF063
:10595000030A99F80030B34289D917F801BBBBF1AB
:10596000000F15D0584607F0FBFD044680B158469D
:1059700003F094F908B1A0F806A001210490F5F70E
:1059800019FBA379049813F0010F03D0F4F708FD75
:105990000136DEE7F4F7FEFCFAE706483A46022154
:1059A000FBF7DAFE099B002B3FF4F1AE0023F2E691
:1059B00090270020DE750608C00D00102DE9F04389
:1059C00080468BB00846FFF703FC0F46044640B103
:1059D000002365491A4601200BB0BDE8F043FCF7EF
:1059E00051BA0846FAF7ECFB1D28054600F3B380D0
:1059F0000A264643781C8DF82740F9F7F1FB044648
:105A000030B1FAF7DDFB9DF8273001338DF82730F0
:105A10002046F9F7E5FB554C074668B1FAF7D0FB8D
:105A20000D2809D80A2303FB054383F8E40F9DF8EA
:105A3000273001338DF82730DFF82C91711C0DF1E0
:105A4000270249443846FAF7BFFBF9F7C9FB074676
:105A500068B1FAF7B5FB222809D80A2303FB0543EE
:105A600083F8E70F9DF8273001338DF8273038464B
:105A7000F9F7B6FB074668B1FAF7A2FB0D2809D87B
:105A80000A2303FB054383F8E80F9DF82730013311
:105A90008DF827309DF82730062B0CD009EB060235
:105AA000002349F80630404653601381FDF7D8FEC5
:105AB0000BB0BDE8F0830A2606FB054600233846F6
:105AC000A6F8EA3FA6F8EC3FF9F78AFB074640B193
:105AD000FAF776FB9DF82730A6F8EA0F01338DF828
:105AE00027303846F9F77CFB58B1FAF769FB0A23EF
:105AF00003FB0543A3F8EC0F9DF8273001338DF825
:105B000027301B4B4FF0FF325A600A2202FB05423E
:105B10004FF46170B2F8EC3F0693B2F8EA3F059398
:105B200092F8E83F049392F8E73F039392F8E61F58
:105B3000192313FB0101029192F8E51F13FB0103E6
:105B4000019392F8E43F009300210A4A2B4608464D
:105B5000FBF7EEFDACE708491D23224640460BB09B
:105B6000BDE8F043FDF754BFB8A90020D499002048
:105B70009405002028630608087506082DE9F74FEC
:105B8000DFF89C91DFF89C8105460F463846FFF709
:105B90001FFB064640B100235A491A46012003B0B4
:105BA000BDE8F04FFCF7D6B9052249463846FAF76A
:105BB000EFF960B9534B00221A601A611A621A6336
:105BC0001A641A651A661A6703B0BDE8F08F4E4969
:105BD00004223846FAF7DCF904463846002C44D152
:105BE000F9F7FEFA83460028EED041F059FF474B03
:105BF000C2B253F804ABBAF1000F07D144493A4698
:105C0000284603B0BDE8F04FFDF7D5BD51465846D4
:105C1000CDE90023FAF7BCF90134DDE9002306469B
:105C20000028E6D1374A0346174600210133082BE6
:105C300042F8101BFAD108EBC403D3F804C0BCF13E
:105C4000000F03D018F834E0764505DB3148324FB9
:105C50005146FBF781FD99E70CEB06130FCB07EBE1
:105C6000061484E80F000136EEE7FAF7A9FA0728D0
:105C700004463DD83846F9F7B3FA064658B3F9F763
:105C800027F8204B03EB041383ED000A012730466D
:105C9000F9F7A6FA064638B1F9F71AF8194B03EBEB
:105CA000041383ED010A01373046F9F799FA0646E5
:105CB00038B1F9F70DF8134B03EB041383ED020A27
:105CC00001373046F9F78CFA38B9284603B0BDE8F9
:105CD000F04FFDF7C5BD0746D9E7F8F7F9FF0948CA
:105CE000032F00EB041484ED030A3FF454AFECE7F8
:105CF0000A4907233246284603B0BDE8F04FFDF7B6
:105D000087BE00BFE03500201B7706086CC405087D
:105D10007F6F06082077060845760608087506088E
:105D2000A77506085CB505082DE9F3410546084648
:105D3000FFF74EFA0C46074640B1002333491A4696
:105D4000012002B0BDE8F041FCF7A2B9304920467D
:105D5000FAF7FAF8034670B92C4A4FF47A704FF408
:105D6000FA610133042B1080518002F10402F8D152
:105D700002B0BDE8F0812046FAF722FA0328064671
:105D80003FD82046F9F72CFA074670B1FAF718FA0F
:105D90004FF0010804463846F9F722FA48B9284678
:105DA00002B0BDE8F041FDF75BBD40F2EE24804655
:105DB000F1E7FAF705FAB8F1000FF0D0A4F2EE22FD
:105DC00040F2DC539A4203D8A0F2EE229A420AD95A
:105DD000104940F6CA0340F2EE22284602B0BDE860
:105DE000F041FDF715BE0C4B0C4A03EB8603002176
:105DF0001C835883CDE9004033460846FBF798FCE6
:105E0000B6E7074903233A46E7E700BFE4AA0020C4
:105E1000A77506082A770608CCAA00205F63060843
:105E200087750608F0B5074689B00846FFF7D0F930
:105E30000E46054640B100231A491A46012009B012
:105E4000BDE8F040FCF768B90846FAF7B9F91F2831
:105E500004461DD83046F9F7C3F90146204631F013
:105E600075FE78B10F4803AE314600EB84003CF07C
:105E70001DFC0D4A0096234629462846FBF758FC90
:105E800009B0F0BD384609B0BDE8F040FDF7AABC46
:105E900006491F232A46384609B0BDE8F040FDF701
:105EA000B7BD00BFF4AA0020706306080875060895
:105EB000F0B5074685B00846FFF78AF90E46054655
:105EC00040B100231C491A46012005B0BDE8F0404E
:105ED000FCF76CB90846FAF773F90F28044622DC80
:105EE0003046F9F77DF90146204631F0ADFDA0B10D
:105EF000124B04F1200203EB8203294693F82B2076
:105F0000029293F82A2001921B8D00930C4A23469B
:105F10002846FBF70DFC05B0F0BD384605B0BDE8DE
:105F2000F040FDF75FBC07490F232A46384605B00D
:105F3000BDE8F040FDF76CBD74AB0020CCAA00209A
:105F40007A63060808750608F0B5054687B0084666
:105F5000FFF73EF90B46044640B100231C491A46A0
:105F6000012007B0BDE8F040FCF768B91949194FA6
:105F700002AA184644F058F803AEB8B1032C04D175
:105F80002846FDF76DFC07B0F0BDFAF719F902AA33
:105F900046F8040B39460020013444F045F8ECE79C
:105FA0000D4832462146FBF7D7FBECE7032CE7D13F
:105FB000DDE90346059B01931A463146E0B231F014
:105FC00087FD019B0028EBD12846FDF70BFCDAE7A3
:105FD000F4AA0020C96206088C6306082DE9F04F78
:105FE000074689B00846FFF7F3F88B46054640B1EF
:105FF00000234D491A46012009B0BDE8F04FFCF7D7
:10600000C3B94A4B084693F874A593F8759593F86D
:106010005E86FAF7D5F8092804467BDC0626464357
:106020000BF101008DF81F50F9F7DAF83E4D834669
:1060300048B1FAF7C5F80D289FBF9DF81F30A85545
:1060400001338DF81F305846F9F7CAF8834660B11E
:10605000FAF7B6F8824508D3062303FB04535870B9
:106060009DF81F3001338DF81F305846F9F7B8F806
:10607000824660B1FAF7A4F8484508D8062303FB26
:10608000045398709DF81F3001338DF81F3050462F
:10609000F9F7A6F8814660B1FAF792F8804508D37F
:1060A000062303FB0453D8709DF81F3001338DF88D
:1060B0001F30311D0DF11F0229444846FAF784F8BC
:1060C0009DF81F30062B09D0AA190023AB51384682
:1060D0009380FDF7C5FB09B0BDE8F08F6343EA1874
:1060E0004FF461765079192111FB00600590107909
:1060F00011FB00610491D17803919178029152785B
:106100000192EB5C00930021094A23460846FBF705
:106110000FFBE0E7074909232A46384609B0BDE8E6
:10612000F04FFDF775BC00BFB4370020D4990020B4
:10613000A06306080875060810B5044608460B4615
:10614000FFF746F828B9094903221846F9F720FF56
:1061500028B90748FBF7B2FB0120FBF7CDFA204630
:106160000449BDE81040FDF726BB00BF387706089C
:106170003C770608A67106082DE9F74F0546084644
:10618000FFF726F80B46044618B9334A92F81871FF
:106190002FB9284603B0BDE8F04FFDF723BB2F49C8
:1061A000DFF8C480DFF8C490DFF8C4A001AA184665
:1061B00043F03AFF264610B902F048FE08E056B90F
:1061C000012201462846FEF7A3F8421C04461AD1D4
:1061D00003B0BDE8F08FF9F7F3FF2F28834634D8DA
:1061E0000FB102F025FEBBF1060F13D01C490123AD
:1061F00009785FFA8BF2E0B206F050FD5946484646
:10620000FBF7AAFA0027154901AA0020013643F03E
:106210000BFFD0E7DAF800301B0112D5FF2C0ED0AF
:10622000E1B22846FEF79CF8E8E72846FEF798F822
:1062300001370B4B1A78F9B28A42F6D8DEE700270D
:10624000F7E70848FBF7E0FAD8E72F22414628464F
:10625000FDF7B1FAD7E700BFCCAA0020C962060853
:10626000C00D0010C96F06086F7706085E77060834
:10627000603500202DE9F04F064685B00846FEF750
:10628000A7FF0B46044628B1304605B0BDE8F04FE5
:10629000FDF7E6BA3049DFF8D090DFF8D0A0DFF89C
:1062A000D0B003AA184643F0BFFE27460546A046D5
:1062B0005DB92A4B3A46D86CA1B23BF0DFFF68BB10
:1062C00027493046FDF777FA28E0B8F1000F06D0ED
:1062D000B8F1010F25D03046FDF7C2FA1EE028467E
:1062E00041F0DEFB4946024601902846F9F750FE90
:1062F00050B3019A51462846F9F74AFE30B3019A45
:1063000059462846F9F744FE10B3019A1549284624
:10631000F9F73EFEF0B13046FDF764FA05B0BDE88E
:10632000F08FBB1E5A425A4129463046FDF7F0FF16
:10633000421C0446F2D0084903AA002043F074FE30
:1063400008F101080546B3E74746F4E70127F2E7FD
:106350000227F0E70327EEE7C9620608D499002078
:106360009B770608987706088F77060892770608C5
:10637000957706082DE9F74380460846FEF728FF83
:106380000B46054628B14046FDF76AFA03B0BDE862
:10639000F0832E49DFF8B49001AA184643F044FE7A
:1063A0002F4604462E467CB9022DECD1A7F57A7310
:1063B000B3F57A7F21D926494FF4FA634FF47A7204
:1063C0004046FDF725FBE1E74DB1012D10D001AAB4
:1063D0004946002043F028FE01350446E3E7012248
:1063E00021464046FDF794FF431C0646EFD1CDE71A
:1063F0002046F9F7E5FE0746E9E7164B1B68B8B2F9
:106400005B689847FF2EBCEEC00A0CD1124BF8EE29
:10641000407A1A78114BA24213DC10EE101A104881
:10642000FBF79AF9B2E70F4B0F48F8EE407A03EB0F
:10643000860310EE102AC3ED477A3146FBF78CF93C
:10644000A4E7E3EC017A0134E5E700BFC96206087E
:10645000A9780608DC140010C00D0010E8AB00207D
:10646000C6770608CCAA0020B9770608F8B5074613
:106470000846FEF7ADFED0B1204BD3F8946001364C
:1064800030460BF0B7FD34460546F0B90134192CFF
:10649000A8BF002420460BF0ADFD0546A8B9B442C4
:1064A000F4D138461649BDE8F840FDF784B90846EE
:1064B000F9F786FE04460BF09DFD054628B92146F6
:1064C0001048BDE8F840FBF747B90C4BC3F89440BF
:1064D00008F054F80C4821462A46FBF73DF9182CE1
:1064E0009DBF0A480C2101FB04000020BDE8F840D4
:1064F00098BF90F8480707F0A9BB00BF940500209B
:10650000D5770608E9770608FF77060898BD0508DD
:1065100038B5124D04460846FEF75AFE60B1104BDE
:10652000104893F900104B1C0ABF0F4BC9B21978E1
:10653000BDE83840FBF710B90846F9F741FE0328DB
:1065400004D8C0B2FAF720FD2946E4E720460749FF
:10655000BDE838400322FDF72EB900BF4576060896
:1065600094050020187806082435002028780608AD
:10657000F0B5032985B005460C46164614D80B4FD6
:106580003970FBF7D1F80A492846FFF7C1FF0949DE
:10659000224601A8F9F79EFB01AB324608212846A6
:1065A000FDF784F8FF233B7005B0F0BD9405002093
:1065B000457606081878060838B5124D0446084690
:1065C000FEF706FE60B1104B104893F901104B1C0A
:1065D0000ABF0F4BC9B25978BDE83840FBF7BCB8C9
:1065E0000846F9F7EDFD032804D8C0B212F02AFEE0
:1065F0002946E4E720460749BDE838400322FDF775
:10660000DAB800BF4576060894050020147806081D
:106610002435002023780608F0B5032985B0054607
:106620000C46164614D80B4F7970FBF77DF80A49D3
:106630002846FFF7C1FF094922466846F9F74AFB99
:106640006B46324610212846FDF730F8FF237B7059
:1066500005B0F0BD940500204576060814780608BC
:106660002DE9F74F434BDFF828A11A785B788AF8B9
:106670000130414B8AF800201B79054688460BB94A
:1066800001F060FDF8F70AFF00263C4CB1460D23EF
:106690003A4A7343414652F803B05846F9F79CFC16
:1066A000002841D0B9F1000F01D0FBF73DF8344884
:1066B0005946FCF70DF9002221462846FDF76CF8F3
:1066C000FBF732F8237903F01803082B45D0102B81
:1066D00048D02046FCF709F9284A0D2303FB06237E
:1066E000B3F80900F8F760F80746D8B12046F8F784
:1066F0001FFCD7E902210090024401442046F8F72C
:10670000AFFB78B9019059461E48FCF7E1F8019AB1
:10671000B9681346009A28460A442146FCF7D4FE7D
:10672000FBF702F809F101090136B6F5157F04F10E
:106730000D04ACD10020F8F7DAFBFF238AF8003013
:106740008AF80130B9F1000F11D10F4942462846AD
:1067500003B0BDE8F04FFDF72EB80C492846FFF70F
:10676000D7FEB6E709492846FFF726FFB1E703B091
:10677000BDE8F08F24350020D4990020F4CB050823
:10678000F16B0608437806087F6F06084576060811
:10679000940500202DE9F74F074608460E4641F0C4
:1067A0007FF9044620B1012825D133782A2B22D144
:1067B000B248B34EDFF8E482FBF726F80025B14675
:1067C0004FF00D0A0AFB05F3404659F80310FCF799
:1067D0007FF8221E18BF0122314638460135FCF7EA
:1067E000DBFFFAF7A1FFB5F5157F06F10D06E9D13C
:1067F00003B0BDE8F08F3D21304643F059FC00283E
:1068000000F0368103461A4613F8011D2029FAD0FC
:10681000921B431C994613F8011B2029FAD0DFF87C
:1068200060B25FFA82FA4FF000080D2303FB08F311
:1068300052465BF80310009130460BEB0304F9F766
:10684000A7FB0546002857D10099084641F028F9D2
:10685000824551D1267906F0E001402900F0CB8035
:106860000ED8002955D0202900F09D803846854952
:10687000FCF7A1FF204603B0BDE8F04FFCF735B8A8
:10688000602900F091808029F0D1484641F008F954
:10689000E379A679DB0705460CD52046F8F77EFBA1
:1068A0000378014633B12A46484643F027FC0028C6
:1068B00040F0D880002D00F0D580AE42C0F0D280EC
:1068C0000D2303FB08B3204693F805A0F8F766FBF9
:1068D0003246002143F0D5FBAA452BD86A492A4607
:1068E000484643F00BFC28B32046F8F757FB2A46EE
:1068F000494643F063FB1DE008F10108B8F5157F38
:1069000093D162493246384603B0BDE8F04FFCF7F8
:1069100052BF06F00703042B1CD10B460A2248463F
:10692000F9F786FBD4F80530834201469ED3204612
:10693000F8F748FB0D2303FB08F855485BF80810EF
:10694000FBF7C6FF00222146384603B0BDE8F04FF2
:10695000FCF722BF052B0FD101230A224846F9F785
:1069600067FBD4F8053083420146FFF67FAF5B42F8
:1069700083423FF77BAFDAE74846F9F721FCB4F8EA
:106980000550B4F8071016F0050FAAB218BF2AB2C6
:106990008BB218BF0BB29042FFF668AF98423FF738
:1069A00065AF0146C3E765793A4A02EBC5050026A3
:1069B00095F890230092B2463346009AB24202D92B
:1069C000BAF1000F03D0002B3FF450AFB2E7D5F877
:1069D0008C1351F8260060B149460193F9F7B4FAD7
:1069E000019B30B9314620464FF0010AF8F7EAFA28
:1069F00053460136E1E76379009306F00706013E4E
:106A0000009BAB4296DD4846814610F8013B202BA7
:106A1000FAD02046F8F7C2FA8246042E04D8DFE8FE
:106A200006F0031010161F004846F9F7C9FB0AF8D4
:106A3000050048462C2143F03BFB013500F10109DC
:106A4000DEE74846F9F7BCFB2AF81500F1E700231A
:106A50000A2200214846F9F7EBFA4AF82500E8E750
:106A60000123F5E70C4932463846FCF7A4FEFDE663
:106A70003146384603B0BDE8F04FF1E553780608DB
:106A8000F4CB0508A17806087E9F06087F6F0608EC
:106A90009678060898BD050866780608F16B060822
:106AA00037B504460846019140F0FAFF01990546C2
:106AB00002462046F9F76CFA70B9625D1046F9F7A4
:106AC0002DFA00B932B901352C442046013403783F
:106AD000202BFAD003B030BD0020FBE72DE9F04FAA
:106AE0000C4695B03449054620461746FFF7D8FFB7
:106AF000064600284FD131492046FFF7D1FF064610
:106B000000284AD12E492046FFF7CAFF0646002832
:106B100045D12C492046FFF7C3FF0646002840D147
:106B200020462949FFF7BCFF0028064612BF08246B
:106B3000264601240FB144F0100424493046FFF7E3
:106B4000AFFF80B344F02004214B1B790BB901F057
:106B5000F9FAF8F7A3FC14F0090F00F01E831D48A2
:106B6000FAF7ACFE0020FCF7B9FA14F4807307932F
:106B70003CD11948FAF7A2FE1848FAF745FE04F08E
:106B80001803182B05D11648FAF798FE1548FAF79E
:106B90003BFE01232BE00124CCE70224CAE70424B6
:106BA000C8E78124C6E710493046FFF779FF00287F
:106BB000CAD044F48074C7E7C2780608C9780608CA
:106BC000D1780608D7780608E8740608FD7106082B
:106BD000D4990020E5780608ED78060805790608BE
:106BE0001179060839790608E0780608002306932B
:106BF000FAF79AFD04F01003BC49BD480593FAF773
:106C0000ABFDBC49BC48FAF7A7FD04F48473082B1C
:106C100007D1BA492846FAF7AEFDB8492846FDF72C
:106C200087F914F0800309930ED1B54B93F83C21FA
:106C3000002AB44A03F59E7306BF012113460021C2
:106C4000B14A2046FAF774FDB0492046FBF7B4FD7F
:106C5000AF492046FAF752FFAE492046FAF745FE03
:106C6000AD4BD3F800B0AD4B1B680493059B002BD4
:106C700040F0D581AA48FAF721FE059EA94B08935A
:106C80009946049BDFF840A36BEA03034FF000082A
:106C90000A9359F8047B002F40F0C381049BDFF86E
:106CA0002C9363EA0B0A089B53F8042B0392089376
:106CB000002A40F0E0819C4B9C4A9D492046FBF70E
:106CC00059F8099B002B40F07A82DFF80493DFF833
:106CD00004A399F800209AF80030964E9A4214BF07
:106CE00001210021944A20460CBF4FF001084FF0CB
:106CF0000008FAF7EFFD9AF80030904A06EB83039C
:106D00000746D3F8D03641462046FAF797FF99F860
:106D100000308A4A06EB83064146D6F8D036884EC4
:106D20002046FAF705FDD6ED007A864AF5EE407A60
:106D3000F1EE10FA0CBF012100212046FAF7F8FC11
:106D40003B4632468049814F814E2046FBF702F98F
:106D5000804B01936FF07F4200923A683168204681
:106D6000FBF7D4FC7C4B019340F202220092BA68FC
:106D7000B1682046FBF7CAFC059B002B40F0AA81B6
:106D80007648FAF79BFD059A75487649DFF848C2C0
:106D90000826012710F8013B11F8018B03F1500E72
:106DA000EE440EF8208C1CF801EB0EF15009E9447A
:106DB00009F8108C2FB1A3EB0E0EDEF1000747EBA4
:106DC0000E07013EE6D187F0010120468DF83860BC
:106DD000FAF780FD644A8DF8486010AB39462046CA
:106DE000FAF72CFF604A0CAB39462046FAF7A0FCB4
:106DF0005E4A5F4B02F5F0712046FBF78DF95D4A64
:106E00005D4B02F5F0712046FBF7D0F9574A5B4B1A
:106E100002F5F0712046FBF711FA594B594A5A49CD
:106E20002046FAF723FF594B594A5A492046FBF7A7
:106E300029F8594A594B02F284412046FBF728F9B8
:106E4000574B584A58492046FBF7FEFA574B584AC9
:106E500058492046FBF798FA059B002B40F03C81EF
:106E60005548FAF72BFD554FDFF870814FF0000BB6
:106E700041460222384643F0DAF8002814BF0121C7
:106E80000021039A97F800A020460CBF4FF001099B
:106E90004FF00009FAF71EFDBAF1020F039040F01F
:106EA0001E8198F801204FF0190A40F2EE231AFBD8
:106EB0000232019298F80020414B9A5C00925B46A6
:106EC000404A49462046FAF7B9FE7A783C4B40F2F0
:106ED000EE211AFB021201923A789A5C00925B460C
:106EE000384A49462046FAF723FC79E059690608F2
:106EF000D16E06086A690608EF6E06084576060830
:106F0000CCAA00207E9F0608497906085679060813
:106F10006079060804660608603E0020CC3B00202D
:106F2000AF780608F0C305087D790608909D00201B
:106F30002CAC002098BD0508847906088A790608DB
:106F4000E035002093790608743C00203437002097
:106F5000E83E0020A2790608A9790608B778060855
:106F60009CAC0020A42F0608906C0608F4AA002010
:106F7000A96F060874AB0020B5790608B079060839
:106F8000BB790608C49E0020C4AD0020BF79060866
:106F9000B8A900203CAE0020E4AA0020C879060869
:106FA000D0790608489F002078AF0020D9790608DC
:106FB000B4370020603D0020BB78060894B0002064
:106FC000A03106086A75060866790608727906080F
:106FD000783F0020D9350020809E002094A9002011
:106FE0000BF1010BBBF1120F07F1020708F10208C8
:106FF0007FF43EAF754B224600212846FCF756FB36
:10700000230700F18280724E224631782846FFF72E
:10701000AFFA717822462846FFF7FEFAB3E06D4ECC
:107020002CE63B7823B30A9A012303FA08F31A40AB
:107030000CBF012100210392204632460B93FAF740
:1070400049FC049B63EA0B020B9B1A4214BF01210B
:1070500000213B46524606462046FAF7EFFD0399CB
:1070600000393B46524618BF01212046FAF760FB23
:1070700008F101080DE6039B1B784BB3049B4FF00E
:10708000010808FA07F813EA080F0BD06BEA0303AC
:1070900013EA080F4A46039B14BF01210021204632
:1070A000FAF7CCFD1BEA080F12D01AEA080832469C
:1070B0000CBF012100212046FAF70CFCB8F10001B9
:1070C0000646039B4A4618BF01212046FAF730FBCB
:1070D0000137E8E5404A57E6404B0393C3E698F88A
:1070E00000203F4B9A5C00925B4649463D4A204651
:1070F000FAF7A4FD3A783A4B9A5C00925B46394A1B
:1071000049462046FAF714FB6AE70027F9B22246FF
:1071100028460137FFF72CFA042FF7D1DFF8B080AB
:10712000314F98F800303B70079B33B92F48FAF77E
:10713000C5FB2F492846FFF7EBF9FF233B70F1B25F
:10714000224628460136FFF767FA042EF7D198F851
:1071500001307B70079BA3B92648FAF7AFFB24499F
:107160002846FFF729FA2448FAF7A8FB2348FAF73C
:10717000BBFAFF237B70002015B0BDE8F04FF7F796
:10718000B6BEFF237B70069B002BF4D01C48FAF799
:1071900095FB1C48FAF738FBEDE7A10706D50C4B29
:1071A000224619782846FFF7E3F9E4E76207E2D5BB
:1071B000074B224659782846FFF72EFADBE7034BA8
:1071C000224618212846FCF771FADCE7C278060847
:1071D000C03F0020AF780608B7780608BB780608DD
:1071E000A03106087A75060894050020DD790608A6
:1071F00045760608007A0608277A060844790608C4
:107200003A7A0608507A0608224BB0F5FA6F1A68E7
:107210000346A8BF4FF4FA63B3F57A7FB8BF4FF4C3
:107220007A73D20416D540F2DC52904215D007EEA4
:10723000903A40F2DB529042F8EE677A1FD8DFEDC9
:10724000166A9FED167A9FED160A77EEE67AA7EE9C
:10725000870A7047B0F57A7F02D89FED120A70470F
:1072600007EE903ADFED106A9FED107A9FED100A5D
:10727000F8EE677A77EEE67AA7EE870A7047DFEDD9
:107280000D6A9FED0D7A9FED0D0A77EEE67AA7EE77
:10729000870A70476035002000007A44D62000C07D
:1072A00000E082440000000000407A446610004084
:1072B0000000404200A0BB44D620004000008344B0
:1072C00010B584464FEA810E102312F4004F14BF0C
:1072D0000E2407245200013BCCF8004092B2F44443
:1072E000F3D100EB81128C01035142F821301220BE
:1072F00010BD00BF10B584464FEA810E0424130B65
:1073000003EB430318331201013CCCF8003092B276
:10731000F444F4D100EB01130A01845043F82140F6
:10732000062010BD704700BF704700BF034B00EB45
:10733000400003EBC000407C704700BF48050010D0
:1073400000234722027043708370C370704700BFF0
:10735000704700BF00207047704700BF0020704793
:1073600001207047704700BF704700BF704700BFE3
:10737000704700BF9FED010A704700BF000000008A
:107380000020704703681B69184730B5084B00227E
:1073900093F900405D7801190132CD729D78055551
:1073A000062ADC788C7503F10403F1D130BD00BFEF
:1073B00038EA0508002383700370C3704370704778
:1073C000C36B33B15B68426D9BB29A4205D3D01A4E
:1073D0007047D0E907239A42F9D2C0681044C01A16
:1073E000704700BFD0E909120369914238BFC9183C
:1073F0008A1A016C39B14968013B12FA81F2934251
:1074000004D9981A7047013B981A704700207047BA
:10741000036C13B190F864007047D0E90903181A9F
:10742000B0FA80F040097047C26B10B4034662B1F5
:10743000426DC1685C69881A013A205C5DF8044BB2
:1074400008BF0A46C0B25A657047006A5C69411CB1
:10745000205CDC68A14238BF0A46C0B25DF8044B2C
:107460001A627047836E70B504460D460BB198479B
:10747000B8B1636AA269D554636A2169226C013389
:107480008B4228BF0023636232B3EFF31183502293
:1074900082F31288226C1168C90703D5DBB283F32B
:1074A000118870BD516889B271B9D4E9095085421B
:1074B00018D0A6690644D66018D9281A80B2506040
:1074C000A562002184F86410116841F00101DBB26B
:1074D000116083F3118870BD226ED36843F080037E
:1074E000D36070BD012284F86420D7E72569281A8B
:1074F00080B25060A162E4E7836E03B11847704721
:10750000F8B590F87C30012B1CD0002A164619DD06
:107510000269436A05460F46D41AB442A869A8BF57
:10752000344639461844224642F048FD6B6A2A69BF
:107530002344361BB3FBF2F0002E02FB10336B62C8
:107540002744E9DCF8BD00BF90F87C30012B0DD05A
:10755000036C43B3EFF31183502282F31288026C61
:107560001168C90703D5DBB283F3118870475168EE
:1075700089B270B471B9D0E90954A54219D08669AD
:107580002644D6601CD92C1BA4B25460856200210D
:1075900080F86410116841F00101DBB2116083F3DF
:1075A000118870BC7047026ED36843F08003D360CB
:1075B0007047012280F86420DBB283F31188F0E782
:1075C00005692C1BA4B254608162E0E770B5094CD8
:1075D000236873B10546002606E099681A681E7391
:1075E00021609047236823B15A68AA1A002A1846D6
:1075F000F3DA70BD34B5002070B5214C2378012B2F
:1076000000D070BD1F4B1B68002BFAD01E4D2B689D
:1076100028465B6898470028F3D01C4B1C4E1A681C
:10762000338892889A420ED21A4B1B4A1B785268B2
:107630000021217003F00203002AE2D0E3B91368AD
:1076400092881A8370BD1549096800224968EA6268
:107650002A6803FB01F12846D36898470E4A33880D
:10766000526801333380002ACBD01368928859695D
:107670000A42E6D05A8370BD13689288FAE700BFC9
:10768000902F0020E4200020E8200020882F0020F8
:107690008E2F00203421002038210020802F002050
:1076A0000C4B1B79DB0700D570470B4A1368002B86
:1076B000FAD04FF47A7101FB03F39842F4D3074BED
:1076C0001B781BB9064B99681B690B60002313607C
:1076D000704700BF34B500207C2F00204C2F0020C5
:1076E000602F00200022FFF7F9B90122FFF7F6B959
:1076F0002DE9F84F1F4DDFF88490DFF884A006468F
:107700000C4638274FF000082046FDF761FDD5F8FC
:1077100000B048B921465846F8F75EFC20B96868C1
:107720002146F8F759FC80B15846F9F7DDFF696842
:1077300011B15046FBF7CCF8A96811B14846FBF7E8
:10774000C7F8F9F7F1FF4FF00108013F05F1100507
:10775000DAD12046FDF73CFD48B9B8F1000F06D15B
:10776000224630460449BDE8F84FFCF724B8BDE88E
:10777000F88F00BF50EA0508667A0608607A0608A6
:107780005A7A060808B5254B1B68DB040AD5B5EE06
:10779000400AF1EE10FA12D19FED210A41F096FE57
:1077A00080B208BDDFED1F7AB4EEE70AF1EE10FA01
:1077B0001CDA9FED1D0A41F089FE80B208BDDFEDA5
:1077C000197AB4EEE70AF1EE10FAE5D49FED177AD4
:1077D000B4EEC70AF1EE10FA14D870EE677A9FED96
:1077E000147A9FED140AA7EE870AE4E770EE677A31
:1077F0009FED117A9FED110AA7EE870A41F066FE10
:1078000080B208BDDFED0E7A9FED0E7A70EE677ADA
:107810009FED0D0AA7EE870ACDE700BF6035002077
:107820000080BB440000404200007A4400E08244F3
:1078300066BEFFBE0060BB4438DFFF3E00407A44B6
:107840000000834466BEFF3E00A0BB44F8B5C54BB4
:107850001D6815F004072DED048B40F0FE80DFED70
:10786000C28AC24C15F0200505D094F8D45015F00A
:10787000020540F08F8023799FEDBD8A13F001034C
:1078800040F0AB8094F80C21002A7ED1D4ED447AEC
:107890009FEDB87ADFEDB86A67EE877A94ED467AA5
:1078A000E8EEA67A38EEC77AC4ED447A84ED457ADC
:1078B00065B194F82021D4F8D830C4F81C310121E6
:1078C0008A4284F80D1118BFC4F81431AB4B1E78EE
:1078D0000E2E00F00681DFEDA47A002794ED4C7A9D
:1078E00094ED4D6A77EEC76AD4ED4B7AA6EE267A10
:1078F00077EE676A84ED4C7AE6EE267AC4ED4B7A31
:10790000C4ED4A7A0FB1C4ED457AD4ED4E6A94EDD8
:10791000507A9FED9B5A94ED516AC4ED4E7A77EE02
:10792000E66AF0EE475AD6EE855AF0EE477AE6EE72
:10793000257A94ED4F0AC4ED507A37EEC07AA6EE60
:10794000070A84ED4F0A41F0C1FD02B282EAE273F8
:10795000A3EBE2739BB2092B7DD9002AACBF0A3896
:107960000A3005B20E2EA4F848515FD0242E09D15A
:10797000DFED847A94ED450A20EE270A41F0A6FD5A
:10798000814B5880BDEC048BF8BD84F80D3184F830
:107990000C317BE7D4ED397AB4F8E830F8EEE77AC9
:1079A000C4ED367A002B00F0898007EE903ADFEDC7
:1079B000746A9FED767AF8EEE77A86EEA78AB4EEDF
:1079C000C78AF1EE10FA88BFB0EE478A237913F028
:1079D00001034FF001053FF455AF94F80C31002B33
:1079E00056D094ED469A78EEC99A002D3AD094F884
:1079F0000D31002B54D0D4ED367A94ED470A5F4B0D
:107A00001E7877EEC07A0E2EC4ED4A7A5FD094F8D5
:107A10002031002B75D0022B02D00FB1012B31D0B9
:107A2000D4ED4A7AF0EE698A012757E7DFED547A00
:107A3000554C9FED540A28EE278A28EE800ABDEEA9
:107A4000C88A18EE103A238041F040FDBDEC048B4B
:107A50006080E580F8BD002584E7444C0127D4ED23
:107A6000328AFFE6454B1E780E2E2AD094F80D512F
:107A70009FED3D8A002DCAD1002FD1D094F820313E
:107A8000002BCBD1F0EE697A0127F0EE698A25E769
:107A900094ED449A012384ED469A84F80C31A2E7D0
:107AA000002F56D0D4ED367A37EEE80A012330EEB7
:107AB000090A84F80D3184ED470AA0E79FED2C8A6E
:107AC00084E7D4ED4A7A94F80D519FED278A9FED13
:107AD0002D0A27EE800A41F0F9FC2B4B0E269880E8
:107AE000C8E7DFED2B7A94ED367A274B27EE277A1D
:107AF0000027BDEEC77ADFED1C7A17EE102A9A80B8
:107B0000ECE6002F8CD094ED4A6A94F82131DFED39
:107B1000216A07EE903A76EE688AB8EEE77A78EE58
:107B2000897AF0EE698AF0EEE77A67EE877AF4EE0A
:107B3000E67AF1EE10FAC4BF68EE266A86EEA78AEE
:107B4000F7EE007A77EEC87A67EEA97AE6EE087A61
:107B5000C4E60A4B1E780E2E7FF462AFD4ED4A7A4B
:107B60003D46B4E7C8A100200000000034B5002065
:107B70009A99993ECDCC4C3FCDCC4C3E94220020DE
:107B80000000C842CDCCCC3D982200206666663FFE
:107B90000AD7233C00401C46F2F74ABB10B5044606
:107BA00041F094FC81B22046BDE81040F2F740BBA2
:107BB00070B50468236A1B69054643B1236AD0F88F
:107BC00094001B69984701282AD002280DD0236A07
:107BD000DA699AB9586958B399692162BDE8704069
:107BE000C3E90522F2F7DEBC2362236ADA691433A3
:107BF000002AF9D1236ADA69002AEBD0216A94F8C5
:107C000024200E7B1433F6B22362D2B996B92846EB
:107C1000F2F74CFC28460121BDE87040F2F70CBC9D
:107C2000236A143B014623622846F2F705FCCEE79F
:107C3000206270BDAB68002BE9D01A689B88538323
:107C4000E5E700212846F2F7F7FB002384F824300B
:107C5000002EDCD0EEE700BF8069002834D0036836
:107C60001A6A127B1ABBD3E904125B6849686AB1CD
:107C700010B4546800220A6022609A885DF8044BB0
:107C800022F003021204120C9A8091E71A8912065C
:107C9000FCD41A89D20708D400220A609A8822F0FC
:107CA00002021204120C9A8082E79A89F1E7826834
:107CB000002AD8D0116892880A83D3E904125B683D
:107CC0004968002AD4D1E1E7704700BF806900B954
:107CD0007047016830B4D1E904424B68646872B1FE
:107CE0005568002222602A609A8822F0030212045A
:107CF000120C9A800B6A1B7B9BB930BC58E71A891F
:107D00001506FCD41A89D20713D4002222609A885F
:107D100022F002021204120C9A800B6A1B7B002BC9
:107D2000EBD08368002BE8D01A689B88138330BCA3
:107D30003EE79A89E6E700BF30B50446006E8389C6
:107D4000A16023F400531B041B0C838195B063795D
:107D5000009113F0040F21794FEA03324FEA032315
:107D600003F48063ADF8083001F0010302F400521F
:107D700014BF4FF480550025002B4FF00003ADF8E1
:107D80000620ADF80C3007BF002208230C23042284
:107D9000ADF804508D07694654BFADF80A20ADF820
:107DA0000A3039F01FFB6279236ED00700F18A8018
:107DB00012F0080F9A8A7FD092B242F008029A829B
:107DC0009A8992B242F400529A812279D10732D52F
:107DD000E06B002800F088800023E26D0793CDE976
:107DE0000B33CDE90F33CDE911334FF4807509938F
:107DF0006369E1680D9505920693626C04924FF4F5
:107E000080634FF480350A9308910E9539F0A0F8FD
:107E100004A9E06B39F032F9E16B236E0A6842F095
:107E200001020A609A8A92B242F040029A8249683C
:107E3000227989B26165920737D5206C00285FD01E
:107E40002369A26D0893A36CCDE90432002240237C
:107E50000025CDE906234FF480314FF480630A9367
:107E60000E91CDE90B55CDE90F55CDE91155099589
:107E70000D9539F06DF8206C04A939F0FFF8226CEB
:107E8000236E506940F080005061106840F0160089
:107E9000106055609A8A92B242F0800203F10C01A0
:107EA0009A820A6842F040020A609A8992B242F4C9
:107EB00000529A8115B030BD22F008021204120C53
:107EC0009A827DE71D498B4223D0A1F54C418B421C
:107ED0001DD001F580618B421DD102200121F2F7F6
:107EE00039F96279236E63E74FF6DF711980D9683B
:107EF00041F02001D960D96841F01001D9609AE7BA
:107F0000DA6842F0800203F10C01DA60C9E701206F
:107F1000E4E70020E2E701F580618B420AD001F539
:107F200080618B4208D001F544418B427FF440AF21
:107F30000520D3E70320D1E70420CFE7001001405C
:107F400030B50446006E21718389A26823F4005382
:107F50001B041B0C8381637995B013F0040F00920E
:107F600014BF4FF480520022ADF804201A031B0204
:107F700003F48063ADF8083001F0010302F400520D
:107F8000002B4FF00003ADF80620ADF80C3007BF12
:107F9000002208230C2304228D07694654BFADF844
:107FA0000A20ADF80A3039F01DFA6279236ED00745
:107FB00000F18A8012F0080F9A8A7FD092B242F0C4
:107FC00008029A829A8992B242F400529A812279E6
:107FD000D10732D5E06B002800F088800023E26DE5
:107FE0000793CDE90B33CDE90F33CDE911334FF4CE
:107FF000807509936369E1680D9505920693626C3B
:1080000004924FF480634FF480350A9308910E95E3
:1080100038F09EFF04A9E06B39F030F8E16B236E75
:108020000A6842F001020A609A8A92B242F0400263
:108030009A824968227989B26165920737D5206CA6
:1080400000285FD02369A26D0893A36CCDE90432A8
:10805000002240230025CDE906234FF480314FF460
:1080600080630A930E91CDE90B55CDE90F55CDE90B
:10807000115509950D9538F06BFF206C04A938F067
:10808000FDFF226C236E506940F080005061106843
:1080900040F01600106055609A8A92B242F0800259
:1080A00003F10C019A820A6842F040020A609A8940
:1080B00092B242F400529A8115B030BD22F008020B
:1080C0001204120C9A827DE71D498B4223D0A1F540
:1080D0004C418B421DD001F580618B421DD10220A5
:1080E0000121F2F737F86279236E63E74FF6DF710B
:1080F0001980D96841F02001D960D96841F0100198
:10810000D9609AE7DA6842F0800203F10C01DA6084
:10811000C9E70120E4E70020E2E701F580618B4236
:108120000AD001F580618B4208D001F544418B42B1
:108130007FF440AF0520D3E70320D1E70420CFE749
:108140000010014038B5074C074DAC4203D3074B34
:1081500001221A7038BDD4E90210A28841F02EFF26
:108160001C34F2E744A9060878B10608D899002023
:10817000302821D0312826D0322828D0332828D0C2
:10818000342828D0352828D0202828D0212828D0C5
:10819000102828D0112828D0122828D0132828D019
:1081A000142812D0152826D0162826D0172808BF44
:1081B0000F2202D0002070470022114B03EBC203B4
:1081C00093F89C0370470122F7E70C22F5E702229F
:1081D000F3E70322F1E70422EFE70522EDE70622A9
:1081E000EBE70722E9E70822E7E70922E5E70A22A9
:1081F000E3E70B22E1E70D22DFE70E22DDE700BF18
:1082000038EA05080123302803FA01F129D0312882
:108210001ED032281CD033281AD0342813D0352849
:1082200011D020280FD021280DD0102810D01128CF
:108230000ED012280CD013280AD0142803D01528E9
:1082400001D0162809D111F0030018BF0120704792
:1082500011F0070018BF012070471728F3D0002045
:10826000704711F0070018BF18467047244B82B0C2
:108270009A7901908AB393F82630DFED226A224A78
:1082800007EE903AF8EEE77A204B127886EEA77A5E
:1082900083ED107AFAB11E499FED1E6AB1F85611AE
:1082A000DDED017A07EE101AB8EE477AF8EE677A3C
:1082B00027EE067AF7EE006A27EE277A002177EE9E
:1082C000266A03EBC202C7EE267A1960083343ED33
:1082D000017A9A42F9D102B070470F4A126812012E
:1082E000F9D593F82630DFED076A07EE903AF8EEFD
:1082F000E77A064B86EEA77A83ED107AEBE700BFAC
:108300008827002055555540C00D00101816001044
:1083100034B5002027D4D2366035002010B5437B19
:1083200082680446581C6073D154627B237B93425D
:1083300006D82AB12368D4E9010198470023637362
:1083400010BD00BF427B42B110B503680446D0E9BE
:10835000010198470023637310BD704730B505686D
:1083600095F800E0BEF1010F95B004468C4608D0A8
:10837000BEF1020F02D119462B6AB3B1002015B02D
:1083800030BD95F90450691CF8D0022DF6DC017956
:10839000009228466246F3F72BFB0028EED02846D1
:1083A00015B0BDE83040F3F79BBACDE90A210DF1D5
:1083B0000F0204920122CDE90532CDE908336CF0B9
:1083C0007F018DF81C308DF830208DF844200D93FE
:1083D0001093129300220023CDE90E238DF80F1085
:1083E000EFF3118C102383F3128803681B6A0BB31D
:1083F000069B04A802461BB1D3691432002BFBD1A3
:108400002B6A6BB1996839B99A4209D0196829B1B8
:108410005B6899680029F7D01433F3E7C3E900409B
:108420005FFA8CFC8CF311882268136A002BFCD154
:108430000120A4E704AB2B625FFA8CFC8CF311885B
:10844000F2F7B0F8F0E700BF30B593B00DF10705D3
:1084500008920022CDE90252CDE906228DF80710DC
:108460008DF81420012109930B920E921092002393
:10847000002204918DF828108DF83C10CDE90C23D2
:1084800001680446EFF3118C102383F3128803680C
:108490001B6A0BB3049B02A802461BB1D3691432BA
:1084A000002BFBD10B6A6BB1996839B9934209D0A3
:1084B000196829B15B6899680029F7D01433F3E78C
:1084C000C3E900405FFA8CFC8CF311882268136AC0
:1084D000002BFCD113B030BD02AB0B625FFA8CFCF9
:1084E0008CF31188F2F75EF8F0E700BF30B405684E
:1084F000EFF3118C102383F3128803681B6AEBB12E
:108500008B6804460A461BB1D3691432002BFBD199
:108510002B6A6BB1986838B9934209D0186828B1B2
:108520005B6898680028F7D01433F3E7C3E900418B
:108530005FFA8CFC8CF3118830BC704729625FFABB
:108540008CFC8CF3118830BCF2F72CB830B58BB0B2
:108550004FF0010C00910021CDE90123CDE9041178
:10856000CDE9061105688DF80CC004468DF820C0D1
:108570000991EFF3118C102383F3128803681B6AAF
:108580000BB3029B684602461BB1D3691432002B21
:10859000FBD12B6A6BB1996839B9934209D019683C
:1085A00029B15B6899680029F7D01433F3E7C3E970
:1085B00000405FFA8CFC8CF311882268136A002B50
:1085C000FCD10BB030BDC5F820D05FFA8CFC8CF329
:1085D0001188F1F7E7FFF0E730B593B000238DF88D
:1085E00007108DF806200DF106010122CDE90332B6
:1085F000CDE90631CDE908320DF107058DF81430CB
:108600008DF828208DF83C200B930E9310930022B8
:108610000023CDE90C23016802950446EFF3118C89
:10862000102383F3128803681B6A0BB3049B02A810
:1086300002461BB1D3691432002BFBD10B6A6BB11C
:10864000996839B9934209D0196829B15B6899686A
:108650000029F7D01433F3E7C3E900405FFA8CFC3C
:108660008CF311882268136A002BFCD113B030BD43
:1086700002AB0B625FFA8CFC8CF31188F1F792FF6E
:10868000F0E700BF30B595B000230122CDE90532F7
:10869000CDE908338DF81C300D93109312930DF132
:1086A0000F030DF107050B928DF830208DF8442053
:1086B0000A93002200238DF80710CDE90E230168EC
:1086C00004950446EFF3118C102383F3128803689A
:1086D0001B6A1BB3069B04A802461BB1D369143264
:1086E000002BFBD10B6A6BB1996839B9934209D061
:1086F000196829B15B6899680029F7D01433F3E74A
:10870000C3E900405FFA8CFC8CF311882268136A7D
:10871000002BFCD19DF80F0015B030BD04AB0B62EF
:108720005FFA8CFC8CF31188F1F73CFFEEE700BF99
:10873000134B1B68B0EB930F14D2B0EBD30F13D2D3
:10874000B0EB131F12D2B0EB531F11D2B0EB931F3B
:1087500010D2B0EBD31F0FD2B0EB132F0ED24FF4C9
:1087600080707047022070470420704708207047CF
:1087700010207047202070474020704780207047AD
:10878000D4200020013902292CD81B4B4FF0280C93
:108790000CFB01FC10B403F5AC746344644493F81F
:1087A000582104604FF0010C022A80F888C003F5BC
:1087B000AC7419D0C9B2114A09015258C3F85C21EE
:1087C00072B1022283F8582100F110014FF4807237
:1087D0004C30A281C3E95C1060465DF8044B7047E1
:1087E0000020FAE70020704793F865216244604654
:1087F00083F86521F1E700BF34B500202C27002065
:1088000010B5036804469B689847FF230122A373B1
:10881000627310BD036810B504461B68984723684F
:1088200001219B6820469847E37B0133E37310BD29
:10883000F0B583B00446089F0193384616460D46AE
:108840003FF02EF92268E6722844A0729769019BD6
:10885000324629462046BC4603B0BDE8F04060479A
:1088600003689B6A184700BF03685B6D03B1184734
:10887000704700BF0368DB6C03B11847704700BF47
:10888000002310B5C37342748A6C016004460373FD
:108890000AB119469047236801219B6820469847F2
:1088A000FF222368A273DB6C012262731BB1204696
:1088B000BDE81040184710BD074A002351688142A7
:1088C00002F1240203F1010303D0102BF6D10020A2
:1088D0007047D8B2704700BFD00200202DE9F04F9A
:1088E000984A537C012B85B021D0022B17D000234E
:1088F0000193954BDFF864B24FF0000A99469BF85C
:108900000030022B15D00AF1010ABAF1030F0BF166
:10891000280B09F10509F2D105B0BDE8F08F937974
:108920002BB19378083B18BF01230193E1E7019332
:10893000DFE799F903506A1C00F0E780EDB22B469F
:108940005FFA8AF6721C0C2102921F46012D4FFA23
:1089500085F800F2D38008237C4A11FB083C0024F0
:1089600005E00134152C02F11C0200F0C7801378D9
:10897000002BF6D15378B342F3D152F80C00002803
:10898000EFD0FFF799FF019B0C2123B1A0F1090360
:10899000072B40F2B8806E4A00F1FF3C0CEBCC0391
:1089A00002EB83031A7F002A40F0A8804FF01402E4
:1089B0001A77029A5A77002800F0A08007461846D6
:1089C000C4EBC403614ACBF8100008EB48089B00D5
:1089D00003EB88031344DB68C360DCF1000303F09E
:1089E00007030CF0070C58BFC3F1000C80F808C057
:1089F0003846F2F7D3F999F904506B1C00F08880DF
:108A0000EDB229465FFA8AF6731CCDE902370F46AC
:108A1000012D4FFA85F851D80C2208214B4B12FB3F
:108A2000081C002404E00134152C03F11C0345D07C
:108A30001A78012AF7D15A78B242F4D153F80C00CF
:108A40000028F0D0FFF738FF019B1BB1A0F109030C
:108A5000072B37D93E4B00F1FF3C0CEBCC0203EB6C
:108A60008202137F53BB4FF01301117702995177A4
:108A700020B31146C4EBC4044246029302EB420207
:108A8000324B039FCBF81410A40004EB82021A446B
:108A90008046D268CA60DCF1000202F007020CF0E6
:108AA000070C58BFC2F1000C81F808C0F2F776F944
:108AB000029B87BB0023CBE9043324E70135EDB2E9
:108AC000AF42A5D2039F002FF4D0214A2423781E61
:108AD00003FB00200024CBF81000CBF81440F1F782
:108AE00093FC5846F1F762FC23461A492246384661
:108AF000F2F76EF901238BF80C3004E70135EDB283
:108B0000BD427FF623AF002775E70123002517E755
:108B10000121002576E7DBF814000293F1F774FCDD
:108B2000DBF81000F1F770FC5846F1F73FFC029BB0
:108B300009491A464046F2F74BF901238BF80C30ED
:108B4000E1E600BF8827002070360020ACAF0508A2
:108B5000D0020020CD7C0108597C01088CB6002091
:108B60004A484B494B4BDFF830C12DE9F04F4FF0ED
:108B7000010A4FF002094FF00408082710262025AB
:108B800040244FF0800E30F8022B12F0010F03D07A
:108B90001960A3F804A0083312F0020F03D0196083
:108BA000A3F80490083312F0040F03D01960A3F85F
:108BB0000480083312F0080F02D019609F80083338
:108BC00012F0100F02D019609E80083312F0200FAF
:108BD00002D019609D80083312F0400F02D0196056
:108BE0009C80083312F0800F03D01960A3F804E0D2
:108BF000083312F4807F05D04FF4807B1960A3F80E
:108C000004B0083312F4007F05D04FF4007B1960E4
:108C1000A3F804B0083312F4806F05D04FF4806BD2
:108C20001960A3F804B0083312F4006F05D04FF4B4
:108C3000006B1960A3F804B0083312F4805F05D00C
:108C40004FF4805B1960A3F804B0083312F4005F9E
:108C500005D04FF4005B1960A3F804B0083312F498
:108C6000804F05D04FF4804B1960A3F804B008334F
:108C7000D20B04D04FF4004219609A80083301F5FA
:108C8000806161457FF47FAFBDE8F08F00B20508D9
:108C900000000240B42300200018024010B504096F
:108CA000013C052C16D80D4A32F8141000F00F03C1
:108CB00041FA03F212F001020ED00120984001386F
:108CC00008403FF019FC064B064A1B5D184402EBB6
:108CD000C00010BD002010BD104610BD00B2050838
:108CE0000CB20508B4230020F8B50C4F97F83430C7
:108CF0008BB10B4C0025A66830790135FFF7CEFF0C
:108D000018B1217DF279F2F779FA97F83430AB4255
:108D100004F18C04EFDC0120F8BD00BF840A0010D0
:108D2000A419002038B5054600780C46FFF7B6FFB9
:108D3000611CC9B2044610B141238371C171204640
:108D40006978F2F737F9AB7820461BB1BDE83840B7
:108D5000F1F720BBBDE83840F1F722BB2DE9F04127
:108D6000FFF79CFF0C4B0D4E1F6805460024BC42CC
:108D700001DBBDE8F08104EB440303EB0608F05C83
:108D8000FFF78CFF854204D121464046BDE8F04103
:108D9000C8E70134EBE700BFDC360020AC3600202A
:108DA000064B53F820303BB11A689B8851690B423F
:108DB00001D0538370471383704700BF38210020D0
:108DC0000D4B0E4A93F800C052F820200123834037
:108DD00003EA0C0361B1003B18BF01233AB11BB198
:108DE000136892881A837047136892885A83704771
:108DF000B3FA83F35B09F1E7342100203821002026
:108E000010B53920FFF74AFF10B140F23E23C3806E
:108E1000064CA36823F0784343F0E043A3600022AC
:108E2000BDE810400A21F2F72FBA00BF0038024017
:108E300010B5054C23681B6998472368002283F806
:108E400036209A6310BD00BFDC14001010B5084C2A
:108E5000236893F8352012B1DB68984700B910BD3C
:108E6000044A236812689A63012183F8361010BD02
:108E7000DC1400102C2100202DE9F041104E114D82
:108E800001244FF05208532716F8010BFFF706FF95
:108E9000202120B1C47180F80680F2F75DF815F842
:108EA000010BFFF7FBFE402118B1C4718771F2F787
:108EB00053F80134E4B2052CE6D1BDE8F08100BFDF
:108EC0002CB5002020B5002038B50C4614F8011B45
:108ED00041B105462B6828461B68984714F8011BCA
:108EE0000029F7D138BD00BF03681B68184700BFD1
:108EF00003682DE9F0415F6A1FB13B46BDE8F041D0
:108F0000184704460D46164600E023689B68204635
:108F10009847B042F9D3002E08DD2E44236815F897
:108F2000011B1B6820469847B542F7D1BDE8F08188
:108F300003685B68184700BF03689B68184700BF59
:108F40000368DB68184700BF03685B69184700BF08
:108F500003689B6A03B11847704700BF0368DB6A68
:108F600003B11847704700BF03682DE9F04116466A
:108F70009A6A04460D460AB1904723685F6A5FB15A
:108F8000324629462046B8472368DB6AC3B12046EB
:108F9000BDE8F041184723689B6820469847B042D7
:108FA000F9D3002EF0DD2E44236815F8011B1B6851
:108FB00020469847B542F7D12368DB6A002BE6D1FB
:108FC000BDE8F081D0E700BF2DE9F04F8E4B1E7851
:108FD0008FB016B10FB0BDE8F08F8C4F3B685905CC
:108FE000F8D58B4D9FED8B7AD5F8FC33C31A07EE7D
:108FF000903AF8EEE77A0446F4EEC77AF1EE10FA0A
:1090000059DA95F80034002BE4D095F804349A0727
:10901000E0D195F80C24002A52D0D5F8100410B1F4
:109020007D49FFF7A1FF002385F80C3495F85434EF
:10903000002B49D195F82836002B40F0FD8095F89B
:10904000B323002A40F07C81744B196895F82936C7
:109050002BB17348D5F82C36834200F0AF8195F8D8
:109060005826704BB3FBF2F3D5F8242613449C42E8
:10907000B0D395F86136C5F824462B4493F85C4686
:10908000E30700F18183A60700F12883600700F160
:10909000F982230700F19C82E70600F1828295F8AD
:1090A000613695F858260133B3FBF2F102FB113318
:1090B00085F861368EE724F07DF8C5F8FC43A0E71B
:1090C00095F85434002BB5D095F85534002B40F06A
:1090D000FF81D5F8B834002B00F02D81DFF85081E6
:1090E000DFF850B108F168094B460027A146A8F502
:1090F000227A1C4662E0012900F03681052E4ED905
:10910000537885F81C3690885388A5F81836911D39
:109110009319C02800F2348200220AEB000EA5F851
:109120001A264148C5F810A60122C5F814E685F8AC
:109130002026AEEB00025B1A934285F821C6C0F2EE
:10914000F981002A40F0CA81384AC5F81406002384
:1091500085F82036C5F808360693DBF80000C5F818
:1091600010A606AB02F11001C5F80046C5F80426AA
:1091700009F0F6F8013000F02382069B0BB10020C5
:109180009847D5F80036C5F80436C5F8004695F876
:109190000C34002B00F0FA80012385F85534013699
:1091A0003744EFF31183502282F31288D5F8B824A4
:1091B000974280F2B780DBB283F31188EB1993F802
:1091C0005864012EEBD97A1CAB1893F85834C3F3CA
:1091D0004111032985F8BC1403F00F0C00F0DB806B
:1091E00013F01003424486D195F820160029D6D0FA
:1091F00095F82116013101F00F01614500F0D7808B
:1092000085F82036CBE700BFC0A1002060350020E4
:1092100034B50020001B374A48B900202C2100201B
:1092200064BB0020A086010004B7002034BB0020EE
:109230008CB900202C060020C44BC5490091A3F135
:109240003F02C827C34904920593C34AC34B85F81C
:10925000BC7306A8F6F73EFDDDF81080002608F185
:109260000103049388F80060049B2922591C04918F
:109270001A70049BEA22591C04911A70049B5A1C10
:10928000049206A81F703EF00BFC471C06A93A4644
:10929000049840F093FE04990122CB1913440493DF
:1092A000CE55049B991804911E70049B9918049143
:1092B0001E70049B991804911E70049B99180491C8
:1092C0001E70049B991804911E70049B99180491B8
:1092D0001E70049B991804911E70049B99180491A8
:1092E0001E70049B991804911E70049B9918049198
:1092F0001E70049B991804911E70049B9918049188
:109300001E70049B991804911A70049BA3EB080328
:1093100004A888F8003032F07BFE85F82866C5F88E
:10932000244657E600224C4695F85564C5F8B82403
:10933000DBB283F3118885F85464C5F8244649E606
:10934000874A85F8B33302F13A03CDE9062385490C
:10935000C5F8BC134FF4327306A8A5F8C03332F039
:1093600057FEC5F8244635E6022E3FF418AF507874
:109370009378A5F81836FF2840F0D980042E7FF6A0
:109380000EAFB2F80300511D9319C2E638F088FE03
:1093900085F8550403E7744BC5F80436734BC5F8DC
:1093A00008360023C5F8004685F8C034EFE6D5F846
:1093B0001006D5F814E6511C9319BAE6D5F8440600
:1093C0008842BFF44CAE95F8B013002940F08E806F
:1093D000D5F84866002E3FF442AED6E900218A4215
:1093E0003FF43DAED5F85036D5F85426E31A9342F3
:1093F0007FF735AE95F84C3695F84D2685F8C23393
:109400005B4B0392114603F13802CDE90632594A0B
:10941000C5F8BC234FF4E47285F8C313A5F8C02344
:10942000D6E90019494500F01584984603F1320B3E
:109430000F78ABEB080A09F1FF3E0B46C1F1010CB6
:1094400003E013F8012FBA4203D173450CEB03007C
:10945000F7D183B2012B5FFA8AFA00F267839A454B
:1094600080F09683494500F0F583D845E0D3039B0F
:109470007BB995F8C23363F07F0385F8C233D6E930
:109480000019494505D195F8C23343F0400385F8EA
:10949000C233069B384E06A89B1B85F8BD3332F0BD
:1094A000B7FD95F80C244AB1D5F8100418B106F1AF
:1094B0005701FFF759FD002385F80C3495F84D3618
:1094C000C5F85046013385F84D36C5F8244681E588
:1094D00038F0E6FD85F8550406462CE7039240F087
:1094E0006DFDD5F81006039A10442DE695F84C163C
:1094F00085F8B02385F84D26204A013182FB010210
:109500000A445211C2EB82128A1A95F8B10395F8F7
:10951000B21385F84C26A3F5687200FB0121A3F570
:109520001F73C5E9ED21C5F848361E4657E7D11C23
:109530009319EEE51A46039340F040FDD5F8102646
:10954000039B1344C5F8103629E600BF30B900204C
:109550002B350020047B0608F87A0608F07A060806
:10956000F6B80020C8057DEAF5B900200000F6FF36
:10957000F8B80020C8007DEAF1B8002083200882F6
:10958000774BC5F80436B5F81836A5F80836032326
:1095900085F8C0344FF6F673C5F80046A5F80A36CC
:1095A000F5E5704B7048C5F8BC0303F13B01C822D8
:1095B00006A80693079185F8C02332F029FD6EE5D1
:1095C000D5F800360222591CC5F800161A70D4E5E9
:1095D000D5E93701B5F8FE30B5F8002185F8C203AA
:1095E000242707FB03F3070E85F8BF73070C85F8E4
:1095F000C07302EB820264273233B3FBF7F385F8C2
:10960000C833C3F3072385F8C733000A530085F82E
:10961000C10385F8CA33080E41F2C81385F8C61392
:1096200085F8C303C2F3C712080CA5F8BC33090AB6
:1096300002234E4E95ED450A079685F8C92385F815
:10964000BE3385F8C40385F8C5133FF03FFF484A91
:1096500003469342A8BF134623EAE373B3FBF7F331
:1096600003F57A73C3F307222E3E85F8CB2306A8B1
:1096700095F80221069685F8CD2385F8CC3332F093
:10968000C7FC09E5394B95F804900793C822A3F16C
:109690003D08A5F8BC2319F001094FF02102CDF8CF
:1096A000188085F8BE2300F09B82B5F89E265005F1
:1096B00040F18A822F4A393B1068C5F8BF030693F0
:1096C000069B0022591C06911A70069B2A4A06A87E
:1096D0009B1A85F8BD3332F09BFCDAE4234A0792EB
:1096E00095F8773640F6C822A5F8BC23082285F8FD
:1096F000BE23002B00F05B82204B1B781BB1204A5D
:109700001288B2FBF3F30A220533B3FBF2F3C3F37F
:10971000072285F8BF2385F8C033D5F89036194E57
:1097200006960A2293FBF2F3C3F3072285F8C233AD
:1097300085F8C1230FF032FDB5F89886034698FAF4
:1097400098F8043685F8C63306A8B5F89A36A5F811
:10975000C483069685F8C33332F05AFC96E400BF02
:10976000F5B90020F5B80020C8040B0030B900207E
:1097700020A10700187B0608F1B800200FA90020DF
:1097800010A90020F7B800209F4AB5F96636079265
:1097900040F6C802A5F8BC23B3F5E16F4FF01E02F6
:1097A00085F8BE2340F37C819AB2A2F561631BB2B7
:1097B000B3F5E16F31DDA2F5E1531BB2B3F5E16F13
:1097C0002BDDA2F52853303B1BB2B3F5E16F24DD4E
:1097D000A2F561531BB2B3F5E16F1EDDA2F58C4318
:1097E000503B1BB2B3F5E16F17DDA2F5A843603B18
:1097F0001BB2B3F5E16F10DDA2F5C443703B1BB2A1
:10980000B3F5E16F09DDA2F5E1431BB2B3F5E16FFA
:1098100003DDA2F5FD43103B1BB207EE903A9FED2E
:109820007B7AF8EEE77A67EE877AFDEEE77A17EE55
:10983000902AC2F3072385F8BF33B5F9643685F85B
:10984000C023B3F5E16F40F3E5809AB2A2F56163FE
:109850001BB2B3F5E16F31DDA2F5E1531BB2B3F5F5
:10986000E16F2BDDA2F52853303B1BB2B3F5E16F5E
:1098700024DDA2F561531BB2B3F5E16F1EDDA2F545
:109880008C43503B1BB2B3F5E16F17DDA2F5A84343
:10989000603B1BB2B3F5E16F10DDA2F5C443703B32
:1098A0001BB2B3F5E16F09DDA2F5E1431BB2B3F5DD
:1098B000E16F03DDA2F5FD43103B1BB207EE903ACA
:1098C0009FED527AF8EEE77A67EE877AFDEEE77A57
:1098D00017EE902AC2F3072385F8C133B5F968362D
:1098E00085F8C223B3F5E16F51DD9AB2A2F5616349
:1098F0001BB2B3F5E16F31DDA2F5E1531BB2B3F555
:10990000E16F2BDDA2F52853303B1BB2B3F5E16FBD
:1099100024DDA2F561531BB2B3F5E16F1EDDA2F5A4
:109920008C43503B1BB2B3F5E16F17DDA2F5A843A2
:10993000603B1BB2B3F5E16F10DDA2F5C443703B91
:109940001BB2B3F5E16F09DDA2F5E1431BB2B3F53C
:10995000E16F03DDA2F5FD43103B1BB207EE903A29
:109960009FED2A7AF8EEE77A06A867EE877AFDEE91
:10997000E77A17EE903AC3F3072285F8C323244A07
:10998000069285F8C43332F043FBFFF77CBB13F536
:10999000E16FE3DA9AB202F561631BB213F5E16F8E
:1099A000DCDA02F5E1531BB213F5E16FD6DA02F50A
:1099B000285330331BB213F5E16FCFDA02F5615350
:1099C0001BB213F5E16FC9DA02F58C4350331BB2B9
:1099D00013F5E16FC2DA02F5A84360331BB213F549
:1099E000E16FBBDA02F5C44370331BB213F5E16FCC
:1099F000B4DA02F5E1431BB213F5E16FAEDA02F51A
:109A0000FD4310331BB2A9E730B9002058A08B41A9
:109A1000F9B8002013F5E16FBFF650AF9AB202F526
:109A200061631BB213F5E16FBFF648AF02F5E15376
:109A30001BB213F5E16FBFF641AF02F52853303387
:109A40001BB213F5E16FBFF639AF02F561531BB2DC
:109A500013F5E16FBFF632AF02F58C4350331BB202
:109A600013F5E16FBFF62AAF02F5A84360331BB2CE
:109A700013F5E16FBFF622AF02F5C44370331BB29A
